:020000041800E2
:1040000000800020AD400018D3400018D5400018B3
:1040100000000000000000000000000000000000A0
:10402000000000000000000000000000D740001861
:104030000000000000000000D9400018DB4000181C
:10404000DD400018DD400018694B0118DD40001804
:10405000DD400018DD400018DD400018DD4000188C
:10406000DD400018DD400018DD400018DD4000187C
:1040700015170118DD400018DD400018DD4000185C
:10408000DD400018DD400018DD400018DD4000185C
:10409000DD400018DD400018034885460DF006FBA2
:1040A00000480047B52C01180080002000200C4972
:1040B00008600C480C49086001200C4908600C4855
:1040C0000C4988470C480D4908600D4988470D4840
:1040D0000047FEE7FEE7FEE7FEE7FEE7FEE700003B
:1040E0002C100040254000180C0000190000001999
:1040F000004000181D280118944801005410034086
:10410000F92E011899400018FEB531210902002549
:1041100040182C46884F01900EF032FE401C0007DC
:10412000000E0090864E854830600198F061C821ED
:104130000098B847304641698907FCD54169890430
:104140008E0E03210903C16164210098B847641CE5
:104150007519E4B2042CDFD3A808FEBDF8B5784C7D
:104160007848A06025210120FFF7CEFF06460421F4
:104170000320FFF7C9FF074608210720FFF7C4FF08
:10418000850135430C210B20FFF7BEFF86013E431E
:104190000F210E20FFF7B8FF07036B482F43A060E5
:1041A00013211220FFF7B0FF050335431721162016
:1041B000FFF7AAFF86043E431B211A20FFF7A4FF46
:1041C00087042F431F211E20FFF79EFF050635435E
:1041D00023212220FFF798FF060627213E430846A9
:1041E000FFF792FF81010143256126636163574810
:1041F000574A866011434560C160F8BDF8B5504824
:104200004030C1694906CA0E0E2A00D114224C4D15
:10421000E96989040C0F4D49082CC96803D10B0BBF
:104220001B0700D10F2401239B075F6A9E143743AD
:104230005F625F6AB7435F62464B2B62464B6B62BD
:10424000464BAB63464BC360464B0361464B4361F1
:10425000464B8361464B92001A43C2611122D20140
:104260000262444A42620722120482621722D20288
:104270000263414E354A0B0CB34209D11368C36047
:1042800050682861906828630805000D686303E0A2
:1042900000F028F8FFF762FFA002E8613748686283
:1042A00037482860F8BD0007000F254A8102D16118
:1042B00026490F231B03CA6800039A430243CA60BE
:1042C0007047224948601E49086170471F4988604D
:1042D0001B490863704700051C49000D8860184998
:1042E00048637047F8B50EF04BFD401C0007050E03
:1042F000134C24484034E0602148114E3838306077
:104300002148F061616B8805FCD50B4F642128467C
:10431000B847606BFC2108401A49703140180B49BE
:104320000860E0600020F06114212846B847144876
:1043300008303060F8BD0000490700005A803200A4
:1043400000C002400026730000266E00D88F0020B7
:104350000000A55A11E34500280612038B23000034
:10436000907D430072D50B05B26609001A33E00058
:1043700001FFDA07087FFF07A55A00002806120789
:1043800052922200907C430011020000174A41081B
:104390001140401A1649024680080A400840101889
:1043A000010908181349084013494843000E704793
:1043B0000CB5002807D011A106C968442038019225
:1043C0000091C07F0CBDFF20F5300CBD0CB501463F
:1043D0000AA005C80192009000206A46135C8B4237
:1043E00003D3401CC0B20728F8D30CBD5555555512
:1043F000333333330F0F0F0F01010101FA96644B72
:10440000321E1400F8B50746000214460E46002579
:10441000C01D0FF0D8F9217843233F2818D01F285A
:1044200016D0FA49BA008A58B300D158A1420DD02B
:104430000121B140014201D002250EE00125D450F6
:10444000C9B22A46384602F0DBFB06E0012504E04B
:104450000C3C2289384602F0EBFB2846F8BD70B5CB
:104460000D46044602F0E8FCC0B2294606F03AF9CF
:1044700000281AD0112809D004DC012806D00C2805
:1044800014D103E0192801D01A280FD1DF4BA20064
:10449000995840318D79AD0608D5487DFD242040DE
:1044A0004875985880680FF040F970BD9030C2B2DE
:1044B0000221204602F0CDFB70BDF7B5040205468F
:1044C000E61D30460FF07FF93F2822D01F2820D06C
:1044D0001F2130460FF04CF9CC4FAE00B95902986D
:1044E0008881284602F0A8FCC0B2019904F07DFB47
:1044F00000280DD09030C3B201212846029A02F064
:1045000097FBB859002803D1E01D00210FF030F9C6
:10451000FEBD432301212846029A02F089FBFEBD1D
:10452000F8B50502ED1D0C4628460FF04CF93F2862
:1045300031D020462030017A2E0ACA0719D0827A5B
:10454000304602F0EFFCB14FB5007959206948635D
:104550007959606A886378591022AD4B214614302E
:1045600098477859214610221431A94B2430984796
:1045700004E000221146304602F0D4FC3502082443
:10458000681D0FF020F9A0430146681D0FF0F0F8F8
:10459000304604F004F9F8BDFFB5150A16460F467B
:1045A0000A4681B000212846FFF72CFF0446012867
:1045B00022D13978072922D004DC032907D0042925
:1045C0001AD10BE0182928D0192915D142E0284624
:1045D00002F032FCC0B204F0CCFB05E0284602F049
:1045E0002BFCC0B205F0AEF9002805D09030C2B265
:1045F0000021284602F02DFB204605B0F0BD012326
:104600003246844804990FF077F80646284602F0AF
:1046100013FCC0B207F064FD27E0284602F00CFC52
:10462000C0B2694606F074FC07000ED17320022365
:104630003246000104990FF05FF8694649784170ED
:104640006946097801700FF070F8002F00D090379C
:10465000FAB2CDE76F4801233246283004990FF0B3
:104660004BF80646284602F01FFC307030460FF02B
:104670005CF80022BCE770B515460C4610460FF0FA
:10468000A2F82B0A00253F280BD0E188062908D183
:10469000000701D5022504E02278211D184601F00B
:1046A000C7F9284670BD70B5154610460FF08BF857
:1046B0002C0A3F2812D05548A10040588068002895
:1046C0000CD00078092809D145220221204602F0A9
:1046D000C0FA2A463B212046FFF7EFFE002070BDBE
:1046E000FFB50546000281B0C01D0FF06CF83F28F1
:1046F00083D0464FAE00B8598468002C15D020787E
:10470000092812D1284602F097FBB959029A403184
:10471000497DC0B2C9438907C917491C002A0FD077
:10472000002903D0A11C06F045F866E76178002255
:10473000284602F0C1FEA11C2846FFF790FE5CE768
:10474000002903D0002106F035F804E06178012249
:10475000284602F0B1FE48220221284602F079FAEA
:104760004BE7FFB5160A17460C460A4681B00221F0
:104770003046FFF747FE054601285ED1207809281C
:1047800002D0172859D149E02389E2886188A0889E
:1047900002F0F4FB002813D01C48B1004158084631
:1047A0004030427D920702D4807980061CD4049860
:1047B000C0B2072806D0A11C3046FFF750FE3CE0EF
:1047C000402236E01348C98908233A46801D0EF07E
:1047D00093FF61880180A1884180E18881802189DF
:1047E000C1800EF0A2FF28E00EF0B4FE0106090E13
:1047F00000D101216170A21C304602F074FE054810
:10480000054A3946E9300EF0F7FF16E08C9000209B
:10481000190F00000907000030750000304602F053
:104820000BFBC0B2611C06F086FB002805D090305F
:10483000C2B20221304602F00CFA2846DDE6000042
:10484000F8B51E460546F84B174680001858002458
:10485000069A012903D11A21403014460170012221
:104860000821284602F0CCF9284602F0E5FAC0B249
:1048700023463246394604F0CAFE002805D090305F
:10488000C2B20121284602F0E4F9F8BD70B516461F
:104890000C46054602F0D0FAC0B2002C08D03146D2
:1048A00004F00AFF01220821284602F0A9F970BD90
:1048B000002104F001FF96220121284602F0C9F9E7
:1048C000D94AA800105800214030017070BDF3B5DE
:1048D00081B001980F468100D348212346580198A2
:1048E000F18902023569D148D21D0EF005FF044658
:1048F000077002213B000CF057FF080537373714CB
:1049000037100C37A87CC006C00E6070403631707E
:104910002AE0019802F0FAFA16E0132040363070CF
:1049200022E0687C012802D1287E01280BD0403685
:10493000B079012280060028E87D0BDB022805D033
:10494000042803D00FE0002060700DE0287C0228CE
:104950000ED108E000280BD0012809D0042802D18C
:10496000287C022804D0617020460EF0DEFEFEBDD9
:104970006270F9E7F7B50F4606468100AA48320291
:104980004558AA48E9891E23801CD21D0EF0B4FEAA
:1049900004460770B81EA64F03000CF005FF06087A
:1049A000042E1E231C2E02980078A0700DE02869AA
:1049B0004030C17BA170427CD207D20FE270407CB4
:1049C000C207D20F304602F0ADFA4035A879BF21B8
:1049D0000840A87111E01C2200E01722A01C0299D7
:1049E000B8470AE01022A01C0299B84710222846B6
:1049F00024300299B8470020A86320460EF095FEA7
:104A0000FEBDF8B5884A81005558884F2E4620369D
:104A1000F17F04028907E137002903DAE11D3846F6
:104A20000EF03DFFAA8F0A204243E11D38460EF0EA
:104A3000E3FEF07F02210843F077F8BD70B505462C
:104A4000794B800019583F22525C002492071CD5F4
:104A50008A8F784CA24214D05204120C8A87A24248
:104A60000DD38C8718582A02C18970481E23801CD8
:104A7000D21D0EF041FE082101700EF056FE0324F7
:104A800000E001242846FFF7BCFF204670BDF0B5CA
:104A90000446654BA2009A5801201269137DD57E09
:104AA0002B409E46537D157F2B409C46937CA50052
:104AB000DE075D4B5B591B69DF7E1D7D3D401F7F1F
:104AC0005B7D3B401D43002E05D0537EDB0702D0AB
:104AD000002D00D10020544BA4001B59ED071B6989
:104AE00040335C7C002D07D001252C435C740129E8
:104AF00005D0022903D007E064086400F6E74032DD
:104B0000527CD20700D10020032901D0042906D10C
:104B10007146490703D46146490700D40020F0BD1F
:104B20007FB50646404980000C586846007A1D460D
:104B300000281BD002AA03213046FFF71BFF002DDF
:104B400002D03046FFF75DFF00220121304602F01F
:104B500080F820690025002802D00EF067FD25614D
:104B6000304601F015F9403425707FBD0022022146
:104B70003046FFF7FFFEE7E770B52B4B82009A58EF
:104B80001469403215782E46143E33000CF00CFEAA
:104B9000060C04090609090C162000E01820107004
:104BA00070BD1423137001E0142DF9D14034237C1F
:104BB000DD0705D015201070207C4008400006E07D
:104BC0009D0706D517201070207CFD2107E020747A
:104BD00070BD5B0705D519201070207CFB210840B3
:104BE000F5E7002904D000231A46FFF799FF70BDAE
:104BF000002100F0B7F870BD30B40B4B82009C5818
:104C000085005B5922691B694033002908D0157D56
:104C1000D27E154014221D744034227030BCABE7A4
:104C2000557D127FF5E700008C90002013070000EF
:104C3000190F0000B80B0000F8B50E46FE4A8100BF
:104C4000545805022034E17FFC4FC907002907D0E2
:104C5000E91D38460EF023FEE07F40084000E07773
:104C6000304608380EF061FD30780B280AD0052850
:104C700008D0E91DF24A38460EF0BEFDE07F012162
:104C80000843E077F8BDF3B50646EB4980000D58C0
:104C900081B02C6940352878102807D0112803D01E
:104CA000122801D013280FD1102028704034207C06
:104CB000C1070AD0C0B24008400020740721304626
:104CC000FFF705FE11202870FEBD81072CD5FD21C0
:104CD00008402074DB48112287690821304602F021
:104CE00080FB0090002F04D01022D74B3946401C87
:104CF000984730460099FFF79FFF08220921304668
:104D000002F06FFB0746CF48CE49203000791E31B4
:104D1000C007C00F78700622CB4BB81C98473946A5
:104D20003046FFF789FF0AE041070CD5FB21084018
:104D300020741320287006213046FFF7C8FD28781C
:104D40001028B4D0FEBD0298002804D00146304699
:104D5000FFF752FFFEBD002301461A463046FFF71B
:104D6000DFFEFEBD30B4B44B82009C5885005B5919
:104D700022691B694033002908D0557D127F1540F8
:104D800010221D744034227030BC7CE7157DD27E29
:104D9000F5E710B58100A84AA74B51588000185874
:104DA000096900694A7C00244030012A02D10A7E48
:104DB000012A07D08A7C520706D44A7E520703D4C0
:104DC00084730FE002220CE0CB7D0A7C032B05D01C
:104DD000032A03D0012B03D8012A01D8002200E0C6
:104DE0000122827308464030827B002A06D0012AC5
:104DF00001D0022A03D10422C27300E0C4738A7C6A
:104E0000D20706D0497EC90703D0C17B01221143D6
:104E1000C17310BD00B5884A800010580029006990
:104E200007D0417F0B000CF0BFFC06060608060801
:104E30000C11817DF6E7012000BD4030C07B4007AA
:104E400002E04030C07B0007C00F00BD002000BD65
:104E5000F7B5009816468500774800244759224642
:104E60000821009801F0CCFE062E0AD0112E0AD09F
:104E7000222E0AD0002E0AD090363406240E06D0F8
:104E80000BE0222409E0232407E0242405E038462F
:104E9000403081790822114381713E4640360099A5
:104EA00030780A020E2830D00F282ED01A282BD1A5
:104EB000002C22D1604F01237859D21DC1895F484F
:104EC000DA380EF019FC009A0021032A12D27A591E
:104ED000002A0FD040329279530700D50121920762
:104EE000920F022A02D0032A04D101E0042200E03A
:104EF0000C22114301700EF018FC00203070224685
:104F00000121009801F0A5FEFEBD002C06D0002373
:104F1000224601990098FFF703FEFEBD0F2823D11A
:104F20003869817CC9071FD0407EC0071CD0424829
:104F30001E234059D21DC1894048DE380EF0DCFBEB
:104F40000446072020701C223F4BA01C396998475B
:104F500020463D4B0822002114305C339847002046
:104F6000608220460EF0E1FB0198002804D0012168
:104F70000098FFF7F7FEFEBD00210098FFF73CFE0A
:104F8000FEBDF0B505462C4A8000105885B02E4F66
:104F9000046903AE002918D00822214601A82E3149
:104FA000B847082221461E313046B847FF2000028C
:104FB00085430320000228180090244B012201A9F8
:104FC000204601F065FC05B0F0BD0822214601A88D
:104FD0001E31B847082221462E31E5E7F7B50546D0
:104FE0008100154816464058174F8AB010220021FC
:104FF000046902A85C37B8471022002106A8B84708
:105000000B98114F002844D00121284601F03CFFA5
:105010008079694608720021284601F035FF8079C1
:10502000694648720021284601F02EFF01460622FB
:1050300006A8B84701210BE08C900020F307000080
:105040003075000064900020190F0000EB5000182C
:10505000284601F019FF0146062207A80230B8478A
:10506000012269468A7202A80330062221461031C5
:10507000B84702206946487404A802300622214637
:105080001731B847FF2000028543002E19D00120B8
:1050900018E00021284601F0F7FE80796946087281
:1050A0000121284601F0F0FE80796946487201210D
:1050B000284601F0E9FE0146062206A8B84700216D
:1050C000B9E7022000020543FE4801950090002E3A
:1050D00002D021461E3101E021462E3106AB02AA44
:1050E000204601F086FC0DB0F0BDF7B50346D7B2FF
:1050F000F548B900405886B0002833D041680029EF
:1051000030D009780A292DD104464034A1798D0682
:10511000ED0F002B03D09033DAB200235CE0066978
:10512000100A0006000E1FD001282CD0022844D0FF
:10513000032817D1384601F0E9FE04460246E34B46
:1051400001A8079998471020021B01A8DF4B0019FE
:1051500000215C339847002D55D001AA0121384623
:10516000FFF794FB09B0F0BD10223046D74B1E303C
:1051700007999847A0794006F4D401222946384679
:10518000FFF72CFFEEE74806ECD4079800901122B9
:105190000321384602F025F906461022CB4B401C6D
:1051A0000099984731463846FFF746FD002D02D05A
:1051B00008202070D6E70720FBE73046C34B1022BB
:1051C0003E308A330799984700280AD00421384690
:1051D00000F0F1FD0123642229463846FFF7A0FCC8
:1051E000C0E7A0794006BDD40E202070002D05D068
:1051F00031461E31384600F0EBFDB3E7002138465A
:10520000FFF7BFFEAEE7002003460146009001AA6B
:105210003846FFF715FBA5E7F8B50D460746AA493E
:1052200080000E584620805D002480064FD56878A7
:1052300004280FD8E878410707D04007400F01281D
:1052400003D0042801D0052804D1A878002803D071
:10525000012801D00A243AE02879C01F0A2801D386
:10526000062434E03846FFF7E9FB002802D0032883
:105270002DD12BE03069002829D19548007901070C
:10528000890F0ED0E97809070DD440070BD46320AD
:105290006946087003246A4621463846FFF76AFBD0
:1052A00015E0052413E03902CA1D08238948C91DE9
:1052B0000EF022FA06460A2030700622691C834B43
:1052C000701C984730460EF030FA00E00924204662
:1052D000F8BDF3B581B00F4601987B4980000E58A8
:1052E00078780024042859D8F878410707D0400777
:1052F000400F012803D0042801D005284ED1B878EA
:10530000002801D0012849D13879C01F0A2847D286
:1053100035464035A879800650D4287801284DD1EB
:10532000781C00F011FD002838D030690622791C65
:10533000664B173098473069417E090706D5807C57
:10534000000703D5A87940210843A871A879400631
:1053500003D45F480079400726D5019800F007FD87
:1053600000281DD03069817D0198FFF790FB00284F
:1053700018D00198FFF70DFD00210198FFF74AFDB5
:10538000002811D00520287030694030817B002929
:105390000CD004210198FFF79AFA0FE00A240DE0DF
:1053A00006240BE0082409E0032407E0417C0422E2
:1053B000114341740021019800F02AFD2046FEBDF2
:1053C000F8B50746404A800014582069002819D0D3
:1053D00025464035AA793D4B9206D60F10223E3025
:1053E000491C9847287807280CD1002E0CD005209E
:1053F000287020694030407C400703D500213846A2
:1054000000F006FD0020F8BD216938461E3100F08D
:10541000DFFC08202870F5E770B506462A4A8000B0
:1054200014582069002815D04034A279274B9206E1
:10543000D50F10222E30491C98472078082809D112
:1054400006202070A079400604D400222946304668
:10545000FFF7C4FD002070BD08B54A78511E0E2923
:1054600000D3082270210A4369460A701649830056
:10547000C9580B69002B07D0403189790023890670
:10548000C90FFFF74DFB03E06A460321FFF772FAED
:10549000002008BD70B504460B4A80001258134620
:1054A000403318781D4615280AD110691022074B81
:1054B000491C9847A8798006C10F2046FFF75CFB7E
:1054C000002070BDEB5000188C900020190F0000D8
:1054D0008490002012070000F0B50546FF4A8000C6
:1054E000145887B026464036307816281ED1887862
:1054F0004A78000210436A46108204A80822F84F36
:105500000230C91CB847102268462169B8472846AE
:1055100001F0FCFC6A46907607212846FFF72AFA3C
:10552000B0798006C10F2846FFF726FB002007B0A0
:10553000F0BD70B50446E94A800012581346403366
:1055400018781D4617280AD110691022E44B491C0F
:105550009847A8798006C10F2046FFF70DFB002071
:10556000AFE7F0B50D460646DC4980000C5887B021
:10557000274640373878182817D10622D84BA91C5F
:1055800004A89847687869468875D54B1022684604
:10559000216998476A4605213046FFF7EBF9B8794B
:1055A0008006C10F3046FFF7E7FA0020BFE770B56D
:1055B0000546CA4A800014584034207819280AD178
:1055C0004A1C06212846FFF7D5F9A0798006C10FAD
:1055D0002846FFF7D1FA002073E7F8B506468700A2
:1055E000BE480D46C059009048780024410709D0B4
:1055F0004007400F012805D0042803D0052801D01A
:105600000A242DE0304601F023FC002828D1304642
:10561000FFF714FA002823D1687800070DD4B148A9
:105620000079400709D463206946087003246A465C
:1056300021463046FFF79EF912E0009800690028E5
:105640000ED1A6483202C0590123C189A648D21DF5
:105650000EF052F86978C906C90E01700EF065F8AF
:105660002046F8BDF3B581B00F4601989B498000F4
:105670000E583F20805D0025410701D5452549E0B2
:10568000800701D5692545E0384600F05DFB00281C
:1056900003D0F878C01F0A2801D36A253AE0B87809
:1056A000010790480029007901DA000700E040076F
:1056B000002801DB63252DE0012152200DF05CFF65
:1056C000874B5222002104465C3330619847072201
:1056D0002046834B394610309847A07CC00701D143
:1056E0002075607507220121019801F07AFE0146BC
:1056F000207C4870607C8870A07CC870E07C087159
:10570000207D4871607D88710198FFF795FA01202E
:10571000403630702846FEBDF7B594460A460098DC
:105720006E4980000C580025002C35D026464036A6
:10573000B0798006C70F206900281DD04030417C19
:105740004B0729D40423194341742069002A0DD042
:10575000634B102261469847002F02D0307805280D
:105760001AD10021009800F053FB15E04030807BF7
:10577000012811D1012500E00825307800280BD040
:105780002946009800F017FB2A46602002430123B7
:1057900039460098FFF7C4F92846FEBDF3B581B03D
:1057A0000C4601984D49800008580026002838D042
:1057B00040300178112934D180798006C00F0090E3
:1057C000019801F0A3FB002102E02154401CC0B26B
:1057D0001028FAD311220621019801F002FE054695
:1057E00010223F4F2146401CB84729460198FFF739
:1057F00023FA0B220721019801F0F3FD0546401C16
:10580000218A0170090A4170214608221231E81CE0
:10581000B84729460198FFF70FFA00990198FFF75A
:1058200032FA3046FEBDF3B506462C4980000C58CE
:10583000002581B0002C22D0204640300178132969
:105840001DD1807910228006C70F2046244B1430CA
:10585000029998470020606311220A21304601F026
:10586000C0FD044610221E4B401C02999847214659
:105870003046FFF7E1F939463046FFF704FA28468B
:10588000FEBDF3B583B00398144980000858002585
:10589000009000286AD006464036B0798006C00FD6
:1058A00001900098046901982746173410370028A2
:1058B0005CD03078022859D10498002827D00146BE
:1058C000074B07222046984706480179090703D469
:1058D000A178F7221140A170A17807E08C900020F8
:1058E000190F0000849000201B070000090706D54F
:1058F000B978090703D5B17940221143B171B17963
:105900004A0606D40079400703D403251FE0082582
:1059100020E004984078002806D17878012803D147
:10592000480601D4022512E0039800F020FA00286E
:1059300007D0049881790398FFF7A9F8002802D0CE
:1059400017E0062503E0B079400612D40825307828
:1059500000280BD02946039800F02DFA2A46602033
:105960000243012301990398FFF7DAF8284605B0AE
:10597000F0BD0398FFF70DFA01210398FFF74AFAEB
:105980000028C2D0A07841072DD04007400F04283E
:1059900029D02079397908402071607979790840D7
:1059A000607107220221039801F01BFD0146207857
:1059B000487060788870A078C870E07808712079A5
:1059C0004871607988710398FFF736F907203070C5
:1059D000009800694030817B002907D0042103989A
:1059E000FEF775FFC2E700202071D9E7417C042251
:1059F00011434174BAE770B50E46FF4B81005C5805
:105A00000025002C12D0214640318B799B060DD504
:105A1000002A07D01A230B700121FEF737FF20342C
:105A2000A67703E000221146FEF730FF284648E53E
:105A300070B514000D4606460ED12A79291D07209F
:105A4000531E0A2B06D89000EC4A80188038C26F8B
:105A500030469047040013D02146304600F0ABF9A1
:105A6000287901280CD00B280AD0304601F0F0F933
:105A7000014660202246024301233046FFF750F8DA
:105A80001FE570B50646DC4980000C5800252069EA
:105A9000002802D00DF0CAFD2561304600F078F9EB
:105AA000403425700DE5FEB5140A16460D460A462B
:105AB0001F4601212046FEF7A5FC019001282AD1AE
:105AC000A000CD49029008584621095C2A78890631
:105AD000C90F0A2A04D00B2A26D00C2A7CD150E008
:105AE000002919D0BE421DD126460446012152206C
:105AF0006D1C0DF041FD5222C14B002120619847E1
:105B0000BF4B206906225C3B294610309847002194
:105B10003046FEF7DCFE5FE0691C2046FFF7A2FD81
:105B2000024653E0422253E02A461435002918D099
:105B3000BE42F7D12146941CC0890A0201460A23BD
:105B4000B048D21D0DF0D8FD0646208A3080AC4BFF
:105B50000822B01C29465C3B984730460DF0E5FD15
:105B60003AE0518A961C009120462B46324601218C
:105B7000FEF766FEA0490298B27E08582030827770
:105B80002AE00029CED020306E78C07F0025410762
:105B900001D5452519E0800701D5692515E09A480A
:105BA00031070079002901DA000700E040070028EA
:105BB00001DB632509E002220B21204601F011FCE4
:105BC000014646702046FFF737F82A46002A03D0E0
:105BD0000121204601F03DF80198FEBD70B50D464B
:105BE0000646854980000C58002C1ED0042D1CD878
:105BF00002220E21304601F0F4FB0146457030468A
:105C0000FFF71AF840342078401E19280DD27D4D38
:105C10003402DC35E11D284600F0FBFD002804D0ED
:105C2000E11D7A4A28460DF0E7FD4AE470B50546C5
:105C300016460C4608460DF0C6FD3F281DD0240A26
:105C4000002E1AD06C48A10040584068002814D09B
:105C500000780A2811D12E2D10D008210D4620469B
:105C600000F0A9F8204601F0F3F860212A460A4323
:105C7000014601232046FEF753FF22E40B21EDE706
:105C800070B50546144610460DF09DFD3F281FD007
:105C9000240A5949A00008585A49DC318D4210D1D4
:105CA0004621095C2030C27F0423520852001A4367
:105CB000C2778906C90F002345222046FEF730FF30
:105CC00006E0C82181872030C17FFD221140C177C5
:105CD000002045E470B516460D4601F09AF8FF28FD
:105CE0001ED04549820089584968002902D00978A8
:105CF0000A2916D001024348CA1D1E23401FC91D90
:105D00000DF0FAFC04460B20207020463C4B082284
:105D10001430658231465C3B984720460DF005FD06
:105D20001EE40121FFF72DF91AE470B50D4601F0CC
:105D300070F80446FF2806D001F08AF801462A468A
:105D40002046FFF785F80BE401460A780120042A73
:105D500001D9002070474A78002A01D0012AF8D1E1
:105D60000A79102AF5D849791029F2D870470146E6
:105D7000214A8900525800201369D97C9B7E9942A0
:105D800000D31946072902D30120203291777047AA
:105D900010B5194A810054582034E17FC90709D051
:105DA00001021848C91DDC300DF079FDE07F400884
:105DB0004000E07710BD70B50C4605460222052173
:105DC00001F00FFB014644702846FEF735FF03E45F
:105DD00070B50E4605461122042101F002FB04466F
:105DE000074B1022401C31465C3B98472146284611
:105DF000FEF722FF1BE600008C900020B859011826
:105E0000750F000017070000849000203075000017
:105E1000FF2212029043090210B50143014800F02D
:105E200068FD10BDEB50001870B50446F94A238890
:105E300000201268002B0AD10CE054899C4205D343
:105E400012895918914200D3012070BD1268002AAE
:105E5000F3D170BD012307E016895D18B54205D363
:105E6000538912685B1C9BB2002AF5D1238070BD58
:105E7000F8B50546CE88888868807004800F14467F
:105E8000022806D00F4601282AD00222022A29D051
:105E90000EE00F68384601F0F7FB0246102807D0E5
:105EA0000320400386430C37042AEFD1D002064377
:105EB000A41AD94B394620469847601B2880F00B1E
:105EC00035D03005000D411D49084900641A208075
:105ED00000206080601B310B09030843A88027E085
:105EE0000422D3E77878397800020843CB49288028
:105EF000884201D10020F1E7C849FF31884202D031
:105F0000491C884203D1F004C00F801CE6E7C34956
:105F1000491E884203D0292109028842CFD102209C
:105F2000A41F208060800021A180601BD6E7AE8086
:105F30002046F8BDFFB583B00020009010200190EE
:105F4000907A15464006800F0F46029003D0022833
:105F500009D001280CD00226022E02D03046103083
:105F60000190002421E0286801F08EFB0646F3E74B
:105F70000426F1E7002F07D0601CC108795C4007B8
:105F8000400FC140C8070ED06868E100401800F01B
:105F9000DBF9002838D00199081880B201900098E8
:105FA000401CC0B20090641CE4B22889A042E1D831
:105FB00000990398FFF738FF002826D100210198A7
:105FC0000DF0DAFA044601986A89201801900298C7
:105FD00002281CD02946069860600398008820811A
:105FE000009BC0186081A281022E1BD001988A4BB1
:105FF000801B3246019098470198001B0838E081C9
:106000000020064600902EE0402007B0F0BD296831
:10601000102EE0D0602082430C31042EDBD12020F2
:106020000243D8E74878097800020843E7E7002FE1
:1060300007D0701CC108795C4007400FC140C807F9
:106040000FD06868F10041180098062250430019EB
:106050001030019AFFF70CFF01900098401CC0B26D
:106060000090761CF6B22889B042E0D8694A002137
:10607000106805E023890589AB4203D30146006817
:106080000028F7D12060002901D00C6000E01460E6
:10609000A089C00505D523460022069C0421104690
:1060A000A0470020B1E770B506465A48046809E0E9
:1060B000A089800505D50122656823460421304664
:1060C000A8472468002CF3D170BDF8B507465148A5
:1060D0000E02B61C046809E0A089400505D5656874
:1060E0002346324604213846A8472468002CF3D1C1
:1060F000F8BD70B5474E3468002C0ED0A08900055D
:1061000005D503220421656823460020A8472046C0
:1061100025680DF08BFA2C00F0D100203060706003
:1061200070BD30B53B4C024609CC083C002B13D067
:106130001D89954210D85889904201D3184630BD28
:10614000186809E0038993420AD84389934202D32D
:10615000037BDB0707D000680028F3D1002030BDA7
:106160000029F5D1FAE7606030BD10B5294B1A68F7
:1061700013E0548984420FD39089C407E40F8C4202
:1061800003D040084000084390815868904201D1F4
:1061900000205860002010BD1268002A02D0148927
:1061A0008442E6D9012010BD30B583885C04A40F79
:1061B0000BD104880525ED02651B032D03D9292584
:1061C0002D02AC4201D1062030BDDC0B04D01B05F2
:1061D0001B0D1818008801E01805000D824201D33C
:1061E000072030BD5118814201D90D2030BD00205B
:1061F00030BD10B50B46014600794006820FC888B5
:106200000ED04118012A10D01846034B102298478F
:10621000102010BD98900020190F000003280000E6
:106220001870000A58700220F3E7184601F045FA8A
:10623000EEE710B50B46014680884004820F0888BF
:1062400008D04118012A0AD01846624B10229847FC
:106250001020DEE71870000A58700220D9E71846AF
:1062600001F02BFAF4E7138983420BD1107B00066F
:1062700001D5594801E00520C0020870000A4870A5
:1062800002207047C01A0623584380180A30D0E70E
:10629000F0B50E4600259C46144607462946FFF7F2
:1062A00040FF01004DD00889B8423FD0381A06227D
:1062B000504340180A306246002A00D0106082889D
:1062C00053049B0F09D103880527FF02DF1B032F0F
:1062D0002CD929273F02BB4228D04088002C23D04C
:1062E0000346E340DB071ED0097BCB0601D508251A
:1062F0001AE08B0701D4D20400D50C250907890FB9
:10630000092C09D00C2C0AD00D2C0AD00007800FC4
:10631000814209D9084607E08007800FF8E70006A8
:10632000F5E78006F3E7062530800BE0002C03D06C
:10633000092C04D0062505E001204002F4E70020E6
:10634000F2E701252846F0BD70B505460188C088F2
:1063500006244004800F1CD0012802D0022802D05D
:106360002CE0042009E0286801F08EF929684A7BB6
:106370000B7B1102194302280BD0841DE888C10B46
:1063800005D00005000D401D4008400004192046BE
:1063900070BD1148801C8142F9D0C01E81420DD0D1
:1063A000401C81420AD00D48814202D0401C8142EB
:1063B00006D1A988052040028843E8D00024E6E7FA
:1063C0000548401C814203D0292000028142D5D1DA
:1063D0000C24DCE7190F000001280000022900004E
:1063E00048207047FFB581B0019816460402002589
:1063F000E01D0DF0E8F93F282ED05F4AFF201188FC
:1064000000290AD0B14208D2701AC0B2062804D9B5
:106410009178490601D4801CC0B2411ECA0F5118A0
:10642000C9050F0E0299002918D001293BD0022975
:1064300012D10027022802D0042850D08025E21D66
:10644000611D06234D480DF057F94221017045703A
:10645000468087800DF069F905B0F0BD022814D0A0
:106460000823621D0093114644489B1D0DF044F91A
:106470000446032F0BD0A31D3946009A01980CF057
:10648000BBFAA080002807D007E02023E9E701201D
:10649000A0800020A07100E0802540202070657061
:1064A00066802046D6E70498018812290BD008257B
:1064B000621D611D042331480DF01EF94121017058
:1064C00045704680C6E7012F07D8428843683946A1
:1064D0000198FFF785FF0546EAE78025E8E70227F0
:1064E000ADE7F0B50C4685B01F210091610601D5DE
:1064F0007F210091210604D5FF22009981321143AA
:106500000091E10504D50322009952021143009144
:10651000194D69466C802880194802900A208881AC
:106520000020C8810320C0028880164B01AA28469B
:10653000FFF700FD06001CD1A006134F400F0AD044
:106540008000001F384382B228880F49001D80B2A6
:106550000C3101F0E6F96007400F0AD08000001FFF
:10656000384382B228880849801C80B20C3101F07F
:10657000D8F9304670E70000E88F002011050000D0
:10658000E4590118E563001800080000FFB581B068
:106590000198164605020024681D0DF014F9102814
:1065A00020D05B48019A00789200301AC7B2029955
:1065B00058480092002917D0012931D0022911D161
:1065C00000210091032F50D080246A1D691D0623ED
:1065D0000DF092F84221017044704680009981804C
:1065E0000DF0A3F805B0F0BD6A1D691D08230DF07C
:1065F00083F8032F07D000238024468083804470D3
:1066000040210170ECE7444D009A0223AA58811DF5
:10661000D28DD20700D002220A70120A4A70ECE72B
:10662000049A032F08D1516852880988022A03D19D
:1066300000290CD002290AD080246A1D691D042378
:106640000DF05AF84121017044704680C8E7324A83
:10665000009BD258D38D5B085B00022903D0002138
:106660000B43D385E9E70121FAE702210091ACE76A
:1066700070B514460D46284A81005158C98DC90786
:1066800015D00102491D51200C230A4600010DF0CE
:1066900033F814210170002141801D490988891CAB
:1066A00081800421C180058144810DF03EF870BDD8
:1066B0001FB5FF21039116491A4B08801748019016
:1066C00003206946088100204881154808806A46F1
:1066D00003A90F48FFF72EFC04B010BDF8B5002445
:1066E0000D4E04250827A300F1582046002909D0A3
:1066F000CA8DAA43CA85F158BA43CA850A4A0121FC
:10670000FFF7B6FF641CE4B2032CECD3F8BD000025
:10671000EC8F002011050000B4900020345A0118BD
:10672000011800008D650018FFFF000030B5D31C74
:106730009C0883000A4D5118A40089085B19890040
:10674000091B400040199C61018498694180996946
:10675000044808809969002048609969886030BDC4
:10676000F88F00205AA50000C088884201D101207E
:10677000704700207047082807D2EFF3108272B6E6
:106780008000024B195082F3108870471C90002043
:106790007FB505460E46EFF3108472B602A80DF0E1
:1067A000E0F984F310880298039900900191281A67
:1067B000000101210009C906884205D20098A842BB
:1067C00005D10198864202D8012004B070BD002096
:1067D000FBE730B5C368826888680125141A240174
:1067E000C9682409ED06AC4203D2904203D18B4222
:1067F00001D8012030BD002030BD0A0C838889B249
:10680000934204D1C088884201D101207047002002
:106810007047094A126906E09388834202D1D388FF
:106820008B4203D01268002AF6D103E0002A01D07F
:106830000120704700207047F88F0020072803D2FE
:10684000024A800080184160704700003C900020A0
:1068500070B50E461C46154601210CF08DFE4660B3
:106860008560446170BD70B50C460646014615460C
:106870004F480CF05BFD4F4A3561F46013782046B9
:106880002946002B03D1012313700DF014F970BDBC
:10689000F8B51C46069B002A0E46054622460DD03A
:1068A00000213820FFF7D4FF434F0446002D0CD0C1
:1068B0001022204629461830B8470DE00021182044
:1068C000FFF7C6FF3246294610E020463A4B102219
:1068D000002118305C33984710222046283031467A
:1068E0000546B84721462A4618312046FFF7BBFF28
:1068F000F8BDF0B589B00E460746002401AD0CF096
:1069000029FEA100641CE4B26850082CF7D33B4672
:10691000012205A901A80096FFF7BAFF09B0F0BD52
:1069200070B505460E4622480CF01DFD0446204871
:10693000002200681F4900280A7005D001220A7051
:106940000169C0680DF0B7F8002C13D0002D07D1F5
:106950006268002A04D0314620469047002809D0BA
:10696000A368002B03D03146284662699847204629
:106970000CF05CFE70BD30B55B1E5BB2002B04DB1F
:10698000CC5CD55C6C40C454F6E730BD10B50F222A
:106990008418203C835CE47F5B00E40923438B5430
:1069A000521E1206120EF3D100784000087010BD7E
:1069B0005C900020CF920020190F0000F8B5064629
:1069C00004462036307E0025002802D001252846C6
:1069D000F8BD204622461830102328320746FFF71C
:1069E000CAFF012030763A462046E168FFF73BFFB8
:1069F000EDE7FFB581B016460F4605460E493C202F
:106A00000B9B0A9AFFF724FF0446324618301023E6
:106A100039460646FFF7AFFF10222046074B2830C5
:106A200004999847002138200155324629462046CE
:106A3000FFF719FF05B0F0BDBD690018190F000080
:106A400070B505460C4606200CF0BDFE04280BD0A0
:106A50000122AA40002C02D00243D1B201E09043AF
:106A6000014606200CF084FE70BD70B5564D0646FA
:106A700084002859002807D00C380168491C03D12C
:106A80000CF0D4FD0020285100213046FFF7D8FF3C
:106A900070BD70B5154604460622022310020CF0A4
:106AA0002BFE047045700CF040FE70BD70B50646BC
:106AB0000D46002406200CF086FE042812D0424A1F
:106AC000B1005358AB420CD00123B340034201D074
:106AD000022407E00124555021463046FFF7B0FF5D
:106AE00000E00124204670BD70B50A4605463649CF
:106AF0008000095800290BD008460C380389DCB205
:106B0000062C05D0072C03D008781946FFF7C1FFE3
:106B1000012D03D12C480421203041712846FFF774
:106B2000A4FF70BDF8B5284B05461E330C46981CD3
:106B300001792678C907C90F0322002E0BD180796D
:106B4000214A800080188068467C828A002E02D00C
:106B500003461633012100912946204600F0D5F85E
:106B60000446FF2807D000F037FB204600F045FA26
:106B70002046FFF798FA2046F8BD70B51546044642
:106B8000FF2811D000F089F80021204606F038FED9
:106B90000021204600F077FB2046012100F098FA02
:106BA00029462046FFF791FA70BD0020074A0146AA
:106BB0008B00D358002B01D0401CC0B2491CC9B275
:106BC0000329F5D370470000649000208C900020CA
:106BD00070B50C460546012901D1FEF752FFF24E71
:106BE000AD007059A4000059002808D00C38016885
:106BF000491C01D10CF01AFD71590020085170BDDB
:106C000070B50502ED1D16460C4628460CF0DBFD5E
:106C10001F280CD028460CF0D6FD002E02D00146CD
:106C2000214301E0A043014628460CF0A1FD70BDC0
:106C300070B5164602021C460D4607200223314657
:106C40000002D21D0CF058FD057044700CF06DFD73
:106C500070BD70B50D460646D349800008581346EE
:106C6000A9004258002A0CD010460C380489E0B222
:106C7000052806D0062804D0117822463046FFF7B2
:106C8000D7FF29463046FFF7A3FF0120A840C1B235
:106C900000223046FFF7B4FF70BDF1B500988600C2
:106CA000C148815900980502002920D0E81D0CF048
:106CB0008AFD074600241F2F04D021460098FFF7C5
:106CC00087FF0AE0B848A10080594058002804D046
:106CD000462221460098FFF7BCFF641CE4B2032C57
:106CE000E9D3B14CA0590CF0A1FC0020A051E81D43
:106CF0003F210CF03DFDE91DAC480CF0D0FDAB4848
:106D0000E91D801C0CF0CBFDF8BDFFB581B0054638
:106D100000242002C01D0CF056FD3F2803D0641C47
:106D2000E4B2032CF5D3032C71D0002158200CF0D1
:106D300023FCA6009C4F58229D4BB8510021984738
:106D4000B859C8218187B9590F20403148752002B0
:106D500000900021C01D0CF00BFDB9590298403184
:106D60008880B859E97B40308175B859DF214030BF
:106D700082790A402978002900D0012149010A437B
:106D800082718B4BB8590622A91C5C3B4E30984748
:106D9000B859697840300175854BB85906225C3B7B
:106DA000473004999847B9590A9840314873B959FE
:106DB000FF208881B9590398C8810398062822D0FA
:106DC00001467A48009A1223F138D21D0CF094FC47
:106DD0000646029830806878754BC007C00F707205
:106DE00030460622A91C0A305C3B984728897080EF
:106DF0006889B080A889F080A87B307228783074C8
:106E000030460CF092FC204605B0F0BDFFE7FF24B1
:106E1000F9E70346644A002081005158002903D055
:106E200040318988994203D0401CC0B20328F3D373
:106E3000032800D1FF20704701465E48032906D28F
:106E40008A0059498958002901D040318888704703
:106E500001460020FF2908D08A005349895800299B
:106E600003D0403188798006C00F704770B54E4D11
:106E700084004F4B285906225C3B473098472859DD
:106E800001214030417370BD02460020FF2A0AD024
:106E9000022908D29300444AD258002A03D0C800DD
:106EA000401A47301018704701468A003E490020BA
:106EB0008958002901D04031887D70470246002062
:106EC0009200394B002909D001290CD0022904D1A4
:106ED000985840308079C006C00F704798584030AD
:106EE00080794007F8E79858403080790007F3E749
:106EF00001460020032908D28A002B49895800291D
:106F000003D0403188798007800F70470146002008
:106F1000FF2906D08A0024498958002901D0203150
:106F2000887F7047F0B5032827D21F4F8300FC5895
:106F3000002C22D04034A579FB263540CE07760FB1
:106F40003543A571FC58EF263540120115434034F6
:106F50000020A5710A0701D5032008E04A0701D5E2
:106F6000022004E0C90701D1290700D50120AA08A1
:106F7000F9589200024340318A7146E710B519244E
:106F8000E401401EA0420AD2491EA14207D20A488B
:106F90000A3B834203D2FF20F430824201D9002011
:106FA00010BD012010BD00008C900020F2070000F1
:106FB000750F0000FFFF0000770C000070B5840023
:106FC000814E0D46012909D13059816808300029C8
:106FD00004D00CF0C8F90CF029FBF5E73059AD00EE
:106FE0004059002808D00C380168491C01D10CF028
:106FF0001DFB31590020485170BD70B50446002179
:1070000030200CF0B9FA3022704B05460021984729
:107010001720A885A0006C4924020D50601D002196
:107020000CF0A6FB0825601D0CF0CDFB01462943A2
:10703000601D0CF09DFB70BDF8B51C46154607465B
:1070400000290BD1A08800F0A1FC060006D06570D5
:10705000A288234603213846B047F8BD0A2D06D141
:107060006088010403D500254004400C6080204660
:107070000C3801893A02052004230002521D0CF04D
:107080003BFB457021780170618841800CF04DFB1D
:10709000F8BD70B50D4604464B4980000858A9005C
:1070A0004358002B03D029462046FFF7C5FF294649
:1070B0002046FFF783FF0120A840C5B22402601DCF
:1070C0000CF081FBA8430146601D0CF051FB70BD24
:1070D000F8B5064685003C480F464059002835D093
:1070E0000024002F05D0462221463046FFF7D1FF6D
:1070F00003E021463046FFF761FF641CE4B2022C36
:10710000EFD3304600F05CFD2F4F07E040880028A9
:1071100001D00CF067F820460CF088FA7859016A23
:107120002030002907D00CF01EF904460C300178FD
:107130000029F0D1EAE7304600F050FD304600F07B
:1071400077FC78590CF072FA00207851340215203F
:10715000611D80010CF0A3FB611D1D480CF09FFB1D
:10716000601D10210CF004FBF8BD17498000085881
:10717000808D704770B5012217235202914200D3CF
:107180001146172900D219460F4D84002A590423AD
:1071900091851049020209590D48C9893F38521D8D
:1071A0000CF0AAFA2959898D0180295949680029CA
:1071B00002D00A78012A04D0002141800CF0B5FAEF
:1071C00070BD4988F9E70000B4900020750F0000F9
:1071D000410500008C90002010B5044600020021FB
:1071E000001D0CF0C5FA002124200CF0C5F9002880
:1071F00007D00021016041608160017301740421A6
:107200004174984AA100505010BDF8B50646C8B266
:10721000B4001746052814D0072811D108460CF0F1
:10722000D2FA3F280CD0904800594068002807D077
:1072300000780C2804D1002201213046FFF709FD17
:10724000F8BD08460CF0BFFA1028F9D0874D285930
:107250000068002807D00078122804D13A4600219F
:107260003046FFF716FF295900204968002900D051
:1072700008780D2801D00E28E2D13A460121304687
:10728000FFF707FFF8BDF3B507468600754881B0E4
:107290008459002C27D0A068002801D00CF0C6F932
:1072A0007349207B4A88101848800BE0A9887148F0
:1072B000814204D1298946223846FFF7A6FF284695
:1072C0000CF0B4F92068002807D020460CF04BF8E9
:1072D000054602980028F2D1E8E7624CA0590CF06C
:1072E000A5F90020A05138023F21001D0CF040FA02
:1072F000FEBDF3B585B005985A4980000E58002EA2
:107300005FD03468002C04D00698002801D00120FA
:1073100000E00020039049E00020694688800127B2
:107320000BF071FF05468088534943185149A088E6
:107330004942C84225D121460C31081D0290E089FE
:10734000002800D000E0002701AA0097891C0298BD
:1073500006F06EFA0090002803D1029800880028F9
:107360000FD12189009A0598FFF74FFF30460BF0A7
:10737000FAFF20460CF05AF90020039000980028EC
:107380000DD16946898838030843E8800598FFF7DE
:1073900053FDC0B2294604F000FD002813D0A88890
:1073A0000BF04BFF0698002802D003980028B3D1B9
:1073B0003068002813D0002101204140059806F0D4
:1073C0001FFA07B0F0BD2A494888401E4880307B2C
:1073D000401C30730698401EC0B20690E3E70121BE
:1073E000EAE770B50D46114608318BB2010214462A
:1073F000CA1D2048091D0CF07FF90621C180848038
:107400000572083070BD70B50D46114609318BB25A
:10741000010214464A1D1748091D0CF06DF904219C
:10742000C18084800572083070BDF8B5069D1E4687
:1074300014460F46042A11D0062C11D004212A46E6
:107440000A32000293B2021D01430A48401C0CF0AC
:1074500053F90770C48085800672F8BD0521EEE7F8
:107460000721ECE7C09000208C900020B490002011
:107470008C9200200604000000800020F8B50F4622
:10748000540021461E460E318BB2010215460A1DDC
:107490007A48091DA41C0CF02FF90521C180211D7B
:1074A000818001210172477244818581002D00D0C5
:1074B000C6810CF03AF9F8BD70B50D4601021446CC
:1074C000CA1D0E236D48091D0CF016F90521C18057
:1074D000062181801321017245720221418184813C
:1074E0000CF023F970BD70B50D4601021446CA1D9B
:1074F00014236248091D0CF0FFF80521C1800C21FE
:107500008180122101724572082141812188818187
:107510006188C181A1880182E18841820CF005F96E
:1075200070BD10B50A790024012A0AD0122A0CD0A5
:10753000132A0FD0002349791A46FFF79FFF2046F0
:1075400010BD091D00F00AF802E0091D00F02BF83B
:107550000446F4E7091D00F062F8F9E770B58B887E
:1075600000244C220546002B04D0012B04D0022B12
:1075700005D103E03C2202E0312200E03322404802
:10758000AE00805900230068002800D00378092B42
:1075900007D140784978814203D100212846FFF77E
:1075A00058FB204670BD70B50C4605460026FFF717
:1075B0004FFC012825D063892289A188E088FFF744
:1075C000DDFC002824D02902CA1D0E232D48C91D28
:1075D0000CF092F80921017061784170A188418016
:1075E000E18881802189C180618901810CF09DF849
:1075F0002348A9004058FD224030417D114041758B
:107600000BE0002361781A462846FFF737FF04E0B5
:10761000617801222846FFF74FFF304670BD70B5F4
:107620000C4605460026FFF713FC002809D0144835
:10763000A90040588268002A1ED01078092807D077
:107640001AE0002361781A462846FFF717FF13E077
:107650006078517888420FD1A088002801D0482254
:1076600000E0002202212846FFF7F3FA054829022C
:10767000E430C91D0CF013F9304670BD060400005B
:107680008C9000200E0700003EB50546B8A107C942
:107690006B4607C31024B94B0C226946284698470D
:1076A000002806D1A87B002802D1E87B002802D060
:1076B000042420463EBD0224FBE7FEB50E460546E7
:1076C000ABA207CA6B4607C3AC4C0C2269462846DE
:1076D0008A3CA0470422284631460C30A047FEBD14
:1076E000F8B51E4615460C46B14202D10A46294657
:1076F00012E00746102C03D1FFF7C6FF04460C37F3
:10770000102E04D12846FFF7BFFF06460C35B442C1
:1077100006D1224629463846984B9847002801D082
:107720000020F8BD0120F8BD70B5154604461029AB
:1077300003D1FFF7A9FF01460C34022907D1607875
:10774000217800020843A84201D1012070BD002029
:1077500070BD10B5491EC9B2FEF766FB10BDF7B586
:107760000E460025144629460098FEF7DAFC020072
:1077700069D010890099824F884206D11046394657
:1077800008302760FEF735FD55E0081A062148430A
:107790008018C1890A308C464904890F20D101889C
:1077A0000523DB02CB1A032B03D929231B029942A1
:1077B00016D1744B994220D100995289491C8A42B2
:1077C00019D327600289801D120A3A70226851700D
:1077D000090A91702168C91CFEF72BFDC01C2AE024
:1077E0006146C90B2DD061460905090D0818011D18
:1077F000216040881FE0802526E062461205120DB8
:107800001018604A521E914217D180880021FEF75D
:1078100088FC0028EFD0276001893970090A797047
:10782000216842898A70120ACA7021680830091DCD
:10783000FEF7DFFC001D308006E0001D2060022006
:10784000F9E7062500E001252846FEBDFFB50F46F5
:1078500081B01546064601240021FEF762FC00288F
:1078600030D001890624B1422CD0711A062251432E
:107870000818C2890A305104890F0FD101880523E5
:10788000DB02CB1A032B1DD929231B02994219D0E5
:107890009B1C994216D05B1C994213D0D10B11D07E
:1078A0001105090D0C1820887E19864209D8334B22
:1078B00060198A3B3A46001D049998476680002467
:1078C00000E00D24204605B0F0BDF8B50E46154683
:1078D000074601240021FEF724FC00281FD001895F
:1078E000B9421CD0791A062251430B18D8890A33A1
:1078F0004004800F09D118880521C902411A0329C3
:107900000DD929210902884209D05E80E9041E4868
:10791000998801D5014300E08143998000242046E5
:10792000F8BDF8B50E461546074601240021FEF7BE
:10793000F8FB00281AD00189B94217D0791A06221B
:1079400051430B18D8890A334004800F09D1188895
:107950000521C902411A032908D9292109028842AF
:1079600004D05888B0432843588000242046F8BDEE
:10797000FB349B5F8000008000100000A30F00001C
:10798000A0900020032800000010000010B5002186
:10799000FEF7C7FB002800D0406810BDF8B51446BC
:1079A0000D4607460A46002669462046FEF770FC4B
:1079B000040006D00C2C02D0062C1CD036E000248B
:1079C000012668460088002830D03846FFF790FA34
:1079D000002822D00E2D22D001213846FFF76EFA62
:1079E000002812D0002E1AD03846FFF78FFA102840
:1079F00015D20C241AE00C2D18D00D2D16D0092DFF
:107A000001D0032412E0022410E002213846FFF7DF
:107A100055FA002801D00F2408E0052406E0384676
:107A2000FFF766FA694609888842F6D32046F8BD12
:107A300070B5FF4D84002859806A002805D00C38A5
:107A40000BF0F4FD29590020886270BDFFB581B0AC
:107A5000174601980D46F64A810050581E46806A26
:107A6000002817D04388AB4211D14478062C02D0AD
:107A7000002C05D000E080240198FFF7D9FF0FE02B
:107A8000808838805058806A801D306013E00198EB
:107A9000FFF7CEFF324639462846FFF760FE044620
:107AA000062C08D12846FFF771FF064600232A4618
:107AB00019460198B047204605B0F0BDFFB585B026
:107AC000088816460C460027049020880121FEF7FE
:107AD00028FB050015D021882889814200D220800A
:107AE00020883188884214D82A466946FEF7BBFBB5
:107AF00003466A4608990E98FFF7F2FD00280AD15E
:107B000004E030882080002F1AD004E02088401C38
:107B10002080002F0ED02288002309210598FFF72E
:107B20003DFF07462088294600F0ACFE3080002F3C
:107B30000AD010E0318880B2884201D80028C4D130
:107B400004980A27208006E02188109B0F9A059848
:107B5000FFF77CFF0746384609B0F0BDF8B5074689
:107B60000020009008780C46122827D01D26E588B2
:107B70003846FFF7FAFAC01E854200D2284685B281
:107B8000281D82B231463846FFF73DFC0646A088E4
:107B9000214670800831A74B2A46301D9847304651
:107BA00008380BF0C2FD2078122805D03902A24A0D
:107BB000A248491D0BF020FE0098F8BD1B26D6E711
:107BC00070B59B4D8400285901691030002904D0FC
:107BD0000BF0C9FB0BF02AFDF5E770BD70B5944DB5
:107BE0008400285981691830002904D00BF0BBFBB0
:107BF0000BF01CFDF5E770BD70B515460E461C4632
:107C000005220121FFF7FFFB46704580047108380B
:107C10000BF08BFD70BD10B5002A05D013460A4647
:107C20001221FFF7E9FF10BD01221321FFF7EBFB43
:107C300008380BF07AFD10BDF3B5814F81B00E46C8
:107C4000BD8B042203210198FFF7DDFBBA8B7188FD
:107C500004468A4200D211460198FFF78BFA20466B
:107C6000658008380BF061FD0020FEBDF3B585B0DE
:107C7000002002900F460598FFF777FA801E86B223
:107C8000049605987C88B9888000002503908C4272
:107C900001D8002C01D101201FE001212046FEF770
:107CA00040FA0090002817D00089844200D2044690
:107CB000B888A04226D3012118200BF05DFC01906A
:107CC000848001992046C91D009AFEF7CCFA0199DB
:107CD000002D887103D003E00A2002901AE00546C7
:107CE000A84203D001980BF0A1FC13E0504903987F
:107CF0000858019918300BF019FB701B801E641C8A
:107D000086B2A4B2B888A04204D3002C02D0A81C2A
:107D10008642C2D2464C039820588069002812D06F
:107D200004980027801B801C82B205210598FFF76C
:107D30006AFB0646022D0AD00220707003983D4D62
:107D40002058846913E00298002817D018E0012019
:107D5000F3E7F019A1884180BF1CBFB2F019E11D03
:107D6000A279801CA847A0792468C01987B2002C8A
:107D7000EFD1304608380BF0D8FC07E00A2002901B
:107D800003467A8839780598FFF736FF002007B058
:107D9000F0BDF3B58BB00C46488869468881204613
:107DA00040380990C68F0B9880000790002E0AD1AA
:107DB0000B98FFF7DAF9401E86B26088A1888842E6
:107DC0001ED800281CD0A01D0A90801C0590099880
:107DD0006946808F04AA083887B2A08808830A9869
:107DE00008A96D4607C5022306AA03A90B98FFF749
:107DF00065FE050006D00A2D50D0062D4ED03FE07E
:107E000001254BE0E0880521C902884202D0491CC7
:107E1000884209D16846008CF9B2C3B2049A059829
:107E2000FFF75EFC002815D16846008CB84209E0D7
:107E3000B4900020190F00003075000041050000CB
:107E4000649000201CD1FD4B3A4604990598984750
:107E5000002815D1012108200BF08EFB0146684651
:107E6000808988806846008BC880F54A0798361F4D
:107E70001058B6B218300BF059FA0B98FFF7D8FD2E
:107E80006946088B401C8881A0888989884205D36F
:107E90006946098B884201D0042E98D20998062D94
:107EA000C68734D0E64E0798305818300BF034FAB5
:107EB000002822D08000801C82B2002407210B9869
:107EC000FFF7A1FA01460798305880690CE063007B
:107ED00082885B185A80641CA2B254006418C3885C
:107EE0006380521C006894B20028F0D1084608381C
:107EF0000BF01BFC062D0DD006E068468289217828
:107F00002B460B98FFF778FE00200DB0F0BD6846B9
:107F1000808960800120F8E7F3B58DB000200690DD
:107F20000D46488869460882284640380A90C48F22
:107F30000027002C0CD10D98FFF717F9801E84B292
:107F40006888A988884201D8002801D101200690BC
:107F50000D98BB498000079008588069002800D020
:107F600087790698002856D1A81D0B900A98A988F1
:107F7000808F6A4691840B9908AB03AA6E460EC6A1
:107F8000801FC3B209AA04A90D98FFF797FD0690B8
:107F9000002840D1684681898F4201D0002F3AD114
:107FA000A01EFD22FD2800D31046814200D20846C3
:107FB00086B23046012108300BF0DEFA05906846A3
:107FC0008789018A05989D4B818005988A3B867137
:107FD00005983246C01D08999847A01B801E84B2A0
:107FE000974907980858059918300BF09FF968468B
:107FF0008089864202D10D98FFF71AFD6A46908C5F
:10800000411C89B21182AA888A4204D3824202D0DA
:10801000B81C8442AAD20A98C487069806283FD082
:10802000874C0798205818300BF076F900282DD08F
:108030000799002661588C69A179891C4143891CE4
:108040008AB209210D98FFF7DEF90546A079801C58
:10805000687011E0A819A1888170090AC170B61C66
:10806000764BB6B2A819E11D8A3BA279801C9847CD
:10807000A0792468801986B2002CEBD128460838F4
:108080000BF053FB069806280DD006E06846028ADE
:108090002978069B0D98FFF7AFFD00200FB0F0BDCB
:1080A0006846008A68800120F8E7F3B58BB00020AD
:1080B00002900D46488869468881284640380890D5
:1080C000C48F00200490002C0CD10B98FFF74DF8C2
:1080D000801E84B26888A988884201D8002801D10E
:1080E000012002900B98564980000790085880693B
:1080F000002801D080790490029800285BD1A81D47
:108100000A900898A988808F6A4611830A9909AB5A
:1081100005AA6E460EC6801FC3B206AA03A90B9815
:10812000FFF7CCFC0290002845D16946898A049863
:10813000884201D000283ED1201FFB22FB2800D31B
:108140001046814200D2084686B2304601210C30EA
:108150000BF012FA07466846808A049068468089C8
:10816000B8806846008BF8803846344B3E72093040
:1081700032468A3B09999847A01B001F84B23049B8
:1081800007980858394618300BF0D0F86846808AAE
:10819000864202D10B98FFF74BFC6A46108B411CBC
:1081A00089B29181AA888A4205D3824203D0049879
:1081B000001D8442A5D20898C487029806284AD098
:1081C0001F4C0798205818300BF0A6F8002839D01B
:1081D0000799002661588C69217A091D4143891C41
:1081E0008AB211210B98FFF70EF90546207A001D7F
:1081F000687019E0A819A1888170090AC170B61CBD
:10820000B2B2A818E1888170090AC170921C96B2B6
:108210000A4B2146A81909318A3B227A801C9847CB
:10822000207A2468801986B2002CE3D128460838C9
:108230000BF07BFA0298062810D00AE0A30F00008A
:10824000B4900020684682892978029B0B98FFF73A
:10825000D3FC002059E6684680896880012054E6F6
:108260007CB50C464A88054600230921FFF796FB9A
:10827000030007D1618801AB6A462846FFF7E6FB99
:10828000030007D0062B2ED0628821782846FFF7FE
:10829000B3FC26E0684604882846FEF766FF401EC9
:1082A000844200D2204684B2601C82B20B21284650
:1082B000FFF7A9F80646FF4B2246401C0199984754
:1082C000304608380BF031FA68460088844208D1FD
:1082D0002846FEF74AFF401EA04202D02846FFF77C
:1082E000A7FB00207CBD01207CBDFEB50D464A8861
:1082F000064600230921FFF751FB040007D16988D6
:1083000001AB6A463046FFF7A1FB04000AD0062CF9
:108310003BD06A88297823463046FFF76DFC062C4F
:1083200033D030E06946A8880988884201D90724FB
:10833000EFE70C1A3046FEF718FF401E844200D2C9
:10834000204684B2601C82B20D213046FFF75BF8F4
:108350000746A8880199D74B41182246781C9847B0
:10836000384608380BF0E1F9A888694609880019F1
:10837000884208D13046FEF7F8FE401EA04202D0E7
:108380003046FFF755FB0020FEBD0120FEBDF3B5D2
:1083900087B00898C84940380390808F0025C003F3
:1083A0004018000C05900798C449800002900858B6
:1083B00018300AF0B1FF06460398C48F002C39D15B
:1083C0000798FEF7D2FE401E84B233E00898710091
:1083D0000F187A88002309210798FFF7DFFA0500B4
:1083E0002FD179886B4604AA0798FFF72FFB050069
:1083F00020D16846008AA04200D3204687B2384682
:10840000012108300BF0B8F8019087800198A94B42
:108410003A46801D00999847A84902980858019942
:1084200018300AF083FF0798FFF702FBE01B761C69
:1084300084B2B6B20598B04203D9002C01D0002D09
:10844000C4D00398002DC48722D10798FEF78DFE73
:10845000001B82B200270F210798FEF7D4FF00907F
:1084600096490298085884690AE00098A11DC0192D
:10847000904BA288401C9847A0882468C01987B2F6
:10848000002CF2D1009808380BF04FF9002D0BD0DA
:10849000062D0CD0089871000818428808982B46C1
:1084A00001780798FFF7A8FB002009B0F0BD012074
:1084B000FBE7F0B506460A78002085B0122A10D0F6
:1084C000522A11D10C464039888F0027001F85B2EF
:1084D000628802AB0A213046FFF760FA002805D017
:1084E0001FE0304600F036FA05B0F0BD0022294604
:1084F0000298FDF759FE002813D152200390678897
:10850000241D3846FFF742FA8446694603980880DE
:108510004D8001946B463A46012130466446A0479F
:1085200001273846E0E7F3B5084685B040380090AB
:108530000025C68F0C462F46002E07D162880023E7
:108540000B210598FFF72AFA050037D105986388B3
:1085500000218000594A049010589C4686460069C4
:1085600005E0C28A9A4201D1012100E0006800289A
:1085700002D00029F5D003E0002901D1002E26D039
:108580000098808F801F80B20290704620300AF0E1
:10859000EAFE039060883105090D01910090A388DF
:1085A000029A0399059800F09CF905001CD04349F4
:1085B00004980858039920300AF0CEFE628821788A
:1085C0002B460598FFF718FB384607B0F0BD60460C
:1085D000FFF7DCF906460023628802210598B047C0
:1085E0000127002DEAD1EFE702981721801D82B202
:1085F0000598FEF708FF054660886880A11D2D4B91
:10860000A81D029A9847A088A880284608380BF031
:108610008CF80227D8E7F3B587B0089800214038D6
:108620000290C08F049100910899497801297DD169
:1086300007998900039100285AD1204840580469BD
:10864000002C55D000200646054605902746E08AB6
:1086500000211437FDF765FD00280DD001897A88C7
:10866000914209D0511A0622514308182289618982
:108670000A30FDF799FD00E00120009001200190F3
:10868000009800280DD178880599884204D005907B
:10869000E68800202546A0802089B04213D9072013
:1086A000009008987A880178009B0798FFF7A4FA51
:1086B000079805E0190F00000000FFFFB4900020AC
:1086C000FFF77EFA11E0B04206D2A54204D0E68060
:1086D00060892546A08005E06189401886B2A88897
:1086E0004018A8802468002CB0D102990198C8874E
:1086F000B24E039830580469002C40D0E08A0490B0
:10870000A0880690254614350498FFF73FF90746E0
:10871000A088694648812089694608816089488027
:10872000A81D019016200880002000E027E0059099
:108730002668002E0ED0069800280BD0F18A354608
:1087400004981435814205D101200590FF2017308F
:10875000694608806B460121049A0798B8479749F3
:108760000398085810300AF0FEFD20460AF05EFF1C
:10877000059834460028CED1012004900DE00798DA
:10878000FFF71EFA0098002807D101221921079847
:10879000FEF739FE08380AF0C8FF049885E6F1B5FF
:1087A0000098864F860024E02C46E8890C34002887
:1087B00003D00AF017FD00206080207A8049C006AF
:1087C000000F401E0006800D0A582146083100980F
:1087D0009047002804D001280FD002280BD108E0D0
:1087E0000098FFF7FBF9B85920300AF0BCFD0AF0F9
:1087F0001DFFB859056A002DD6D1F8BDF8B506465B
:108800000A7A0402FF2580006C4B1E2A02D0D7078B
:1088100015D033E01858002100680D46002800D01C
:108820000178132901D0142928D1611D65480BF066
:1088300036F8002211463046FEF72BFC1EE0002AD7
:108840001CD0D706FF0E182F18D8142A16D01A5885
:10885000126A002A14D000270022CA8018580C3946
:1088600020300AF063FD0125601D0AF0ACFF00070F
:1088700004D4002F02D03046FFF791FF2846F8BD00
:108880000127E9E7F0B50C89844201D14889F0BDA0
:10889000021B06235A435218D3890A325B049B0FEA
:1088A000F5D11388484EB342F1D1401C002583B264
:1088B000771E488910E05189921D4904890F04D11F
:1088C0001188B14205D0B94203D05B1C9BB2002D88
:1088D00002D05B1E98B2F0BD9842FCD39C42EAD312
:1088E000F0BDF8B58600002534480095855914463A
:1088F0002D69069A2746002D09D0AD8801272D192C
:108900007F02BD4202D911200090F8BDAFB24C8168
:108910000B81079B2948CB8080590D460469103094
:108920000AE0E18A914206D92A4621460AF077FDFB
:10893000002C03D008E02468002CF2D11F482946FF
:10894000805910300AF0F2FC1C4880590069878079
:108950000098F8BDFEB5074608464038808F0C46A3
:10896000001F85B24A8800266B460B213846FFF768
:1089700015F8030006D1002229460098FDF714FCE3
:10898000030006D0628821783846FFF735F9304673
:10899000FEBD122002906688241D3046FEF7F6FFC9
:1089A00084466946029808804D8001946B463246A1
:1089B000012138466446A0470126E8E7B49000202C
:1089C0004C5A01184105000003280000F3B50024AB
:1089D000224FCE0781B0F60F1C206043C519A87B3B
:1089E00009280BD12946143101980AF0A6FD002868
:1089F00004D0A87EC007C00F864204D0641CE4B235
:108A0000042CE9D303E0042C01D20120FEBD002098
:108A1000FEBD1C214843114910B540180021817347
:108A200003F0C5FF10BD70B50C49054600241C209D
:108A300060434018807B002805D0641CE4B2042CFD
:108A4000F5D3072070BD1C20604340180822002188
:108A5000034B143098472C70002070BDCC90002040
:108A6000750F000010B50446814B80001B58403341
:108A70009878002809D199701146204603F03BF9F7
:108A800003220221204605F0CCF810BD70B5054642
:108A9000774A800010580029046825D161780029A0
:108AA00002D0012920D11AE003220221284605F034
:108AB000B8F800220121284605F0F0F8217928466F
:108AC00000F019F80120607000221146284605F0D8
:108AD0000FFA01220021284605F0E0F870BD617907
:108AE00001222846FFF7BEFF0021284605F000F9C5
:108AF00070BD0021CAE708B502226B461A70597092
:108B0000C0B25C4A694605F077FA08BD002901D178
:108B10001178BBE7704770B50E4604465449800093
:108B20000D5800221146204605F0B8F80022012118
:108B3000204605F0B3F8E88F7178C007C2172046C9
:108B4000521CFFF78FFF002070BDF8B5150A484989
:108B5000A8000C58D8B21646162801D04221085554
:108B60002346423300221F461146284605F0E2F80C
:108B70003B4600220121284605F0DCF803220221B1
:108B8000284605F04EF8FF2130460AF0F1FD40344A
:108B9000A2780021284604F099FC0021284604F020
:108BA00098FF2846FFF735FF0020F8BD70B5144642
:108BB00006462F4A80001058C08F800512D4002925
:108BC00005D00022631D1146304605F0B3F801259B
:108BD00022460021304605F04BF800213046FFF7D1
:108BE00055FF00E00225284670BD70B50E462049AD
:108BF00082008C580025002C09D040342178C943CC
:108C0000890704D06178C90703D03A2517E00C25FD
:108C100015E00102491CFF2006230A4607300AF02E
:108C20006BFD07210170002141700671132E08D0E1
:108C300046710AF07AFD6078012108436070284689
:108C400070BD16214171F4E710B50C460102491CB4
:108C5000FF2006230A4607300AF04EFD0721017067
:108C600000214170047144710AF05FFD10BD0000E5
:108C700090920020F38A0018F8B50F46064681004E
:108C80005748445825686878002815D0012825D011
:108C90001F27E87800280AD022463032394630466D
:108CA00004F047FC40346078FD21084060700021EA
:108CB000304605F01DF8F8BDE08F4007E9D4304696
:108CC00000F07FF8E08F08210843E08701206870FA
:108CD00002460021304604F0E1FFF8BD00221146B3
:108CE000304604F0DBFFD4E7002901D11178C3E757
:108CF000704770B500250446FF2909D001250021E1
:108D000004F0B6FF00212046FFF7B6FF284670BDED
:108D1000D0780028FAD03249A0000A584220815C5D
:108D20002046303204F005FCF0E770B52C4D82008F
:108D3000AC584E7830231E554B8863868988A186AF
:108D4000E38F04210B43E387A9580968002902D067
:108D50000978012909D0190705D400F032F8E08F0D
:108D600008218843E087002070BD0021FFF784FFC1
:108D7000F9E770B51A4982008C580025002C09D0FB
:108D800040342178C943890704D06178890703D525
:108D90003A2514E00C2512E00102491CFF200423AF
:108DA0000A4607300AF0A8FC012101700022427037
:108DB000C1700AF0BAFC607802210843607028464E
:108DC00070BD1CB50C216A4611700B21517005490C
:108DD0005180052191800022694605F00DF91CBDE6
:108DE00090920020C509000010B5FF498200895803
:108DF0004968002906D00978062903D100221121EB
:108E000000F010F810BD10B5F74982008958496884
:108E1000002906D00978062903D10022122100F08A
:108E200001F810BDF0B51746064685B08000EE4A41
:108E30000090155804206C6862788A420BD0132980
:108E400001D03D2701E03D2F04D1012239463046B3
:108E5000FFF708FEC0E00A390B0008F0A5FC090680
:108E60003F46577389A8BDBC55000021304602F02B
:108E7000CEFF01220021304605F03AF82746E98F5F
:108E80002037B87D8906C90F884207D0D74B2422E6
:108E90000321304605F000F912206070B87D0028EB
:108EA00012D00021304603F0CDF8012202213046D5
:108EB00004F0B7FE0B256946304600220D7005F020
:108EC0009BF8657001221BE002221146304604F037
:108ED000A8FE304600F049FA0D203CE00021304663
:108EE00003F098F80C206070ECE70222114630463F
:108EF00004F097FE304600F038FA0D206070002232
:108F00000121304604F0CAFE05B0F0BD6A4610707B
:108F1000254600A820350822B54F013021462C31C6
:108F2000B847042202A829460130B8470022694602
:108F3000304605F061F8A18E221D3046FCF7CAFECE
:108F40000E2008E0002F08D0A84B0622032130464F
:108F500005F0A2F812206070D6E720462146A54B06
:108F600001220C3024310096FDF792FC0F20F2E72D
:108F70002146224630460C311C3203F07BF8012199
:108F8000304603F05FF805216A4611703046002232
:108F9000694605F031F81020607001221146304614
:108FA00004F07CFEE88F01214902084347E00022DB
:108FB0000121304604F072FE0121304603F02AF808
:108FC0001120607006216B46197030468A4A694646
:108FD00005F012F898E706278348009940580028C2
:108FE00025D040300078C043800720D00121304692
:108FF00002F00DFF00220221304604F012FE002F85
:1090000003D02034A07D002803D039463046FCF739
:109010008CFEE98F20208143002F12D000204001D8
:109020000143E98700221146304604F061FF012127
:10903000304604F05DFEE88F012149028843E8874D
:1090400062E70120EBE710B567498200895809689B
:10905000002906D00978062903D10022022100F058
:1090600001F810BDF0B51746064687B080005E4A8D
:10907000009015582C68607888421CD0092901D0CE
:109080003D2712E0132F0ED004DC062F07D0082F47
:10909000F6D108E01A2F04D0222FF1D103E00528E1
:1090A00001D00428ECD13D2F04D1012239463046AD
:1090B000FFF7D8FCCCE0030008F076FB09061F1A86
:1090C000427785A240C540000021304602F09FFE55
:1090D0003620005D00280BD00A216A461170304608
:1090E0000022694604F088FF01206070024657E0C4
:1090F000304600F03AF903201FE0012200213046FB
:1091000004F08FFD01221146304604F0F1FE0022EA
:109110001146304604F0C2FD0021304602F092FFB5
:109120000021304602F076FF0B216B461970304665
:10913000324A694604F060FF0220607007B0F0BD5B
:109140002246A08E2432069203236A461370507280
:10915000000A9072274600A81C370822244D0130CF
:10916000211DA847082202A803300699A847042217
:1091700004A839460330A84700226946304604F067
:109180003BFF0420607001220021304604F086FD80
:109190002034A07D002802D00222114601E00222E4
:1091A0000121304604F03DFDC8E70222002130468F
:1091B00004F037FD01221146304604F099FE0520E7
:1091C000607001220BE0204621460A4B01220C3040
:1091D00024310096FDF75CFB062060700022002120
:1091E000304604F05BFDA9E790920020078E00183E
:1091F000190F0000BF920018E98D00184790001861
:109200002146224630460C311C3202F033FF012148
:10921000304602F017FF0121304602F0FBFE062126
:109220006B46197030460022694604F0E5FE0820BE
:10923000607001220021304604F030FDE88F0121EA
:109240004902084337E000221146304604F026FD6B
:10925000FE4800994058002821D040300078C04393
:1092600080071CD0284640304178F72211404170D9
:109270000121304602F0CBFD00220221304604F0ED
:10928000D0FC00220121304604F032FEE98F20207C
:109290008143002F11D0002040010143E987394666
:1092A0003046FCF742FD0021304604F021FDE88FF6
:1092B000012149028843E88740E70120ECE7F8B53F
:1092C0000F461006E149800D0858154600282AD09F
:1092D0004022125CD243920725D0AA008958DC4E66
:1092E000C98FC90720D00468002C1CD0207806281C
:1092F00019D16078032802D006280FD109E0042292
:10930000204639461C30B0470822391D20462430FB
:1093100003E01022204639460C30B0476178E8B2AD
:109320000022FFF79FFEF8BD4468002CFBD0207898
:109330000628F8D160780D2802D00F280FD109E057
:109340000422204639462030B0470822391D2046E5
:109350002C3003E01022204639460C30B0476178AB
:10936000E8B20022FFF75EFDF8BD10B50146B9482E
:10937000FDF7BFFA10BD30B4B44C8300E3580029A8
:1093800010D0012910D0022912D0032912D151780E
:1093900003290BD04033197889070BD03D2230BC0C
:1093A00009215FE61278FAE71A22F8E79278F6E7E1
:1093B0005278F4E730BC704710B5A44C8300E358F2
:1093C00000290ED0012903D0022901D0032907D199
:1093D00040331978890703D03D221321FFF722FD7E
:1093E00010BD1278F9E770B5054698498000085815
:1093F0000024C18FC90702D14068002802D024246C
:10940000204670BD0122FF203823114607300AF0A4
:1094100073F90246062010700A2050700121362090
:109420008154284604F024FC00220A212846FFF734
:10943000F9FCE5E710B58549820089580024CA8FF8
:10944000D2070AD0096800290DD0097806290AD167
:1094500000220121FFF706FE06E04968002902D03C
:109460000978062902D02424204610BD00220B21B1
:10947000FFF7D8FCF8E7F7B500980D468100734870
:1094800000264458E08FC0070BD02068002825D064
:109490000078062822D13D2209210098FFF7E2FD3D
:1094A0001DE060680C27002814D10122FF2038231A
:1094B000114607300AF020F90746062038700020D0
:1094C0003621C8553A460121009804F0D1FB0A2004
:1094D0007870074660680178062902D02426304655
:1094E000FEBD0446A97A687A09020143A18629468D
:1094F000042213312046564B1C3098472946082237
:109500000B312046524B243098470822691C504B9F
:10951000201D9847002239460098FFF783FCDEE7BC
:10952000F8B50E4605468100484800244058C18FD2
:10953000C90706D00068002809D0017806290FD095
:1095400005E04068002802D00078062802D02424D4
:109550002046F8BD3D2213212846FFF763FCF7E7BC
:109560003146074604220931394B203098470822FA
:10957000711C3846364B2C3098470022042128466F
:10958000FFF770FDE4E710B53049820089580024E8
:10959000CA8FD20706D00968002909D009780629A0
:1095A0000ED005E04968002902D00978062902D0CA
:1095B0002424204610BD3D221321FFF733FCF8E799
:1095C00000220521FFF74EFDF3E710B51F49820089
:1095D00089580024CA8FD20706D00968002909D00B
:1095E000097806290ED005E04968002902D00978DB
:1095F000062902D02424204610BD00221021FFF7A6
:1096000011FCF8E700220821FFF72CFDF3E7FFB576
:109610000E4982008E58002581B0002E1ED037469C
:1096200040373978C943890718D0F18FC90715D059
:10963000042815D22821895DC907C90F00D001214E
:1096400000290DD0797809070CD505E0909200200B
:10965000190F0000BF9200183A252BE00C2529E0D5
:109660001A2527E00102491CFF2038230A4607304B
:109670000AF042F80446062020700020607004982A
:10968000002805D0A0860822344B201D0399984756
:1096900010222046314B0C3002999847F08F8006FB
:1096A000C10F3620015520460AF03FF8787808218E
:1096B00008437870284627E4F8B5294F0646850008
:1096C00078590C2400282ED04022125CD2439207F5
:1096D00029D04068002826D00278062A23D1427873
:1096E0000E2A20D10024002905D010221B4B0C305B
:1096F0009847002213E02030807D00280ED0012101
:10970000304604F0F5FA78590122C18F5202914394
:10971000C18706213046FFF797FA04E006220E21A2
:109720003046FFF77FFB2046F8BD70B500250446A4
:10973000FF290AD00125002104F09AFA00221146DF
:109740002046FFF78FFC284670BD0549A000085849
:10975000403081782046FCF7E8FAF4E7190F000062
:10976000909200203EB56C462170EB236370D122AD
:10977000A2700122E27000226271A271E271227273
:109780002271092906D19B4A810051582031097A5A
:109790000B4063700022214604F02EFC3EBDF8B55C
:1097A0000F4606468100934844582568687800288B
:1097B00015D0012826D01F27E87800280AD0224695
:1097C00028323946304603F0F2FE40346078FB21FF
:1097D000084060700021304604F08AFAF8BDE08F3E
:1097E0000106E9D4C00701D0082100E00E2130466F
:1097F000FFF7B8FF0120687002460021304604F0F0
:109800004DFAF8BD00221146304604F047FAD3E77E
:1098100030B400290ED001290ED002291ED0032910
:109820001ED151780E291BD19178002918D01A2900
:1098300006D011E01178F8E751780E2910D11A21DD
:10984000042809D26B4B82009A58002A04D0203297
:10985000137A0824A343137230BCA0E75178E4E7DD
:1098600030BC704770B5634A8300D2580024D38F50
:10987000DB0701D0242418E013464D7820321572FE
:109880008D785572CD7895720D79D5724D791573A5
:109890008D795573CD799573097AD173D98F8022DB
:1098A0001143D9870921FFF75DFF204670BD70B5D0
:1098B000504A8300D2580024D38FDB071AD01346B6
:1098C0004D78203215728D785572CD7895720D795C
:1098D000D5724D7915738D795573CD799573097A54
:1098E000D173D98F80221143D9870921FFF73AFF1D
:1098F000204670BD2424FBE770B53E4D84002B59F3
:109900004E781A46203216728E785672CE7896723B
:109910000E79D6724E7916738E795673CE79967308
:10992000097AD173D98F80221143D98729590968BF
:10993000002905D00978022902D10021FFF72FFF65
:10994000002070BDF8B5014682002A4800248058E6
:10995000021E0AD0054640352B78DB439B0704D016
:109960006B785B0703D53A2426E00C2424E000261C
:109970000127042907D22030007A0823184000D09C
:109980000120002806D1D08FC20703D1000601D4E0
:109990001A2411E00902491CFF2004230A4607305B
:1099A00009F0AAFE022101704670C77009F0BDFEE1
:1099B00068780421084368702046F8BD70B500251A
:1099C0000446FF2909D00125002104F051F90021A6
:1099D0002046FFF7E4FE284670BDD0780028FAD074
:1099E0000449A0000A584220815C2046283203F036
:1099F000DEFDF0E790920020F3B50646FE4A8000B7
:109A0000155800272C6883B06178002902D00129FD
:109A100070D13BE001216170E98F09060CD5042E5D
:109A20000AD21058002807D02130007A08210840B7
:109A300000D0012000280AD1E088F049884200D3F4
:109A40000846E0806089884200D308466081E38848
:109A5000A1886289248914276D462F706C70240AAE
:109A6000AC70EA70120A2A716971090AA971EB7166
:109A7000190A297230460022694604F0BDFA012213
:109A80000021304604F00AF905B0F0BD002211466D
:109A9000304604F003F90498002819D1298A208956
:109AA00081420BD1E989A288914207D1A98A6289B2
:109AB000914203D1698AE288914209D0009063897A
:109AC000A288E188304602F006FA00281FD000275D
:109AD000002F0FD020892882A088E8816089A88281
:109AE000E0886882208900906389A288E1883046F6
:109AF00003F031FEE078002804D040356878DF219B
:109B0000084068700021304604F0F2F8BCE70127F5
:109B1000DEE7FFB583B003980C9C8500B64840593A
:109B2000C58EA54200D22C46058FA7B29D4200D318
:109B30001D467C237C2A00D91A464524240116465A
:109B4000A14200D80C46C18F09060CD503990429FF
:109B500009D2010007D02921095C0822114000D058
:109B60000121002906D1A5498D4200D30D468C4222
:109B700000D30C46018AB14208D1C189B94205D14E
:109B8000818AA14202D1418AA94211D00682C781AD
:109B90008482458223463A4629460096039802F07D
:109BA0009AF923463A4629460096039803F0D3FDD6
:109BB0001522694603980A704E70320A8A70CC707A
:109BC000220A0A714F713A0A8A71CD712A0A0A7201
:109BD000002204F011FA07B0F0BD30B4002910D013
:109BE000012910D0022920D0032920D1517814292D
:109BF0001DD1917800291AD0192908D01A2906D028
:109C000011E01178F6E75178142910D119210428B0
:109C100009D2794B82009A58002A04D02032137A54
:109C20002024A343137230BCE6E65178E2E730BC4F
:109C30007047F8B5704B82009A5800255268002A88
:109C400001D0242529E08B784E781C024A1C34432D
:109C50001B2C1DD3537916791A0232431B2A17D3B2
:109C60000B79CE781B023343FF264936C91CB34219
:109C70000ED34F7909793F023943B14208D3FB2C07
:109C800006D8FB2A04D85E4EB34201D8B14201D9AE
:109C9000202502E00094FFF73CFF2846F8BDF8B508
:109CA0000A460546810054480024405801680029AE
:109CB00002D00878042801D0242443E09078567814
:109CC0000002531C30431B2816D35E791F793602DD
:109CD0003E431B2E10D31679D77836023E43FF271A
:109CE0004937D21CBE4207D35679177936023E4314
:109CF000FF274937BE4201D220241FE08E888642CA
:109D000000D23046888050781778CE8800023843D9
:109D1000864200D23046C88058791B790E890002ED
:109D20001843864200D230460881507912794B8917
:109D300000021043834200D218464881214628463B
:109D4000FFF75AFE2046F8BDF7B517462A498200AC
:109D50008C580025002C0AD0264640363178C9435D
:109D6000890704D07178890603D53A2531E00C259E
:109D70002FE004282FD22821095D2022114000D095
:109D80000121002927D0E28901998A4202D1618A02
:109D9000B9421BD00102491CFF200C230A460730A0
:109DA00009F0AAFC04210170002141700121C17059
:109DB00001998180C7807C21018145210901418170
:109DC00009F0B3FC70782021084370700198E08698
:109DD00027872846FEBD1A25FBE738B5002405462F
:109DE000FF290FD00124002103F042FF0021284663
:109DF000FFF702FE204638BD909200204808000080
:109E000090420000D0780028F4D00020034602469B
:109E100001460090284603F09EFCEBE730B5F74C76
:109E20000398E47AA40701D5012400E006248A42BD
:109E300016D8FF25F435AB4212D81925ED01A942F9
:109E40000ED8A2420CD3A8420AD80A2808D30A2264
:109E500050438A00891849085B1C5943884201DA3B
:109E6000002030BD012030BDF0B50C460746E44966
:109E700080000E588DB0384602F041F9A1880222C8
:109E800049000091E18849000191A189022900D887
:109E900011460291E1890222022900D81146254685
:109EA00020350391E9786A46490091741782F18F51
:109EB000C9070BD10199401E081807F09DFB084601
:109EC0000299C91C02910399C91C0391C107C90FCA
:109ED0006A46D174E17800291DD1697A00291AD126
:109EE000618AC84A914216D0002914D0A1886A46D6
:109EF0004900089102990991118A9185618A490066
:109F00000818A188490007F077FB08A80A9102F019
:109F1000B4FD00280BD0684602F04FFD00280AD09F
:109F20000020E084E088A084E8700DB0F0BD608A75
:109F3000E084089815E0F18F0698C90704D1401C09
:109F4000059907F059FB084683B20598218AC0039A
:109F5000020C384602F02BF8AB4907F063FBE084B3
:109F60000598C003000CDEE770B586B014466A465B
:109F7000117005460822211DA44E00A80130B047EB
:109F80002320005D6A46507221460E22103102A83D
:109F90000230B04700226946284604F02DF806B08A
:109FA00070BDF7B5164686B0954A810001905458A9
:109FB0002922F178925D114301D0012700E00027AA
:109FC0000799002945D1B18C2289914207D1328964
:109FD00063899A4203D17289A3899A4205D021816B
:109FE000318961817189A18101271C21884A4143FE
:109FF0008D18B1890222022900D811460491F189F5
:10A000000222022900D81146039102F078F800904C
:10A01000208940000290284602F0C9FC0298A880DE
:10A020000098E8800498288103996981E08FC0072F
:10A030000CD10098A988401E081807F0DDFAE980C5
:10A040002889C01C28816889C01C6881284602F0C4
:10A050007CFC002F07D0A089009063892289079992
:10A06000019803F009FBF078002804D040346078B0
:10A07000EF210840607009B0F0BDF0B51646074604
:10A0800085B0BA005E4B00929D5800202C680629CE
:10A090000BD062788A427DD161780B0007F084FB97
:10A0A000072B280896BCBABCBA0006216170F3E7FA
:10A0B00000221146384603F0F1FD002E18D0042F7F
:10A0C00016D24F4900980858002811D02030007A45
:10A0D00000210222104000D00120002808D0E88F83
:10A0E000C00704D11C204A4A78438018C17393E00A
:10A0F000012028210855E88F10210843E8872046D1
:10A1000020300390007A0028384626D001F040FF26
:10A1100001463B4A009810584089C2008018081830
:10A1200009302084039A012191702082214638460B
:10A13000FFF79AFEE28CE2832089238C61896E46C8
:10A140000BC60398A38C8178384601F083FE06463F
:10A1500004206070002E5FD121E001F019FF208201
:10A1600021463846FFF780FEE08C60822548A082B9
:10A17000E08220836083A08322460F213846FFF7C8
:10A18000F3FE01220021384603F088FDE88FC00766
:10A1900003D000E018E002202EE003202CE0002194
:10A1A0006A4611700399384689785170E18B518065
:10A1B000A18C91802189D18061891181218C51816B
:10A1C0000022694603F018FF05B0F0BD00221146D9
:10A1D000384603F063FD002E1ED12089228C618950
:10A1E0006B4607C32220015DA38CE28B384601F049
:10A1F00031FE060010D104206070E5E75091002088
:10A2000090920020FFFF0000E2040000190F000000
:10A21000CC9000200028D7D0E078002805D128462F
:10A22000403041784906490E417022463146384651
:10A23000FFF7B7FE0021384603F05AFDE88F1021E2
:10A240008843E887C0E730B4F84B84001B59DC8FA3
:10A25000E40701D0022400E00324002910D00129E2
:10A2600011D002291FD003291FD151780F291CD1E9
:10A270009278002A19D0192A09D01A2A07D00FE09B
:10A2800006241278F5E751780F290ED11A220428F6
:10A2900006D2002B04D02033197A0225A943197263
:10A2A000214630BCE9E65278E3E730BC7047F7B5A9
:10A2B00084B0049B16469C00DC4B00221D591046BE
:10A2C0006C680B290BD063788B422DD16178C91F44
:10A2D0000B0007F069FA05113D077F7F7B000B211A
:10A2E0006170F3E7002E75D100220121049803F07C
:10A2F000D5FC012028210855E88F10210843274666
:10A30000E8872037387A002810D02089228C61898C
:10A310006B4607C3A38CE28BB978049801F09AFDD1
:10A32000060057D10A20607007B0F0BDA1882889C7
:10A33000814216D8E288824213D322896B899A42DD
:10A340000FD16289AB899A420BD1A0802889E08025
:10A35000002E12D0002332460F21049803F09CFEF9
:10A3600041E0608900902389E288049803F0CCF9E9
:10A370000820607001207872D6E7E88FC00713D0FC
:10A3800004982A230102491CFF200A46073009F0DD
:10A39000B3F9A74B05462A22214698470120687049
:10A3A000284609F0C2F91EE021460498FFF75CFD3B
:10A3B000224610210498FFF7D7FD09206070012282
:10A3C0001146049803F06AFCAEE703E0002AABD024
:10A3D000002808D1224631460498FFF7E2FDE98FB4
:10A3E00010208143E9870121049803F081FC9BE759
:10A3F000092300290AD0022906D003290CD151785B
:10A40000102909D1927803E0527801E012780B23E9
:10A41000002A01D019464AE77047F7B582B00C46CA
:10A420000298824980000E5820890090A188174622
:10A430000025E3880A460298FFF7F0FC002803D0C5
:10A44000F08FC00741D101E020253FE060897949C4
:10A45000381A80B2884201D2282537E030680028B7
:10A4600002D00178032904D070680921002813D094
:10A4700027E0A1888184E188018121894181618966
:10A4800001846188C1836178203081702A4603216C
:10A490000298FFF7F2FD19E00122FF202A2311465E
:10A4A000073009F029F90246032010700021D1700D
:10A4B00029208154481E50820121029803F0D8FBC4
:10A4C000072170680278032A02D0242528467BE6FB
:10A4D0004170A2888284E288028122894281628955
:10A4E00002846288C2836278203082700122027204
:10A4F00000220298FFF7DBFEE8E7F7B582B00C46D2
:10A5000002984A49800008580190406800270028B6
:10A5100001D0242779E0207AE179000208430090F5
:10A52000A079617903020B43A078617802020A43A3
:10A530002179E07809020143E61C651C0298FFF7C7
:10A540006DFC00280AD00198C08FC00708D00321F5
:10A55000029803F0F6FC070002D056E01E2754E0F4
:10A5600002982A230102491CFF200A46073009F0FD
:10A57000C3F8024603201070072050700023D370E8
:10A58000697828780902014391807178307809024E
:10A590000143D180687929790002084310817079DC
:10A5A00031790002084350811146657A2031CD701F
:10A5B000E07AA57A000228431082607B257B0002A6
:10A5C00028435082E07BA57B000228439082607C78
:10A5D000257C00022843D082E07CA57C0002284331
:10A5E0001083607D257D000228435083E07DA47D9B
:10A5F0000002204390834B720121029803F038FB44
:10A60000002207210298FFF752FE3846DCE5F7B535
:10A6100082B0029800278200044880580468002C09
:10A6200002D02078032807D0242759E090920020F8
:10A63000190F0000FF7F0000087ACA79000210435A
:10A6400000908879CD1C4E1C497903020B43707829
:10A65000317802020A436978287809020143029896
:10A66000FFF7DCFB002833D0707831780002084314
:10A67000A18888422ED3E288944690422AD86A78EC
:10A680002B7812021A43624524D88A4222D3727967
:10A69000337912021A4323899A421BD1814200D98D
:10A6A0000846A08068782A7800021043844500D9C3
:10A6B0006046A08068792A7961890002104381424E
:10A6C00000D9084660810020E0832034A07002E0B9
:10A6D0001E2700E020273A4602210298FFF7CDFC12
:10A6E000384671E5F8B50C4605468000A149009052
:10A6F00008580026002810D0074640373978C9434B
:10A7000089070AD0042D0AD22821095C02221140AF
:10A7100000D00121002902D004E00C2648E0C08FBF
:10A72000C00704D07878C00603D53A2640E01A2640
:10A730003EE02902491CFF202A230A46073008F080
:10A74000DBFF03210170002141700123C370618888
:10A75000628949008A4200D21146C181218822893A
:10A7600049008A4200D2114681816188C1802188D6
:10A770008180A1880181E18800224181042D0CD2D1
:10A780007C4C00996158002907D02031097A0222B7
:10A79000114201D0012200E0002201465A4020313E
:10A7A0000A724B7208F0C1FF787810210843787064
:10A7B0003046F8BD10B503466E4A9C0012590C2075
:10A7C000002A25D04024A45CE443A40720D052688A
:10A7D000002915D0002A1BD0D4884888844200D98B
:10A7E0002046D08090880C88A04200D820469080D7
:10A7F0005489C888844200D920465081002202E052
:10A80000002A05D03B2208211846FFF750FD002002
:10A8100010BD70B514460646564A800000251258F1
:10A82000FF2912D0D08FC00602D5607800281CD036
:10A83000012522460021304603F01AFA61780022F1
:10A840003046FFF71AFC284670BDE078002806D095
:10A850004032917822463046FFF7A3FBF3E74032BF
:10A8600050784006400E5070EDE70225EBE7F8B552
:10A870000D46100A1C21404A414300278C18FF2B2B
:10A8800006D0DEB2314602F0DCFE012E0BD014E021
:10A89000E088A188401C06F0AFFE288888420CD0D2
:10A8A000204602F084F82888A1884018401E06F04F
:10A8B000A3FEE180204602F048F83846F8BD70B5A6
:10A8C000C5B22C4EAC003059002850D04030017831
:10A8D000C94389074BD04078C10648D4C00946D146
:10A8E0002902491CFF202A230A46073008F004FFEA
:10A8F0001C21214A6943335989180A89DB8F498908
:10A90000DB0701D1C91ED21E03230370002343704D
:10A91000C3708281C18131590989C1803159098946
:10A920008180315949890181315989894181315960
:10A93000CA8FD2070BD0042D1AD2002918D020318B
:10A94000097A0222114000D00121002910D00022F2
:10A95000014620310A724B720021C943418208F03E
:10A96000E4FE30598022403041781143417070BD7F
:10A970000122EDE790920020CC900020F7B582B044
:10A98000029817468200FD4800268558002F2C6843
:10A9900005D000221146029803F080F9E8E06078C3
:10A9A000884278D1030006F0FFFE0504403BC2EB6D
:10A9B000BB00E88F10210843E8872846E179203062
:10A9C000C176A1798176E17A0177E179EA7D480063
:10A9D000D040C00705D0A079AA7D4000D040C00774
:10A9E0007ED1A27916266B4602981E7099705A7015
:10A9F0000022694603F000FB01220021029803F0C7
:10AA00004DF9E88FC00701D00220B7E0A0790121FD
:10AA1000C00700D00021029801F09DFA0320ADE0AC
:10AA200000221146029803F039F9A079012100288B
:10AA30000CD0AB7D4200DA40D20701D0002002E00A
:10AA4000800702D50220207200E02172E079002800
:10AA50000CD0EB7D4200DA40D20701D0002002E0AA
:10AA6000800702D50220607200E06172A07A00289F
:10AA700012D0207AA97D002801D04108491C607AB3
:10AA8000EA7D002801D04208521C914204D00020E7
:10AA90006072207246E043E0207A002802D1617A99
:10AAA00000293FD0A97D002801D04108491C491E3A
:10AAB000C8B20090607AE97D002801D04108491CA5
:10AAC000491ECFB2029801F063FA6989CA00891859
:10AAD0004018093083B2A3803A460099029800E0FA
:10AAE00045E001F014FA07001ED001260020A080E6
:10AAF00020726072627A217A9446A2886B469646EA
:10AB0000182202981A70597062469A707246DA706A
:10AB1000110A19710022694603F06EFA002E41D124
:10AB200005B0F0BD0126E5E704206070E2E70022F1
:10AB30001146029803F0B2F8207A002802D1617A17
:10AB4000002915D0617AAA7D002901D04A08521C3B
:10AB5000521ED1B2EA7D002801D04208521C521E7A
:10AB6000D2B2A388029801F0D2F9070005D019E00B
:10AB70000421029801F0EFF914E004206070CFE79F
:10AB8000E88FC00702D0617A207A01E0217A607AEA
:10AB9000002902D04908491CE975002802D0400864
:10ABA000401CA875E98F10208143E987E0780028D0
:10ABB00005D1207A002802D1607A00280DD0EB7DE3
:10ABC000AA7D3946029802F0E6FDE078002804D01C
:10ABD00040356878BF21084068700021029803F072
:10ABE00087F89DE7002910D0012910D0022920D034
:10ABF000032920D1517816291DD19278002A1AD024
:10AC0000192A08D01A2A06D011E01278F6E75178EE
:10AC1000162910D11922042809D2584B81005958FD
:10AC2000002904D021310B7A5B085B000B720021F4
:10AC3000A4E65278E2E77047F8B517460646820068
:10AC40004E48002F85586C6804D00421304601F02E
:10AC500082F914E06078884258D1052813D006287C
:10AC600055D0072852D1207A002802D04008401C35
:10AC7000E875607A002802D04008401CA875E88F6B
:10AC8000C10767D075E0E88F10210843E887C00747
:10AC90001ED03102491CFF200C230A46073008F061
:10ACA0002BFD05210170012141700021C170294651
:10ACB00020318A7EA3791A408271CA7EE3791A40D4
:10ACC000C271097FC172A17A817208F02EFDD6E7A8
:10ACD0002035A87EA27901211040C00700D00021B4
:10ACE000304601F038F906206070A97EEA7E17230D
:10ACF0006C462370A270617030460022694603F0F2
:10AD00007BF901221146304602F0C8FFF8BD00224F
:10AD10000121304602F0C2FF207A002802D1617A78
:10AD2000002992D0617AAA7D002901D04A08521CDC
:10AD3000521ED1B2EA7D002801D04208521C521E98
:10AD4000D2B2A388304601F0E2F8070097D107207D
:10AD50006070F8BD10218843E887207A002802D16E
:10AD6000607A002805D0EB7DAA7D3946304602F096
:10AD700012FD0121304602F0BBFFF8BD9092002089
:10AD8000002901D1127857E7704770B50C46064686
:10AD9000A1498000085800254168002901D02425D8
:10ADA00037E0A17800290CD06178002909D0C08F44
:10ADB000C00708D00521304603F0C3F8050002D0D3
:10ADC00027E01E2525E03102491CFF200C230A46FE
:10ADD000073008F091FC0521017041706178C17164
:10ADE000A17881710246A0786178884206D1002856
:10ADF00004D0411E084201D1012000E000209072E1
:10AE00000121304602F034FF002205213046FFF7D1
:10AE100013FF284670BD70B57F4A83008C78D258E6
:10AE20000025002C02D04B78002B00D11E25D38F9B
:10AE3000DB0705D01368002B02D01A78052A01D051
:10AE4000242517E09A7922409A71DA794C782240C9
:10AE5000DA718C7849788C4206D1002C04D0611EBE
:10AE60000C4201D1012100E0002199722A46022101
:10AE7000FFF784FD284670BDF8B513464A780546AD
:10AE800096080024B600C81C002E03D18E78B7089F
:10AE9000BF0001D020240DE0002A01D1002E09D0EE
:10AEA0004678077836023E439B1B5C4E9BB2B3420A
:10AEB00000D22824584BAE009E593368002B02D094
:10AEC0001F78052F08D07368002B02D01E78052E3E
:10AED00010D02424204650E71A728978597241789C
:10AEE0000278080210439880224603212846FFF783
:10AEF00045FDEFE71A7289785972417802780802A5
:10AF000010439880224606212846FFF795FEE1E788
:10AF100002469300404A0C20D258002A0AD040230F
:10AF20009B5CDB439B0705D0D07D4870907D08700B
:10AF3000002088707047F8B50C468200364900261C
:10AF40008F583146042807D2002F05D02921C95D2A
:10AF5000C907C90F00D001214D0001210D43002F69
:10AF600009D040373978C943890704D07978490630
:10AF700003D53A2625E00C2623E06178294202D049
:10AF80002178294201D11A261BE00102491CFF2029
:10AF90000C230A46073008F0AFFB052101700021A1
:10AFA00041700121C17061782940C1712178294027
:10AFB0008171A178C17208F0B8FB7878402108430C
:10AFC00078703046D9E6F8B515460746124A800033
:10AFD00000261458FF2912D0E08FC00602D56878E9
:10AFE000002817D001262A460021384602F040FEEC
:10AFF000697800223846FFF7C1FC3046BDE6E878A4
:10B000000028FAD0E37DA27D4034A178384602F0D2
:10B01000C2FBF2E70226F0E790920020FF7F0000DB
:10B0200070B5304D1C21A87A48432F494418A08C94
:10B03000002802D108F0C0F8A084208A4004400C07
:10B040002082A87A0621401C06F0D6FAA97270BDAB
:10B0500024491C22897A5143234A89180A8AD20B2F
:10B0600005D0898BC90A814201D101207047002097
:10B070007047F8B50E46054608F06CFA194CC02228
:10B08000A17B1346CB40217BC0B20907090F0B43BC
:10B090008707BF0F0121B9400B432B70A37B1746D5
:10B0A000DF40237B1B091F436F70A37BDA4033070C
:10B0B0001B0F1A43AA70627B00095201203202431F
:10B0C0000A43EA70607B0321401C06F095FA617325
:10B0D000A07B0221401C06F08FFAA173207B401C4C
:10B0E0002073F8BD5091002000830020F8B5FE4980
:10B0F00080000C5826464036F08D009000281DD068
:10B10000FA48216E0289708E0F4610184143F848A4
:10B11000192278439202801A06F06EFA401E85B218
:10B120003946606E06F068FA401E854200D2284615
:10B13000009980B2884200D30846F085F8BDF8B582
:10B140000F46E94980000C580821F940E07D23466C
:10B15000101A8033E74AC01E5043420894465A7B77
:10B160004820D04062460830101A5A881D78963818
:10B170001E46904200D310464822FA400832801AF8
:10B180004034E28F520601D58A00801A06F034FA64
:10B19000854200D22846B071F8BDF8B5D24A810088
:10B1A000555800902E468036B07B4822C2407088A9
:10B1B000B1880832884200D80846101895304000FF
:10B1C000CC4906F019FAEA7D296E401C8A1A101A39
:10B1D000801E2F4644084037F88FC00713D0C3485D
:10B1E0007A8E0089801848431921890106F004FAF3
:10B1F000C049103006F000FA241A388E002802D018
:10B20000844200D30446009870214843BA4941184B
:10B210000C80B94940394018C4877088B1884018FB
:10B220004B214000C9004018A8652861F8BDFEB553
:10B2300007468000AC4A0190105800284AD00646C4
:10B2400038020A46411CAB48633808F07FFA3046A2
:10B250002430009008F087F83446054680341CE01E
:10B26000207AA17A800040180006010DA348091831
:10B27000488F8007800F012806D0022804D00328B9
:10B2800002D1888F08F005F8207B0421401E20732E
:10B29000A07A401C06F0B0F9A172207B0028DFD113
:10B2A000308C002809D007F0F4FF06E0A88807F0EA
:10B2B000C4FF009808F057F80546002DF6D139462E
:10B2C000042001F04DFC304608F0B0F986490198A1
:10B2D00000220A50FEBDF8B50546834980000C588F
:10B2E000844B264640362902B078643B491C01282D
:10B2F00004D002280DD0032824D10FE003221846E1
:10B3000008F024FA2846FFF748FF226E8034A17B1C
:10B3100015E00822184608F019FA13E0052218462D
:10B3200008F014FA204620302746417C8037797394
:10B33000007CB8732846FFF730FFB97B226E2846A1
:10B34000FFF7FDFE0020B070F8BDF7B588B0089893
:10B350008C46810064483C274458002005902546CF
:10B3600000904035E88F666C810727D5C00725D04F
:10B370002146002080310874002A1FD05B48C07B22
:10B3800000281BD1E88D002818D0EA8F530515D569
:10B39000530713D4120711D4AA78002A04D0AA8E16
:10B3A0002B8812189A4209D2226E42439219160132
:10B3B000EA8E36091018E886012008740121C906B2
:10B3C0006046801B00010009884207D2206E801968
:10B3D0000601E88E3609401CE886F1E7606D0190B1
:10B3E000A878012846D1204620300290C07F00284E
:10B3F00040D1A88EE98E40182988401A81B2404871
:10B40000814237D20298807F002820D1208F801976
:10B410000601E88F3609C10704D0A18F49088919B0
:10B420000E013609226B2266618FE985626B6266C6
:10B430000121029AC007917706D08820005DFFF7AE
:10B4400055FEE88FC00702D102990120C877019606
:10B45000A88EE98E40182988401A80B205E0226E35
:10B460000199891A0901090901910146401E80B21A
:10B470000029F4D1E88F800701D5606E01E0206ECD
:10B4800080000390C6E00296E88F0690C00764D063
:10B49000002004902A20285E0090E16C701A0101BF
:10B4A000124809090289688E101848431921890138
:10B4B00006F0A2F8470006984037800705D401201F
:10B4C0000490A88D0B494843C719A878012807D1D3
:10B4D00020462030817F002902D0C07F002811D073
:10B4E0000498002813D018E06091002050910020AB
:10B4F00090D0030071020000808100208083002032
:10B50000FF7F0000A08FFD494843C71905E0FB49B4
:10B51000206E48434008B84270D979080491F74931
:10B52000049806F069F80299091A090109090291BB
:10B53000F24948430499091A0098401A009008D526
:10B540000298EE49401E0001000902900098401840
:10B550000090A060A06DC119216102986060204632
:10B5600000F015FF002860D0A07D401CA075206E63
:10B5700080190601E88E3609401C81B2E986A87858
:10B58000012847D1204620300290C07F002841D1B9
:10B59000A88E40182988401A81B2D948814239D2F0
:10B5A0000298807F002821D1208F80190601E88F22
:10B5B0003609C10704D0A18F490889190E0136093F
:10B5C000226B2266618FE985626B6266C00703D0D9
:10B5D0008820005DFFF78AFD029901208877616E5F
:10B5E0000391E98FC90701D10299C8770196A88E06
:10B5F000E98E40182988401A80B206E012E0226ED7
:10B600000199891A0901090901910146401E80B278
:10B610000029F4D10198301A0101039809098142E7
:10B6200000D230E7059800280CD000208921085569
:10B630006664E88FC00703D0009828853C37A7646C
:10B640000BB0F0BDE88F800701D5082100E03E2156
:10B650000898FFF7ECFDF3E7F0B5AA4980000D5814
:10B6600087B0E86A002808D1686AE862002804D038
:10B67000C0888105890D7C2041532C464034E08FE1
:10B68000EE6AC00609D5002E07D0A08F002802D18F
:10B690003068002801D0012000E000200290298CB1
:10B6A000014318D02F468037387B042815D1F87A0B
:10B6B0000421C01C05F0A0FF387A8000081800069D
:10B6C000010D91480818018FC90B04D1428F102138
:10B6D0008A430A43428707B0F0BD04900428FAD297
:10B6E000288C002807D0698C0390032001900091DA
:10B6F000002028842DE002980028ECD0A08F00289C
:10B7000008D13068002805D00646E862C088800568
:10B71000800DA087F088B1888205920D8A18A18FCC
:10B72000521A92B203928204920F012A00D002228E
:10B730000192BA79914200D3114600910321090385
:10B740008843012109034018F080A08F0099401A16
:10B75000A087387A82000292F87A1118C9B205914E
:10B760000421C01C05F048FF029A8818C2B2E08F7D
:10B77000C10609D5002E07D0A18F002902D131685A
:10B78000002901D0012100E000210291410603D5EA
:10B790000099091D89B2009181040DD402990029F4
:10B7A00008D1C00708D00198032803D05748C07AB1
:10B7B000C00701D0012000E00020059B00999C46B5
:10B7C00009020001019B01431943634618014E4BD6
:10B7D000C018418703998187E18F890409D4110139
:10B7E000C9180A8FD20B04D14B8F102293431343F5
:10B7F0004B87018F4904490C0187F87A0421401CCA
:10B8000005F0FAFEF972387B401C38730498401C2E
:10B81000C0B262E7FEB505007ED02E468036377A8C
:10B8200000202C46403401970290A08EE18E4018F3
:10B83000A086019F70214F433549791800910886F1
:10B84000E08FFF2101318843E087800516D5E08E27
:10B85000F1794843618F4018252105F0CDFE08B2EB
:10B86000002801DA253000B2294AC1B2403ABB189B
:10B870001A8D920992010A431A8560870020E0869A
:10B88000E08FC0071BD0A86C2249401C40088842AA
:10B890000CD91A494A1E801805F0AEFE0121C903D1
:10B8A00001431B4840383818C18508E0C103012016
:10B8B000C00308181649000C40397918C885A178CA
:10B8C000002941D0A08E2288801A0D4A80B2904271
:10B8D0003AD22846203002290CD1009A298E518074
:10B8E000009A698E91800099027DCB885B095B018B
:10B8F0001343CB80A17803291ED10EE07102000012
:10B90000FF7F000060910020808300205091002084
:10B9100080810020FF3F000029E0FF49427C791828
:10B92000CB8A0C27BB4392001343CB82027CCB8A89
:10B930009B089B001343CB82A178012902D1C07FD1
:10B94000002801D0012002900020019B00901A469F
:10B95000F249284600F042FE707A022801D0012008
:10B9600070720298002802D0307AFFF7B4FCFEBD56
:10B9700010B5040015D008F0E9F80146226E606C9D
:10B98000801800010009606420464030C28E521CBD
:10B99000C286A07D0022401CA0758034207AFFF76B
:10B9A000D4FC10BDF1B500988100DD484458214613
:10B9B0008031487A00282AD125464035E88FC007D3
:10B9C00025D0087C002822D0274608F0BFF8616CFB
:10B9D0000646881B0001216E0009884217D9002104
:10B9E000384600F0CDFD216E06E0401A0001000946
:10B9F0006064E88E401EE886606C821B12011209AA
:10BA00008A42F2D8002231460098FFF79EFCF8BD2A
:10BA1000F3B587B00798C24E8700F0590C250C4645
:10BA200000287DD10021942007F0A6FDF0510028C8
:10BA300076D007460020029008F088F80590079815
:10BA400094220490B74B002138469847B648F861D5
:10BA5000B648B8610320F87500211020B960B875A8
:10BA60004002B8823E46803607983D4630724035E7
:10BA7000E88F420820785200002800D001200243BD
:10BA8000012080028243EA870020A886E886688732
:10BA900020462030039000798000A885608C8100CA
:10BAA000F9652089810039666089E885A0894101AE
:10BAB000796603984079F071A07BF8F779FC688685
:10BAC000E88F10210843E88700213173B172F172C9
:10BAD0003984F962A9871B22FF21328049317180A4
:10BAE000B180B27103998979717303998979B173BE
:10BAF0000021F173C00702D0307AFFF7F7FA2178FE
:10BB0000049800297ED0032170225043824A0346C4
:10BB1000801800900190018203981121807900E043
:10BB2000E6E009028200114301430198C1820498B2
:10BB3000010220200143019841820198218AC1839A
:10BB40000198618A0184A17E607E09020143019807
:10BB500041840198E17E828C120A12020A43828497
:10BB6000E07B002800D00120F1790122D2034003BC
:10BB7000C9060243C80C024301980285664A0021A7
:10BB80004032981804900187E98F10158143E07BBB
:10BB900000286CD0002040020143E987019906206B
:10BBA00048850798FFF7F9FA04997C2008810499E1
:10BBB000002048810146019A1E20D085049AA08A5F
:10BBC0005080049AE08A9080049A207ED080019868
:10BBD00041870198C28ED209D201C2860198828D16
:10BBE00052085200828500200190307A019980002D
:10BBF00004904018C0B20690481C042105F0FCFCDB
:10BC0000049800E031E0081801060A0D7721C90008
:10BC100051188A080121C9030698114302014448BA
:10BC2000101801870021418781870198401C0190ED
:10BC30000428DADB307A81017720C00008180099E7
:10BC400080088886EB8FD80713D00399E0698A793A
:10BC5000FF215931D140228C083149005118354C0F
:10BC600089B28446624202910FE002214CE7012032
:10BC700091E7E1690020F9646885E06913E009193A
:10BC8000401C89B20001000902919142F7D261463D
:10BC9000F96402996985F96D001D0818A98D490894
:10BCA000081800010009F96C396579657864D807CE
:10BCB00000D00298D90700B2288504D01D4AA98D6A
:10BCC0005242514300E03C21B964D90700D1002021
:10BCD000B860002205990798FFF737FB0020009015
:10BCE000388A317A83B204203A6E00F026FF0025AC
:10BCF000284609B0F0BD70B505460C22EFF310845C
:10BD000072B683000648C058002826D0034680300B
:10BD1000427A002A13D00FE0408100203F400118F2
:10BD200060910020750F000071B9001815B8001857
:10BD3000808300208FFDFFFF012A0DD10AE000293A
:10BD400008D00021184600F01BFC16212846FFF7FA
:10BD50006EFA01E002214172002284F3108810463D
:10BD600070BD70B505460C20EFF3108472B6AE00BE
:10BD7000ED4B9B59002B0DD01A8459844033D88F3A
:10BD800008210843D8872846FFF766FC2846FFF7B6
:10BD900009FE002084F3108870BD70B5054684004C
:10BDA000E2480C23005900282FD040300278D243BB
:10BDB00092072AD0CA88960522D0C678002E04D0D1
:10BDC0009E02B243CA800022C270EFF3108672B6A0
:10BDD000D5480059002810D00446243007F0A6FAB0
:10BDE00020464030C18F08221143C1872846FFF703
:10BDF00033FC2846FFF7D6FD002386F3108804E0C5
:10BE00009104890F01D10121C170184670BD70B530
:10BE100006460C20EFF3108572B6B300C24AD25822
:10BE2000002A14D014464032D08F102398430B01BF
:10BE30001843D087002909D03046FFF70DFC803425
:10BE4000207B002802D03046FFF7ACFD002085F3B0
:10BE5000108870BDF0B504460C20EFF31086079FE4
:10BE600072B6A500B04C6459002C16D0254640355A
:10BE7000A87800280DD10120A8702F808800A08705
:10BE800090002087980020630598608706984001FD
:10BE9000606300202034A077E07786F31088F0BD3F
:10BEA00070B50C24EFF3108572B683009E48C0581D
:10BEB00000280CD0034640339E78002E07D1022480
:10BEC0009C701A8005229A4B30309847002485F3E5
:10BED0001088204670BDF8B507460C20EFF3108699
:10BEE00072B6BD00904C6559002D0DD02C468034A3
:10BEF00022806180A3803846FFF74FF9A17B384646
:10BF00002A6EFFF71CF9002086F31088F8BDF8B5FB
:10BF100094460C27EFF3108672B68400824A1459B7
:10BF2000002C14D025464035AA78002A0FD10322D0
:10BF3000AA702B80224620321174634653748E22DD
:10BF4000125D8A4202D9226EFFF7F9F8002786F3C4
:10BF500010883846F8BD70B505460C20EFF3108404
:10BF600072B6AB00704AD358002B0AD004290BD00C
:10BF70008E20C05C884203D91A6E2846FFF7DFF88E
:10BF8000002084F3108870BD1A6E8033997BF4E72B
:10BF900001460020EFF3108272B68B006249C95847
:10BFA000002901D04031888E82F310887047F8B59F
:10BFB00000259C462E462C46EFF3108772B6830070
:10BFC0005948C058002807D0034640339C8EDB8E6A
:10BFD000466CE318056E9CB287F310880123601A43
:10BFE000DB03984200DC081B910400B20C0C684390
:10BFF000614680194900401A00010009214605F0F8
:10C00000FBFA601AA04200D100204A494843401C74
:10C010004010F8BD10B5444A8300D258002A10D011
:10C0200070235843444BC018438A0424A3438C0014
:10C03000234343824032D08F4023984389010843F1
:10C04000D08710BD10B5384A8300D258002A10D0CE
:10C0500070235843384BC018438A0224A3434C0032
:10C06000234343824032D08F202398434901084321
:10C07000D08710BDF0B52C4C8300E358002B2ED098
:10C080002D4F7023002458434037C3199C84DC840F
:10C090001C855C859C85DC85234615196E782D787A
:10C0A00036022E435D004519ED19AE83A41C5B1CBE
:10C0B000DBB2E4B2042BF0D300220F23CC18257896
:10C0C0001D3C247F2D0225436CBA55004519ED19FE
:10C0D000AC819B1E521CD2B2DBB2082AEED3F0BD5B
:10C0E00001460020EFF3108272B68B000E49C9584A
:10C0F000002901D08F20085682F31088704710B5B0
:10C1000001460020EFF3108472B68A000649895870
:10C11000002906D0086D096E4008490805F06CFA40
:10C1200088B284F3108810BD6091002090920020A6
:10C13000190F0000710200004081002072B6BFF3A9
:10C140004F8F04490248C860BFF34F8FFEE70000DD
:10C150000400FA0500ED00E0F3B581B00F46486831
:10C1600001994968421A140101222409D206944215
:10C1700003D9081A0001000944420198BD68866885
:10C18000002C02DC28D1AE4226D20069FA493018D0
:10C19000451B281E04DD681E05F044FA201A03E042
:10C1A00005F040FA201A401C002801DD0020FEBDE9
:10C1B0003869F149281A002804DD401E05F032FADA
:10C1C000201A03E005F02EFA201A401C002801DD99
:10C1D0000120FEBD0220FEBD3F69E749E819801B32
:10C1E000002805DD401E05F01DFA0019401C02E084
:10C1F00005F018FA0019002801DC0520FEBD0198A1
:10C20000DD4900693018401BC01B002804DD401EBA
:10C2100005F008FA201A03E005F004FA201A401C81
:10C22000002801DD0320FEBD0420FEBDF1B584B071
:10C23000D24800900027046857E0A08A2268810550
:10C24000890E0292820B4ED000294CD0002201921E
:10C250001646A27D03071B0FD2180901049D103951
:10C26000A2758905890D3F22120190430143A182E5
:10C2700034E029462046FFF76FFF002830D005281C
:10C280002AD02969A8684618BB49304605F0B4F998
:10C2900001466868B84B40185943A268711A8A422F
:10C2A00000D2401C060136096660A08A800B022875
:10C2B00012D3B149206905F09FF9E1680346881B54
:10C2C000000101220009D206904203D9701A000130
:10C2D00000094042834206DC2E462D68002DC8D15D
:10C2E0000198002817D02746029C002CA5D1009861
:10C2F000006800280DD0082105200007016282692E
:10C300008A430A43826101680122D20691431143A4
:10C31000016005B0F0BD22463946009807F048F8A4
:10C320009648224631460C3807F08EF8DCE7FEB519
:10C3300092480C380068002826D0C27D4168876882
:10C34000891A0E013609684607F00BFC019D8A48E0
:10C35000FF359135009C854204D340422D18641C62
:10C3600024012409301B000101210009C90688426B
:10C3700003D2B44203D1AF4201D826462F463946F4
:10C38000304607F00EFBFEBD0021481EF9E7F0B570
:10C3900005467A4887B00C38059000200646019083
:10C3A000009007460290EFF31080069072B603A843
:10C3B00007F0D7FBE97D03987D224018049900011E
:10C3C000D2006D4B000989185B4203E0C918401C7C
:10C3D00000010009684A9142F8D26A68131A1C01E8
:10C3E00001232409DB069C4204D282420DD1AA68B3
:10C3F00091420AD9AA8A920B1FD06860AA688A4221
:10C4000003D2401C000100096860A88A800B022842
:10C4100016D35949286905F0EFF8EA6869680446B7
:10C42000501A000101230009DB06984203D9881A3B
:10C43000000100094042844202DD0120029094E0A4
:10C440004E480C388468002C67D10598046864E075
:10C4500021462846FFF780FE002860D0052839D005
:10C46000A97DA27D91420FD9444B0C3B9B68A3420E
:10C470000AD0002E00D126467F1CFFB2009401286E
:10C480004DD003284BD025E0AB8A9B0B17D02169F8
:10C49000A06846183849304605F0AEF80146606895
:10C4A000354B40185943AA68711A8A4200D2401C81
:10C4B0000001000900266860374600960AE09142B4
:10C4C000BBD92E490C398968A142B6D1032826D0A0
:10C4D0000428B2D1A88A800B022815D326492869DE
:10C4E00005F08AF80346E86869688446401A000146
:10C4F00001220009D206904204D96046081A0001C0
:10C5000000094042834298DC1C480C388068A042F5
:10C510009BD0002F00D101942468002C98D1029860
:10C52000002822D1002E0AD01448009A0C38019914
:10C5300006F04BFF31461148009A06F002FF0198C1
:10C54000002806D001460D482A460C3806F07CFF2C
:10C5500006E00A4829460C3806F0FEFEFFF7E7FE23
:10C56000002E02D02846FFF761FE069880F310885F
:10C57000029807B0F0BD000071020000C4910020D5
:10C5800070B504460026EFF3108572B600281FD060
:10C5900011488268A24202D10021816018E000297E
:10C5A00016D10068A04205D10B4806F0DCFEFFF76B
:10C5B000BEFE0DE02146084806F0DFFE002807D148
:10C5C000054821460C3006F0D8FE002800D102268E
:10C5D00085F31088304670BDB8910020FFB5394D05
:10C5E0000646EC7CA87C81B0201A0007000F8C4620
:10C5F0000E2801D3012000E000200090314AA00065
:10C60000803A811877680F64111980310B70614688
:10C6100011500120298AA040014329822A49220180
:10C62000B0885718788070680001000DB880308994
:10C6300027210901081AF88024493069884208D95D
:10C640002349401804F0D8FF0121C903014379812F
:10C6500005E0C1030120C0030818000C78810A9886
:10C660001F211F2800D308460002B881F8891F2126
:10C67000090288430F2109020843F88103987021B9
:10C680004843FF30513080083881B07D1F211F287A
:10C6900000D308460099C0028902022208431043D1
:10C6A000388090070B4920430860E87C401C000755
:10C6B000000FE8740848018820221143018005B06A
:10C6C000F0BD00004C92002000800020FF7F0000A1
:10C6D0007102000000010050F08F0020FFB58FB004
:10C6E000064611981F46304363D0012E01D1002F1A
:10C6F0005FD000200690012E04D011988068002E93
:10C7000002D006E07868FAE71099002901D0119864
:10C71000C0680890012E0AD01198008A0990012E55
:10C7200007D01198C07C002803D0012002E0B8890E
:10C73000F4E70020009007F009FA0001C00F019013
:10C74000D04800218160D0488079002815D0019818
:10C75000002812D1CB4804680DE0A58801202946A5
:10C76000000704F049FF681AE1884018294604F0E0
:10C7700059FFE1802468002CEFD1C34901988871EA
:10C78000012E14D011984069019008980D900198DD
:10C7900000280ED00D9800280BD0012E0CD0009848
:10C7A00000280BD00125B7480468059482E038685A
:10C7B000EAE7012013B0F0BDBD68F4E70025F2E719
:10C7C000002E04D11098002801D0678900E0278945
:10C7D000A088029000286CD0002F6AD0A189099807
:10C7E000814266D001990298884200D3084604909D
:10C7F0000D9839180498814201D90320DAE7E088BE
:10C80000049904F0F9FECF1907917F1E049901984D
:10C8100004F0F2FE00294CD10499029804F0ECFED9
:10C82000002946D12846049904F0E6FE0D980A91A5
:10C830000818401E03900798814201D3B9421ED9BF
:10C8400007990398884201D3B84218D90A988842B8
:10C8500002D80398B84212D20498874206D3014600
:10C86000384604F0C9FE0A98814208D20499039818
:10C8700088421ED304F0C0FE0798814219D3012ECE
:10C8800004D0781C049904F0B7FE05E07D48019DB2
:10C8900084600CE004980918A942FBD900980D4661
:10C8A000A84303D100988143C80700D06D1C059CA4
:10C8B00000E02468002C02D00198854280D30198C2
:10C8C000854202D3032006903DE0002E3BD1119813
:10C8D0008561119846690898019500901198AD19E5
:10C8E000008A03906D1E059C25E0A1890398814272
:10C8F00020D0A0880290B04201D3374600E007461E
:10C900003946304604F078FE002913D139460298A2
:10C9100004F072FE00290DD1E088394604F06CFE67
:10C9200000E0C91901988142FBD90098081AA84271
:10C9300000D205462468002CD7D13146284604F0A1
:10C940005BFE1198C161069834E71FB504468088E4
:10C95000009020890190A08969468881E0880022A2
:10C9600002906B4611460120FFF7B8FE032819D14B
:10C9700044488068002815D0E17B002902D1C27BA1
:10C98000002A0FD0002901D0224600E002460029EB
:10C9900005D0C37B002B02D0994200D20246908979
:10C9A000FDF78DFF2146374806F0C0FC1FBD10B5CE
:10C9B0000146344806F0E1FC10BDFEB5044640686F
:10C9C00000906061216800980291814242D2002566
:10C9D000ED432E4600212B4809E08289238A9A42A2
:10C9E00005D0491C8288C9B2B24200D216460068FE
:10C9F0000028F2D1002908D00098B0420FD3314668
:10CA000004F0FAFD704305461DE0A67C002E1AD006
:10CA10003146009804F0F0FD3546454313E00746E3
:10CA20000020019009E03946304604F0E5FD002978
:10CA300002D101203D460190BF1E0298B84202D8A3
:10CA400001980028EFD00298A84203D80098A84285
:10CA500000D365610023224601211846FFF73EFE00
:10CA6000002809D0E268A168914205D2002322463D
:10CA700019461846FFF732FEFEBD00220346114656
:10CA800001202BE660920020C0920020F8B53E48BD
:10CA90003C4981800021C94301603C48384F4668C9
:10CAA0001DE0304606F027FD1F210D1A3748A9006A
:10CAB00009188C68002C0FD069000818008B3449C5
:10CAC00004F09AFD201A84B2022C01D9A41EA4B24B
:10CAD000A74200D23C46A7B20120A8408643002EC0
:10CAE000DFD1294A2A4990884F43B84200D33846BB
:10CAF000908026480068411C0AD011684B1C06D063
:10CB0000091A090101230909DB06994200D31060C3
:10CB1000F8BD022801D11D480160B7E710B5022811
:10CB200002D11A49C01E0860FFF7B0FF164800681E
:10CB3000401C01D101F0EEFE10BD30B4032801D03D
:10CB400004280BD111488C002418A2604A00121846
:10CB50001383012342688B401A43426030BC95E73F
:10CB6000032801D0042809D108488B0000221B1893
:10CB70009A60012342688B409A43426086E7000036
:10CB8000FFFF0000E4570000C09200206C920020DC
:10CB900071020000F7B50098164605020F46002402
:10CBA000681D06F010FE4322102811D00099BB002A
:10CBB0008A00F8498958CA58B2421CD00122BA40AA
:10CBC000024201D0022408E0C88DC00607D54322E6
:10CBD000334639460098FAF72FFA2046FEBDCE506C
:10CBE0000124D6B2681D06F0EEFD30430146681DF3
:10CBF00006F0BEFDF1E70124EFE7FEB5100A0C4692
:10CC00000A4601210090FFF7C5FF029001287AD162
:10CC10002178204605260C30F602DF4D01900B00EE
:10CC200004F0C2FD107109471A713A3A5365685E03
:10CC3000A7D9BD71FE716088FF2201461739EA321B
:10CC4000D64C914200D8A083042202210098FAF722
:10CC5000DAFB0146A08B8AE06078022815D010220A
:10CC6000062108320098FAF7CEFBA1884180E188BE
:10CC70008180C6806278214608310746042A06D0A2
:10CC800038460830A8473946E1E00222E8E738464E
:10CC90000830FAF712FDF6E7082211460098FAF775
:10CCA000B2FB0146A0884880E0888880BC4ACA80E0
:10CCB000CDE0082210210098FAF7A5FB0146A088D4
:10CCC0004880E0888880CE80C1E006220421009858
:10CCD000FAF799FB0146A0884880E0888880B6E092
:10CCE0000098AC4980000858806800280CD0E08883
:10CCF000002835D006220C210098FAF784FB014663
:10CD0000E088888032E0C1E0A188E088814201D9D2
:10CD10004022B7E0207A102805D0042803D002284A
:10CD200001D05122AEE0022810D010220821921D1D
:10CD30000098FAF768FBA1884180E1888180227A17
:10CD4000214609310646042A02D005E00222EDE719
:10CD5000B01DFAF7B2FC01E0B01D76E0314676E096
:10CD600004220A210098FAF74EFB0146A088488069
:10CD70006DE060780E214200921C0098FAF743FBA8
:10CD80000146002207E09000001953005B188088DC
:10CD9000521C588092B260789042F4D857E02646F0
:10CDA00024890098FAF7E1F9C01E844200D2204697
:10CDB00087B2381D82B252210098FAF724FB04464C
:10CDC000B08860803A46201D0199A847204608385F
:10CDD00006F0ABFC5AE06078002809D00098FAF71A
:10CDE000C4F92189C01E884202DBE088002820D0D7
:10CDF0006189208981422ED2461A0098FAF7B5F946
:10CE0000401F864200D2304687B2B81D82B216213A
:10CE10000098FAF7F8FA0646A0887080E08800E0EB
:10CE200036E061893A464018B08061890198091856
:10CE300092E7091D8AB212210098FAF7E4FA064631
:10CE4000A08870802289301D0199A84786E7009844
:10CE500003F013F91AE06278002A0ED0022218219A
:10CE60000098FAF7D0FA014660892289904201D1F0
:10CE7000012000E000204870E9E7814201D1002252
:10CE800000E0522201210098FAF703F90298FEBD52
:10CE9000022218210098FAF7B6FA01466078EAE70C
:10CEA00010B51046140A06F08EFC102802D0204659
:10CEB00003F0DAF8002010BD70B5150A0E460A46D8
:10CEC00000212846FFF766FE0446012816D13148A6
:10CED000A9004058806A002806D04088B18888425E
:10CEE00002D12846FAF7A4FD31462846FAF736FE65
:10CEF000020003D000212846FAF7CBF8204670BD87
:10CF0000F8B515460C460027104606F05CFC1028C4
:10CF10006CD0280A1F4E8500009073598446186A09
:10CF2000002801D0017D00E000212278402A04D0B1
:10CF3000412A0ED0422A59D146E0002956D0986A9B
:10CF4000002802D00C3806F071FB7059012784626A
:10CF500049E0122906D0182910D0522907D0D22929
:10CF600023D104E0627861886046FAF754FE705974
:10CF7000203006F0F8F906F059FB13E06378002B37
:10CF800010D0628818216046FAF736FE0098FAF74A
:10CF900017FEECE7B4900020190F00006490002009
:10CFA000032800000098FBF7FAFB607800281DD1E9
:10CFB0007059806A002819D040886188884215D14C
:10CFC0000098FAF735FD11E016290FD16378002B90
:10CFD0000ED062886046FAF70FFE7059203006F0D6
:10CFE000C2F906F023FB0098FBF7D9FB3846F8BDE1
:10CFF000A1880122D20311434182F4E7FFB581B039
:10D000001746104606F0DFFB3D0A102821D02F4EB0
:10D01000AC003059C08DC00606D42D483A460059A0
:10D02000C1892C4806F092FB30591022C18D114362
:10D03000C185152101988901401A02D0012808D123
:10D0400002E04522012101E0452200212846FAF7AD
:10D0500020F8002005B0F0BD70B516460D4610460C
:10D0600006F0B1FB0024102825D02878360A0028C5
:10D0700004D0342812D03F2810D024E0294630466E
:10D08000FBF7BCFB0446FF281DD12946304603F0C0
:10D090008DFC0446FF2816D1002414E0297A4A06A4
:10D0A00011D43F2805D0042300223046FAF7A4FD0E
:10D0B00009E00623F8E72878002804D168880028CA
:10D0C00001D006F08FF8204670BD0000B49000201B
:10D0D0008C9000201B05000030B504460120F84D5F
:10D0E00000218A0052199268002A09D0537B022B32
:10D0F00001D0012B04D1527CA24201D0002030BDCE
:10D10000491CC9B20429ECD330BD10B5F9F74DFD67
:10D11000EB4C002291000919896800290DD0CB7BC6
:10D12000032B0AD14B7B002B02D0022B03D004E04F
:10D13000097C890601D5401CC0B2521C042AE9DBD7
:10D14000032801D3012010BD002010BD70B50E468C
:10D1500005460021304606F00FFA04000AD0D94BEC
:10D1600032460021984725730020E073D449A80077
:10D1700040188460204670BD30B50023D04C0AE0D2
:10D18000820012199268002A04D0D57B8D4201D109
:10D19000134602E0401C0428F2DB184630BD01466D
:10D1A0000120002904D1C64820300079C007C00FF3
:10D1B000704770B50D00044607D0007B00F074F98D
:10D1C00029460120F9F790FC70BDA18A03230622AD
:10D1D000BD4806F091FA217B0170617B417006F039
:10D1E000A4FAB74820300079C007C00F0ED0B44968
:10D1F00020461630B34B06221E3106465C3B98474C
:10D20000607B002805D0304603F027FC0120E07346
:10D21000D6E7207B314603F06CFCF7E770B5044697
:10D220000D460120F9F760FC002D01D0012003E03C
:10D23000E07B022801D10320E07370BD70B50D467C
:10D240000446818AA04804230622401C06F054FAB2
:10D25000217B0170617B4170857006F066FAE07B8E
:10D26000042819D1964900204968002900D008787F
:10D27000A52802D0A62805D00EE000210120F9F74C
:10D2800033FC09E0207B0321401CC0B2FFF774FF90
:10D290000028F2D0416888470120E07370BD10B5C6
:10D2A0008749044649680020002900D00878A7284B
:10D2B0000CD0A8280ED1207B0121401CC0B2FFF762
:10D2C0005BFF002802D08168884703E0002101202D
:10D2D000F9F70AFC207B00F0E7F810BDFFB581B03C
:10D2E0000D460120F9F7E2FB009001287BD1297857
:10D2F00000260846A43834460427714A030004F087
:10D3000053FA050425313A4A57006878294604281B
:10D3100061D2800080188768002F04D0F87B012834
:10D3200003D0032804D0432456E00220F87305E01C
:10D33000787B0028F7D1B87B0028F4D13A683846CA
:10D340009047040048D00120F87345E0687804282D
:10D3500041D28000801880680028E4D0C17B032976
:10D36000E1D105E003210020FFF706FF00281DD0D2
:10D37000C77341680DE0687804282CD280008018BB
:10D380008068002812D0C17B0129CCD10521C1734E
:10D390008168884720E003210020FFF7EDFE002888
:10D3A000C1D10121FFF7E8FE0028EFD1012613E0EB
:10D3B00004200024A3009B189B68002B16D0641C3B
:10D3C000E4B2042CF6D3042812D0A02912D0A1294B
:10D3D00016D0A2291AD040242046304303D021463B
:10D3E0000120F9F781FB009805B0F0BD2046EAE77F
:10D3F0004B24F1E769782B1D049A02F038FA03E018
:10D400006978049A02F0F2FB0446E5E76978049A29
:10D4100002F04FFDF8E710B502462B480C460123F9
:10D420000621401F06F068F9047006F07EF910BD71
:10D4300010B5084600781946002800D09030204BDF
:10D44000C2B2586800281DD0007800281AD01846AB
:10D45000203040798000C0188068448A8C4211D105
:10D4600000234382437B002B04D0012B05D0022BE9
:10D4700008D105E002F059FA04E002F0E1FB01E016
:10D4800002F07FFD002010BD10B514460246FF20BB
:10D49000002903D121461046F9F744FB21780029E1
:10D4A00001D102F031FD10BD810010B504480C1807
:10D4B000A068002801D006F0B9F80020A06010BDD7
:10D4C00064900020750F0000A4060000F7B582B03C
:10D4D00016460546F9F79DFC04020090E01D06F093
:10D4E00072F93F2823D000988700C248C05981892B
:10D4F000FF2900D1C189E21D0423BF4806F0FCF8D2
:10D500000580867006F011F9BA48C0598289FF2A51
:10D5100008D00398002800D09030C3B201210098B1
:10D52000F9F786FB324629460098F9F726FB05B045
:10D53000F0BDF8B516460D46F9F76BFC0746040238
:10D54000E01D06F040F93F2812D0B800A94900902C
:10D5500008580068002806D00278032A03D1002D5D
:10D5600007D09035EDB22A4600213846F9F771FB15
:10D57000F8BD0C380189A048E21D0623001D06F005
:10D58000BBF8044630782071B088608070882080B5
:10D59000204606F0CAF820790628E4D89549009874
:10D5A000FD2208584030417D11404175DBE7F7B559
:10D5B0000C46F9F72EFC06460502E81D06F003F9B5
:10D5C0003F283DD08B4AB700D1590868002832D097
:10D5D0000378042B2FD1002C0DD090344031887962
:10D5E000E4B2800627D5A12C21D01CDC912C1ED0C2
:10D5F0009C2C20D11BE00C380189E120EA1D082376
:10D60000C00006F079F8054602987C4B017879480D
:10D61000C05940304175082228460299984728464B
:10D6200006F083F807E0A92C01D0AA2C03D1487D8D
:10D63000FD2210404875224600213046F9F709FBCB
:10D64000FEBDF8B50C460546F9F7E3FB06460702B2
:10D65000F81D06F0B8F83F280DD06649B00008580C
:10D66000FA1DC18964480423401E06F045F8058070
:10D67000847006F05AF8F8BDFFB581B00F46F9F78F
:10D68000C8FB05460602F01D06F09DF83F281FD096
:10D690003C469034574A3946112F0BD006DC0029FE
:10D6A0001DD0012906D00C2F2AD103E0192901D061
:10D6B0001A2F25D1A9005058403083799B061FD5D9
:10D6C000437DFD24234043755058806806F02DF8B3
:10D6D0002DE7E2B202212846F9F7BBFA27E7A800B6
:10D6E0001058F21DC189444806230E3006F004F894
:10D6F00003990180049941800A99818006F015F808
:10D70000002FE6D10024E4E7FFB581B015460E46B0
:10D71000F9F77FFB04460702F81D06F054F83F288E
:10D7200018D03548FA1DF91D0E230B3005F0E4FF23
:10D730003049A2008958022340314A7D1A434A7574
:10D7400009210170858046800499C1800A99018170
:10D7500005F0EBFFEBE6FFB581B01C461546F9F787
:10D7600058FB06460702F81D06F02DF83F2811D099
:10D770002049B0000858FA1DC1891F4808232930E4
:10D7800005F0BAFF0A998180C48005800299418022
:10D7900005F0CBFFCBE6FFB581B00D46F9F739FBBD
:10D7A00004460702F81D06F00EF83F2821D0114E5E
:10D7B000002D0ED1A0003058FA1DC189732002231C
:10D7C000000105F099FF049941700399017005F07B
:10D7D000ACFFA0003058806800280AD000781728D5
:10D7E00007D1002D00D09035EAB202212046F9F78A
:10D7F00030FA9CE68C90002003070000190F00000F
:10D8000070B50124094D8440288800290BD020429E
:10D8100005D16888002802D0062006F07DF8288807
:10D820002043288070BDA043FBE700008C920020BD
:10D83000FFB583B00D46044600210C980193271DC7
:10D840008E4B0091002814D026887C207C2E00D995
:10D85000064628883246C1190198984705980680DF
:10D860002888801928802088801B2080009807B095
:10D87000F0BD6188207904290AD18149C140C907D6
:10D8800006D10121298078702088401E20807F1CCD
:10D890007C482188808B884202D231200090E6E7C4
:10D8A000764B0422214601989847019826887821D2
:10D8B000001D782E00D90E46704B324639469847E7
:10D8C0000599301D0880CBE7FEB51D460023019366
:10D8D0006D4B800014461B580A9A081D099E009043
:10D8E000022A21D10879012222804A88042A08D1FB
:10D8F000634AC240D00704D1022020800888401C1F
:10D900000880587C1946401FC7B2228800981731FA
:10D9100010185A4B3A469847781C2988C0B2081A02
:10D9200028802088C0192080002E12D02888B0427C
:10D930000DD321880098514B081832460899984712
:10D940002088801920802888801B288001E03420CE
:10D9500001900198FEBDF8B506464B4980000C5871
:10D960000025A068002806D0342101730C3005F092
:10D97000DCFEA56011E0207C617C88420DD2042889
:10D980000BD3A28A101F022807D80095A37D34214B
:10D990003046F9F74AFD05F0C8FE2574042060748E
:10D9A000F8BDF7B582B0002001900F4602983649C5
:10D9B000800016460C5821E0904214D2121A8A4276
:10D9C00000D2114622468DB2123280182B4B2A46C5
:10D9D00039689847207C401920743088401B30807B
:10D9E000386840193860207C042807D1608A0C21EF
:10D9F0000C2800D30846617C40186074207C627C4F
:10DA0000904202D231880029D6D1C0B2D1B2884228
:10DA100030D1A68A658AA77D301F02281FD81948F1
:10DA2000808BA84206D3042E06D10298F9F79DFBFD
:10DA3000A84201D2312006E0002D03D00198002831
:10DA40001AD001E034200190002000903B4632467D
:10DA500001990298F9F7E9FC0C38A060E581A0680B
:10DA6000002807D00199002904D00C3005F05DFE94
:10DA70000020A06005B0F0BD2846E6E7190F0000C1
:10DA800022AA0A4364900020C090002010B50C46E2
:10DA90000102491C0346002C11D0FF200230002A4D
:10DAA00014D0FA4A9B00D258002A0BD040239B5C2A
:10DAB000DB439B0706D0F64A05F09EFE10BDFF2013
:10DAC0000130ECE792890A235A43F5E705F0E7FEB7
:10DAD00010BDF8B506468700EC48C559002D28D082
:10DAE0002C6A03E02046246805F0A0FD002CF9D143
:10DAF0000124A0002858002802D00C3805F096FD1B
:10DB0000641E64B2002CF4DA002211463046FFF79E
:10DB1000BDFF002201213046FFF7B8FF3002FF2190
:10DB2000401C05F025FE284605F080FDD748002161
:10DB3000C151F8BDF8B5D54C06468700E0590D46F1
:10DB4000002802D0FF242046F8BD0021442005F023
:10DB500013FDE051002862D0044630020021401C31
:10DB600005F006FE4422CB4B002120469847298928
:10DB7000218169896181A989A18129462046C54FF2
:10DB80000522143118305C3FB84720462830EB217D
:10DB90000170D1214170012181700821C1700021E3
:10DBA000017141718171C1711B23FF21E3814931F1
:10DBB00061822382A182B84926228B8FE386C98F96
:10DBC0002187515D0838491CA175E17502216177F3
:10DBD000B14940310A7882764978C176E08F4108B0
:10DBE00028784900002818D000200143E187294601
:10DBF0003046FDF70DFF04461C204643A64806228A
:10DC00004038361830461430A91CB8476878B076CA
:10DC10002878F0760920B07395E70120E5E707241E
:10DC200091E770B5994C8300E358002B1AD040332C
:10DC30001C78E543AD0715D0A508ED43AD0711D01D
:10DC4000002910D0012905D002290BD1A108890093
:10DC5000114319701978F32421409200114319706F
:10DC600000F086F970BDA00880001043187070BDE8
:10DC7000F8B504020646641C17460D46204605F01A
:10DC8000A2FD824AB1005158AA008F500121A9403B
:10DC90000143C9B2204605F06BFDF8BD30B47B4BA3
:10DCA00084001B59002B10D08C001B59002B0CD06A
:10DCB0009C78002C0BD0012C0ED0022C14D0032CFD
:10DCC00003D1002A01D00220987030BC7047002A8E
:10DCD000FBD001229A7001E0002A02D0012230BC60
:10DCE000D4E600229A70FAE7002AEED10320EBE78F
:10DCF000F8B505460002401C0F46009005F063FD94
:10DD000006466249A8000C58002239462846FFF70B
:10DD1000C5FFBD0060590C3805F088FC002060513B
:10DD2000FF2E06D00120B84031468143009805F00F
:10DD30001FFDF8BD70B51C461546544B82009A581D
:10DD4000002A11D08B00D258002A0DD0127813006F
:10DD500003F02AFD090A060B101A1F2933380A009E
:10DD600022462946FAF7C0FF70BD22462946FBF736
:10DD70004FFD70BD00292246294602D0FCF738FB32
:10DD800070BDFCF760FA70BD22462946FBF725FFFF
:10DD900070BD00292246294602D0FCF7F1FF70BD74
:10DDA000FCF720FF70BD00292246294602D0FBF770
:10DDB00003FB70BDFBF7DFFA70BD22462946FAF778
:10DDC000A5FE70BD2246294603F0BBFB70BD70B5B1
:10DDD00013461C0A2D4B0A46A5005B590020FF2163
:10DDE0001578002B0BD04026F65CF643B60706D01C
:10DDF0001968002907D0072D04D0022070BD072D17
:10DE0000FCD200E009782B0003F0CEFC0805060ADE
:10DE10000E12161A1E05F1E72046FAF76AFF70BDCA
:10DE20002046FBF7CBFD70BD2046FCF7F2FC70BD31
:10DE30002046FBF7D2FF70BD2046FDF7C4F870BD49
:10DE40002046FBF772FC70BD2046FAF7AFFE70BDAE
:10DE5000100A10B5D9B20D4A8300D258002A3DD01D
:10DE600040239B5CDB439B0738D01368002B1AD000
:10DE70001B788B4217D1032902D005292ED10DE042
:10DE800000220421FCF7F9F828E00000909200201D
:10DE9000409C0000750F00000C910020002204211E
:10DEA000FCF76CFD1AE05268002A17D012788A42FB
:10DEB00014D1032904D0052907D008290ED109E07F
:10DEC00000220A21FCF7F3F908E000220721FCF701
:10DED000B3FE03E00022042103F00AFB002010BD82
:10DEE00010B5100A01222221FAF7BCFD002010BD56
:10DEF00010B51E4B84001B59002B10D08C001B59F1
:10DF0000002B0CD09C78002C0AD0012C0CD0022CB9
:10DF100010D0032C03D1002A01D10020987010BD2D
:10DF2000002AFCD00320F9E7002AF8D002229A70D8
:10DF3000002203E0002AF2D101229A70FFF7A6FD29
:10DF400010BD0246094B92009A5800201268002A20
:10DF500003D012788A4201D123207047032A03D0CC
:10DF6000052A01D0082AF8D12A2070479092002073
:10DF7000F8B50746824980000D58E88F800728D4FD
:10DF800001262A4640327F4B2C6A32E01078617AB3
:10DF90000007800F4900C9184978C140C807C00F61
:10DFA00025D005F05AF92146774B09310090C01869
:10DFB000764B227A9847E88F02210843E887217A36
:10DFC0003846009AFDF7CDFE002803D0009805F0F2
:10DFD00060F9F8BD002EFCD12846203021460546C8
:10DFE00005F0CBF92146284605F0B6F9F8BD2468BE
:10DFF0000026002CCAD1F8BDF7B50F46009860493D
:10E0000080000E58002F1ED0002E1CD03878192802
:10E0100019D25C4940000D5C012128460C3005F006
:10E02000ABFA0446029860602046584B2A463946AF
:10E0300009309847304625722146203005F076F9A0
:10E040000098FFF795FFFEBD70B50C460B460546E0
:10E0500002220021FFF76EFE2346022201212846FC
:10E06000FFF768FE002070BD70B50C460B460546F4
:10E0700003220021FFF75EFE2346032201212846EA
:10E08000FFF758FE002070BD10B50B46012200219D
:10E09000FFF750FE002010BD38B504280CD2384DD3
:10E0A00084002C59002C07D02034247A04252C40DD
:10E0B00000D00124002C01D10D2907D911246D466F
:10E0C0002C70AA7069701A46694605E00D216C46ED
:10E0D000217062701A466946FFF78EFF38BDF0B5B1
:10E0E0000C460546264980000E582188264B1822EA
:10E0F000C9188BB0254B01A898474036307869463F
:10E1000080070979800F192926D21E4B4A0066889C
:10E110009F5CBE422AD1D2185278C240D2071DD08D
:10E120008800194664390B58E28801A928469847A7
:10E13000010009D03D2914D0684600790A460146FD
:10E1400000232846FFF7A8FF208805F04BF80BB006
:10E15000F0BD022804D0F7E7002807D00128F8D145
:10E160003D2101222846FAF77DFCEDE707226B46A8
:10E170001A705970284600226946FFF73DFFE3E711
:10E1800090920020E05A011800800020190F000032
:10E19000F7B5164607468500FE494859002828D09D
:10E1A00004460021FEF7ECF9A08E000702D50220FC
:10E1B000FEF7B4FC0198002815D00423FF220021AB
:10E1C000F54805F099FA077000214670C170002EDD
:10E1D00005D0218F002902D02034A17E00E000214B
:10E1E000817005F0A2FAEB4C605905F01FFA00208F
:10E1F0006051FEBDF8B51F4600230D4606461C467D
:10E20000002A04D0104605F06FF883780488B10026
:10E2100048190006020DE1481218908F568F9B1D79
:10E22000F6B21B021E4356879487012D10D10B06B0
:10E23000548F0421240924010C435487190D77239A
:10E24000DB00C918138F89089B0B9B030B431387B3
:10E25000002F03D0002801D005F04BF8F8BD38B5E9
:10E26000002817D0014620310C46CA7E416A4B1C5B
:10E2700008D04368CA4DC91AC9037023090C534317
:10E280005B1919800C2100911346C649FEF7A6F9C7
:10E290000120207738BD70B504003DD0A08E254602
:10E2A00000072035002803DAA07D401CA07523E07C
:10E2B000A16A6068411A0A01E16A120949008A42AA
:10E2C0001AD3A17D491CA175A06205F043F9112163
:10E2D00003F092F94804E97F000C002907D00028D8
:10E2E00002D0202802D002E0012000E01F20616857
:10E2F00008180101090961602046FEF748F8002866
:10E300000AD0E87F002807D1606A401C04D0E87E6C
:10E310003C220121FFF73CFF70BD30B5EFF31083C5
:10E3200072B684009B48002500593A242554028780
:10E33000828E120704D5012241681203891804E075
:10E34000002905D04268490151180901090901E075
:10E350000021C94383F31088416230BDF7B586B010
:10E3600006988C4D8600A8590C2400287ED10021E7
:10E37000402005F001F9A851002877D005460698FD
:10E380001C214843884940180190046905F0DEFBD0
:10E39000069A039202904022844B00212846984717
:10E3A0008348E8618348A8610320E8750520A875C3
:10E3B0000020A8608048A88228462030069A009055
:10E3C0000146C276A068E8626088A886607F4877C8
:10E3D000207F401E887708982887F0B2761CF7B215
:10E3E00004900026607805F05FF80146A88E132897
:10E3F0000AD004DC10280DD012280FD108E015280F
:10E4000004D01D280AD101E06C4805E00126FBE795
:10E410000626F9E76A480226414329610498012E3D
:10E4200004D1617BC90701D0012300E00023217BD7
:10E43000DB01CA076349520EC97A4907C90F8C46E6
:10E440000321490219430A43614649010A43010174
:10E45000524832430E187287217B0422C907490EA5
:10E4600011433A0110180592049000E0F4E041874E
:10E47000A88E400716D500980621C07E4B4B484316
:10E48000AF21C9004718504821460E3106223818DE
:10E490005C3B9847708F0321C0B2890208437087A4
:10E4A000B7870DE001980023027D19460698FFF713
:10E4B000A1FE01980023827D01210698FFF79AFEB4
:10E4C000A88E410701D4800704D4308F800B8003CD
:10E4D00030870EE077210598C9004018318F8008F9
:10E4E000890B8903014331870498018F4904490C42
:10E4F0000187308F4004400C3087A88E28490207DE
:10E50000069870235843403946180190002A0CDAC7
:10E51000029849144018010109090220FEF7F9FA8E
:10E520002A4881880520296100E004203082A078F3
:10E53000400701D5002000E0A07E01020198F1848F
:10E54000214BFF308D30C0182146184B0E3106226A
:10E550005C3B9847124A0198617B801807464182CC
:10E56000A88E000702D4F120000200E01848308590
:10E570001F2070850098C07E8006000E0101772064
:10E58000C00008188008B0860E498888F083C888C3
:10E5900030841FE0A092002006020000808300204B
:10E5A000808100202F430118CC900020750F0000BF
:10E5B00097E200185FE20018016000002E070000DB
:10E5C000B20500005091002000800020C092002081
:10E5D0002780000042487084B18C5520090A090246
:10E5E0000143B184002038817881A88EC006C00F15
:10E5F000C00038800098807F81000143F182217B38
:10E600000398C907C90F00022022104308437082F3
:10E6100001982146334BFF30143106225930C0187F
:10E62000314B98476178FA88E0239A4349010A43BD
:10E63000FA80029868600020A8602846FDF7A7FECF
:10E64000002808D106AB07CBFFF767FE0099002032
:10E6500008776868A8620024204609B0F0BD10B5AC
:10E6600003460C20EFF3108472B69A001F498958B4
:10E6700000291ED02031087F002802D0012817D1A0
:10E6800005E0002201211846FFF782FD10E0CA7E56
:10E6900070235A43164B0120D218108005231B0704
:10E6A0001868012252069043104318600220087730
:10E6B000002084F3108810BD70B5EFF3108472B69B
:10E6C00085000A4B5B593C25ED5C002D04D02031C0
:10E6D0005A5484F3108870BD0123FFF78BFDF8E7CF
:10E6E0005555000000800020190F0000A092002066
:10E6F0008081002070B5FF4C00252068006800284C
:10E7000028D0014620310A7E002A02D0012A21D1D8
:10E710000FE00021FDF734FFFEF7B8F9206800682C
:10E7200004F084FF20680560017A490849000172FD
:10E7300010E0087D70235843EF4B0122C01802807F
:10E7400005200007026801231B069A431A43026052
:10E75000022008762068007A00280FD10223FF22C9
:10E760000021E64804F0C8FF2168497A417005702D
:10E7700004F0DBFF206804F059FF256070BDF7B599
:10E780008100DC4882B005686C5826462036307D12
:10E79000009005F0DBF903990746401A00010009D3
:10E7A000401C216A4008814201D9091A12E0FEF793
:10E7B0006DF9D3480068411C01D0606007E0A18D6D
:10E7C000E08D081A4000C119CE4801406160002068
:10E7D000A060E18D21620846CB494843C849898839
:10E7E000884200D308462061C6496868491C8842AF
:10E7F0000BD86168081A000101210009C906884286
:10E8000003D2FFF777FF05B0F0BD0498002803D1CD
:10E810000521A17561686162BC49A182F17D012079
:10E8200000038A0010430843009B70214B43B24908
:10E83000403959180F46C882AF49208C59180880B2
:10E84000B07D0B2801D00A2801D1B1480881B14A16
:10E85000206A904200D310460122D2030243FA8577
:10E860000020C884287C800708D52946AA48FF33A1
:10E870000A31062259331818A84B9847287CA97CDE
:10E8800082076B7CD20F002901D1800701D50120BE
:10E8900000E000201B0209010B43910000250B43FF
:10E8A0000343FB84B17D3A8A520952010A433A82FA
:10E8B0002046FDF76CFD0028A5D175776586A2E797
:10E8C00038B500280CD004462034227D0C2100915C
:10E8D000A37E9349FDF782FEFEF7D8F8012020764B
:10E8E00038BD10B5040014D03820005D002810D1C8
:10E8F00005F02CF9616A411A0A01A18D120949003B
:10E900008A4203D3A17D491CA17560622046FDF7B0
:10E910003EFD10BD70B577490C200968002920D054
:10E920000D68002D1CD03820405D002818D105F05E
:10E930000DF969680446081B000101220009D2068E
:10E94000904203D9601A0001000940423C2807DDCB
:10E9500000212846FDF714FE28466C60FDF717FDE0
:10E96000002070BDF1B5634D0C24286886B00028E6
:10E9700076D10021142004F0FFFD286000286FD01C
:10E98000044605F0E3F804900020039006981C214B
:10E9900048436449614F40180090142200210669E1
:10E9A0005C372868B847B078C00733D000216420AE
:10E9B00004F0E2FD206000282CD0642205460021EE
:10E9C000B8475948E8615948A8610320E87505200F
:10E9D000A87530894C49484349498988884200D301
:10E9E00008464A492861A982F088A8853289EA85C3
:10E9F00028463179203000234175C3752A62837619
:10EA0000069A027501290BD000200390207A01217B
:10EA1000084320723078C007424803D0763002E0C5
:10EA20000120F2E7703001460290062220463B4B5F
:10EA30000A30984730782074707860740698607255
:10EA40000025A5740098808A00280AD038494843D8
:10EA5000491102F0D1FD049940180001000902E0BB
:10EA6000F2E00020C0436060069827688006000E30
:10EA700000010590002F7DD001972037387D0021BF
:10EA80003977092179762B491B4B8A8870214143BC
:10EA9000403BCD188C46EA83264AD2882A84264AEF
:10EAA0006A84AB8C55221B0A1B021343AB84124BA6
:10EAB0000022C9180091CA843178A27C8907637C3E
:10EAC000C90F002A02D1227C920701D5012200E061
:10EAD00000221B0289000B431343EB84174929854D
:10EAE000009A00211181009A51813178C907C90F1C
:10EAF000000225E0B0920020808100200502000085
:10EB0000C0920020FEFFFF0FE20400000160000041
:10EB1000723E0000FF3F000000800020190F00003F
:10EB200015470118CC900020E3E80018C1E8001850
:10EB3000204E000050910020555500002780000015
:10EB4000202210430843688260465B4BFF30062258
:10EB50005930C018594B0299984706206885787D2E
:10EB600001280AD00020A88600998882387F0028D2
:10EB700012D000E039E00A200FE077210598C900A3
:10EB800040188008A88600998882387F002801D024
:10EB90000B2002E0092000E00820B875C0B20B2865
:10EBA00001D00A2802D1009945480881B87D288201
:10EBB000F87D01210903820011430143E982019894
:10EBC0000099008C088001983E49006A884200D371
:10EBD00008460121C9030143E985E88EC009C00147
:10EBE000E886A88D40084000A8850398002818D022
:10EBF000354A059803218018428F120912010A43F1
:10EC0000428700218187418F0322C9B292021143BA
:10EC10004187018F890B89030187018F4904490CC2
:10EC200001872B49294848622068002500280AD01E
:10EC30000499416004464162FDF7A9FB002802D116
:10EC40003D20055565860024204607B0F0BD10B56F
:10EC50000C20EFF3108472B61E490968002902D017
:10EC6000FFF748FD002084F3108810BDF8B519495E
:10EC700005460C680C201646002C1BD0002D0BD02E
:10EC800004F064FF074614481449684302F0B4FCDA
:10EC900038180001000901E00020C0436060002E28
:10ECA00005D006222046054B31460A309847FFF72B
:10ECB00031FE0020F8BD000000800020190F000088
:10ECC000723E0000FF3F0000808300200100010031
:10ECD00000010050B0920020204E000071020000A0
:10ECE00070B5FA4C002520680068002827D001463E
:10ECF00020314A7B002A02D0012A20D10FE00021D6
:10ED0000FDF73EFCFDF7C2FE2068006804F08EFCB3
:10ED100020680560C17C49084900C1740FE0087E85
:10ED200070235843EA4B0122C018028005231B07B9
:10ED30001868120690431043186002204873206838
:10ED4000C17C002912D14068002809D14120042348
:10ED5000FF22C00004F0D0FC2168097D0170C5705D
:10ED600004F0E3FC206804F061FC256070BDF7B599
:10ED70000D46D649800009680C5804F0E7FE0646A7
:10ED8000401B000100092546401C2035216A40082F
:10ED90002F7E814201D9091A09E0FDF777FECD489F
:10EDA0000068411C11D060600020A060618D21626C
:10EDB0000846C9494843C7498988884200D308465C
:10EDC00020610298002808D00BE0218D608D081A80
:10EDD0004000C24980190840E5E70A21A175616831
:10EDE0006162BF49A1820120687570204743B8481D
:10EDF000218C38180180218C0122D2030A43B449A6
:10EE000040397918CA850026C6842046FDF7BFFA26
:10EE1000002800D1AE75FEBDFEB504002DD0AB4874
:10EE2000254620350068297E01916E7D0291018979
:10EE3000408900908F003946606802F0DDFB009841
:10EE4000791A40000818B1000831814200D93818F9
:10EE50000299702251439E4A8008801B403A8918CB
:10EE6000C8870C200090EB7D9E492046019AFDF753
:10EE7000B5FBFDF70BFE01206873FEBD10B5040065
:10EE800014D02D20005D002810D104F05FFE616ACF
:10EE9000411A0A01218D120949008A4203D3A17D3A
:10EEA000491CA17560622046FDF771FA10BDF1B5ED
:10EEB00092B003200990692000010F9004F046FEF3
:10EEC0000E9004F047FB814C070220683F0A00289F
:10EED0007DD10021442004F04FFB2060002876D033
:10EEE00000210D9112991C2251437F4A7F4B8918B2
:10EEF00044220D69044600219847129921756978CA
:10EF0000A176A978E176264629782036F175002188
:10EF10003176402001556878C007734801D07630BB
:10EF200000E07030014608902046704B06222630E3
:10EF30005C3B984720466D4B0622E91C2C305C3B1D
:10EF40009847BF2060759F20A0750320E075CD20F5
:10EF500020761F20607620461C3012990690FCF720
:10EF600088F837802220390C01550220F07038468D
:10EF70000C2102F041FB4F1D5D4837710089F5F708
:10EF800025FA7071594B042268465C3B06999847F4
:10EF9000564B032231465C3B01A89847F0786946FE
:10EFA000C871002008812146504B052215315C3B79
:10EFB00004A8984770796946400138434875274648
:10EFC000687A0837C00748D000213C2000E028E1DB
:10EFD00004F0D2FA206000283FD03C22434B069038
:10EFE00000210790984707984249C1610798424914
:10EFF000816107980421C17507980A2181750798D6
:10F0000000218160A889344A5043324A9288904254
:10F0100000D31046079A10610798314A82820698F9
:10F020006A8902850698AA8942850698203001736C
:10F03000069B1A62C1757F22027501234375129ADD
:10F040000276688B3880A88B7880688AB880A88A16
:10F05000F8803972E07C1843E0743888694648814A
:10F06000B8888881F888214BC881162223485C3BE8
:10F0700098470120A07468780021B174129A800723
:10F080009206120E21681201C00F0C9200297DD049
:10F09000069120311091097E70230B9159430C4B3E
:10F0A0000622403BCF180A917A85094B2289C9185C
:10F0B00007914A8077230C9ADB00D2189208BA860F
:10F0C0008A82A17C00291BD00F211AE0B492002073
:10F0D00080810020C0920020E2040000FCFFFF0FAE
:10F0E00001600000514A0118CC900020750F00000B
:10F0F000509100207DEE001819EE00189086002037
:10F100000E2100233982504A9188F983D1883984AD
:10F110004E497984BA8C5521120A12020A43BA84E4
:10F120000799CB842978B27C090280000143500002
:10F130000143F984B07C002802D007990D9888819A
:10F14000287800280ED1B07C00280BD10A98404BBB
:10F15000FF30E91C06228D30C0183E4B98470799B6
:10F16000A87848820126F6033B4900203985079993
:10F1700008810799488169780B98C907C90F00026F
:10F180002022104308437882062200E017E00A9804
:10F190002F4BFF305930C0182E4B089998471098C4
:10F1A000B110007B820011430143F9820698079950
:10F1B000008C088006983146008C0143F985274A67
:10F1C0000C9805218018428F120912010A434287C8
:10F1D0000F998187418F1122C9B252021143418791
:10F1E000018F890B89030187A9781D4BCA07120E6D
:10F1F000052100251A430A434287018F4904490C1F
:10F2000001876560206800280BD00E994160044694
:10F210004162FDF7BCF8002801D12034A57500201B
:10F220000990099813B0F0BD10B50C20EFF31084CD
:10F2300072B60C490968002902D0FFF751FD002081
:10F2400084F3108810BD0000509100205555000037
:10F2500000800020190F000027800000808300201C
:10F2600020220000B49200201CB541480468002C04
:10F270001ED0684604F075FC01980099E02801D37F
:10F28000012000E00020401C081800010009009047
:10F2900060680099401A000101210009C9068842EE
:10F2A00001D2606801E00098606004F069FB1CBD59
:10F2B0000020C043F9E7FEB506460025EFF31087AE
:10F2C00072B6684604F04DFC019800997C2801D381
:10F2D000012000E00020401C0818000100090090F7
:10F2E00070680099401A010101200909C006814295
:10F2F00001D3009971601E490C6808E0616872686A
:10F30000891A09010909814203D325462468002C82
:10F31000F4D1002D05D032462946154804F094F862
:10F3200005E03146124804F017F8FFF79DFF87F318
:10F330001088FEBD70B50025EFF3108472B60C4E38
:10F340003168814208D1304604F00DF83068002859
:10F3500009D0FFF789FF06E00146054804F00DF8E3
:10F36000002800D1022584F31088284670BD0000D3
:10F37000B8920020F8B51F4614460D46104604F01A
:10F3800022FA0026240A3F280DD0574A2946A00019
:10F390000C39105803F0CAFF012631462046FEF70B
:10F3A0002FFA3046F8BD462239462046F7F72DFFA2
:10F3B000F7E770B54D4D6C88F7F72BFDFF2808D0A7
:10F3C0006988491C6980810047484058017B491E73
:10F3D0000173002C02D1062004F09EFA70BDF0B536
:10F3E00087B014460E46104604F0EDF93F284CD085
:10F3F000200A05903C4980000D5800200490708838
:10F400006946888130883A49401804903779012F3D
:10F4100004D0022F39D10598FEF79DFA287C697C2B
:10F42000884205D203AA04A90598FEF7BAFA022772
:10F43000A968002929D088882E4AD04225D10C46B7
:10F440006846808904990C3400912B4601900E3354
:10F45000A21C0297211D0598FEF736FA070002D17B
:10F46000E889002811D10020A8602770204604F008
:10F470005CF9E088042808D100206080002F04D1C6
:10F48000207A522807D01B2805D0308803F0AAFE26
:10F49000002007B0F0BD30886080F9E770B51446F1
:10F4A0000D46104604F08FF90146200A00243F293A
:10F4B00011D0EA88291D052A0DD12A78002A0CD0FE
:10F4C000332A08D04979312A0BD0002903D00023F0
:10F4D0001A46F7F7D3FF204670BDF8F722F8044626
:10F4E000F9E717230122F4E7C09000208C92002056
:10F4F00000800020F9FBFFFFF8B50020009008789D
:10F500001D460C46012807D003280BD0402219467F
:10F51000F7F7BFFA0098F8BD05F0D0FE00222946A3
:10F520000120F5E70020F7F7C1FA00900128F1D19A
:10F530006078002507073F0FF7F737FB002808D151
:10F5400029484068002804D10321FDF715FE002852
:10F5500001D0432543E00020002801D042253EE0B1
:10F56000608C1B38E12807D2A08CFF2149318842EA
:10F5700002D31E49884201D9402530E0E17E1A4E6F
:10F58000C9073801490F084320363071B8080DD03B
:10F59000E08C012217215202904200D31046172816
:10F5A00000D2084610498883F6F7A3FD3079A17E82
:10F5B00080088000084330710B480622211D0C4B47
:10F5C0001E309847201D01F06AFA20462030017A4B
:10F5D000407A01F021FAA18C608C01F02EFA2946C4
:10F5E0000020F7F781FA95E76490002048080000B2
:10F5F000190F000070B50C46062004F0E4F804284A
:10F600001BD061480068002817D00178192914D14F
:10F610000C380189C320002510230622C00004F005
:10F620006BF85A4B0646102221469847304604F0A4
:10F630007CF829460020F7F757FA70BDF7B5044665
:10F6400086B01546062004F0BEF804282BD04E4F95
:10F650003968002927D00878182824D1002C02D036
:10F660009034E1B21CE02846484D01260C460028A3
:10F670001BD00F460C39C120098908230622C0007F
:10F6800004F03AF804460322791CC01CA847032260
:10F6900020460799A847A671204604F046F80021A5
:10F6A0000020F7F721FA09B0F0BD0322601C07998A
:10F6B000A847E07821798006800E0843334BE0703C
:10F6C0001022002101A85C3398470322611C01A885
:10F6D000A847B8692E4B012201A90096F7F7D8F880
:10F6E000E1E770B50C46062004F06DF804281AD046
:10F6F00025480068002816D001781A2913D10C3843
:10F700000189002508230622224803F0F5FF1F4B3C
:10F710000646082221469847304604F006F8294656
:10F720000020F7F7E1F970BD38B50C460020F7F777
:10F73000BDF90546012821D12078182804D01928C0
:10F7400013D01A281AD11BE02079C02808D000282D
:10F7500006D0402804D040210020F7F7C5F90DE07D
:10F7600000210B48F7F7C5F808E000210091214679
:10F77000094B01221131601CF7F78AF8284638BD81
:10F7800000210648EEE7000064900020190F0000F9
:10F790003DF600181A060000F5F50018E3F600180B
:10F7A0001CB5027B6B461A70002906D001225A70E4
:10F7B0004A885A800979197101E000215970E44C96
:10F7C0004482184601F064FA0146684640780843CE
:10F7D00002D02046FDF71FFE1CBD70B50446012572
:10F7E0000878002A11D0A28B4B889A420DD1A92803
:10F7F00002D0AA2803D006E0207C042101E0207C6E
:10F80000082108432074002509E0A92801D0AA286E
:10F8100005D1204600F064F9A18B4018A08328464A
:10F8200070BD10B50024C477CA4A037B5371FFF73B
:10F83000B7FF204610BD0021C177C649027B4A713F
:10F84000017C490601D50021AAE7704710B50021C7
:10F85000C177C049BE4C027B4A71E41C4482007BE4
:10F8600001F07FFA01462046FDF7D5FD10BDFFB53A
:10F870000F4658881021084381B058801C46164610
:10F88000002520210198FDF761FC00282FD00021E0
:10F8900041732278827347748682C1776178817759
:10F8A000AD490160AD494160AD498160A94A019906
:10F8B0005171817B0029A1781BD0890706D4017C76
:10F8C000022211430174A178890703D5017C01222A
:10F8D00011430174A178C90703D0017C2022114390
:10F8E0000174214600F0BCF8284605B0F0BD4B2558
:10F8F000FAE74907E3D5E6E770B50C460120F7F7CC
:10F90000D5F8054601280ED160789249800020394B
:10F9100040188068002181838E4962784A710022F4
:10F920002146FFF75AFF284670BDF8B5C77B894DC1
:10F93000874C203DBF263B0001F036FF0604101D1A
:10F940001037420F824BDB1C994200D0C277418AAC
:10F95000002902D1C17FFDF72CFCF8BD69681400B5
:10F9600004D10122FFF739FF0028F6D121460120FA
:10F97000F7F7BAF8F8BDA14205D1C37F002B02D03A
:10F98000017C314009E0C277002A07D1704A524217
:10F99000D14203D1017C402211430174418A0029E4
:10F9A000E8D1C17FFDF73AFCF8BDA14202D1017C4C
:10F9B00031400174418A0029F6D1FDF73FFCF8BDC2
:10F9C000FDF76DFCF8BDF7B50E46624905468000AF
:10F9D000203940188068002814D0C17B032911D138
:10F9E000818AD52008230622C00003F085FE057019
:10F9F0000446C67106225B4B02A9401C984720466C
:10FA000003F093FEFEBD70B5524B8000203BC01842
:10FA100084680025002C22D0607B00281FD1E07B69
:10FA200003281CD1207CBF2318402074002904D057
:10FA30003C290FD043290ED10CE0607C00280AD06D
:10FA40001046F7F7E6F9FF2805D021461631F7F7FB
:10FA50000DFA00E0452529462046FDF7EFFB70BD75
:10FA6000F8B50D4606460021202003F085FD04462A
:10FA7000307B2070A8784006400E60802869606066
:10FA80006869A060287E6070687E2077707CFDF7D2
:10FA900086FB2073A878400707D5287B6073062271
:10FAA000A91D20462F4B0E3098476879A0762879FB
:10FAB000E0766888C00501D5012000E00020244FD1
:10FAC0006077FF1E7782204601F03EF8050002D0E5
:10FAD000204603F0ABFD29463846FDF79CFCF8BDF7
:10FAE0007CB50A4653880146FB2B01D8032007E06A
:10FAF000888B002806D0181A83B2FB2B04D802206A
:10FB0000DCB203E0012000E00020FB240B7B6D460B
:10FB10002B706870EC708B8B101D1818019010788A
:10FB2000A9280ED001202A46A870094D6D1E4D82CD
:10FB3000104601F04AF801462846FDF76CFC2046C5
:10FB40007CBD00202A46A870014DAD1EEFE70000E5
:10FB5000392000008490002023F8001837F800189E
:10FB60004DF80018190F00007CB50C46B1496B46E2
:10FB700049681C700A795A70827B012300259B0218
:10FB8000891C012A12D0002A10D08A896B465A801B
:10FB9000C9899980A84D4582684601F0AEF90146B1
:10FBA0000C4302D02846FDF736FC7CBD69464B80ED
:10FBB0008D80EFE710B58A788273CA780024891C9B
:10FBC000920603D4027C01231A430274994A037BF0
:10FBD00020325371037BD37100F0EDF8204610BD45
:10FBE0009449027B20314A710021BDE770B504467B
:10FBF00090481646203000790D46C00601D44324B3
:10FC000018E00846FDF768FA002815D01C212046A8
:10FC1000FDF79CFA002811D00121417345748682BA
:10FC200086490160864941608649002481602146F9
:10FC3000FDF7BFFA204670BD4024FBE74B24F9E7EF
:10FC400070B57C4BC57B04242033022D06D0042DD7
:10FC500003D1DC710021FDF7F1FA70BD002A04D058
:10FC6000DC711146FDF7DAFA70BD734A521E9142FB
:10FC700003D10121FFF778FF70BD6F4A9142FBD19C
:10FC80000021EFE7F8B505466A482030C07904281E
:10FC90007AD06849800040188768B87B042802D36E
:10FCA000687DC00770D0687D00214006800F0091FC
:10FCB000002802D0022803D005E00120009002E0D5
:10FCC000387CC00760D06E7FB98A3346163306226F
:10FCD0005D4803F011FD0446002E0BD0A682298C4E
:10FCE000AA7F20468918594B163089B2C918584B3B
:10FCF00032469847687D010747D5C00601D50320E5
:10FD000000E002206070687DC00703D06078102199
:10FD100008436070687D800703D560782021084320
:10FD20006070687D400703D56078402108436070AB
:10FD30000098002803D06078082108436070387B61
:10FD40002070287F6074E87E2074687E401CA07458
:10FD5000E87DFF281CD0C007C00F20720622291D95
:10FD60003B4BA01C9847687D40070AD5287E294652
:10FD7000C007C00FE07306220A312046344B093019
:10FD80009847204603F0D1FCF8BDC006C00FB9E784
:10FD9000FF202072E7E7274910B52031C8790428F1
:10FDA00008D0244A8000801880680422CA71452146
:10FDB000FDF744FA10BDF8B50D4606460021442073
:10FDC00003F0DAFB044600274030C7708770707C70
:10FDD000FDF7E5F920706770B07B0121032801D0A1
:10FDE000052800D16170707C012806D16878C006B2
:10FDF00003D56078022210436070A7706878C0074E
:10FE000008D0A170A888E080E88820816878400741
:10FE1000C00F2071084F20467F1E778201F032F814
:10FE2000050002D0204603F001FC29463846FDF7C4
:10FE3000F2FAF8BD6490002042200000B5FB0018E3
:10FE4000E1FB00189FD20018A706000000800020E8
:10FE5000190F000070B504468878A073002654205E
:10FE600006558A888D1C002A05D00A2042430621A7
:10FE7000764803F0C1FC7648217B4171217B81717A
:10FE80002946204600F0A3F8304670BD70B5044600
:10FE900006216E4803F003FD6D48217B41716D4DD5
:10FEA000658201F06FFA010002D02846FDF7B3FA2F
:10FEB00070BDF8B5074666480D4600790024010973
:10FEC00005201646884301D0432417E02846FDF755
:10FED00003F9002814D058213846FDF737F90028D7
:10FEE00010D002214173457486825B4901605B49F1
:10FEF00041605B4981600021FDF75BF92046F8BD58
:10FF00004024FBE74B24F9E770B5514E0025B17949
:10FF100032468900203A89188C68FF280DD0617C10
:10FF2000002903D021461631F6F7A0FFA07B002858
:10FF30000AD10621454803F0B2FC042201252046DF
:10FF40000021B271FDF77AF9284670BD70B54048BE
:10FF50008479042C13D03E49A000203940188568CC
:10FF60000622352002231146400103F0C5FBA521DE
:10FF70000170447003F0D9FB4520403528750020FE
:10FF800070BDF8B50746C17B04263048304C0229C5
:10FF900007D0032910D004290DD154213846C95D5A
:10FFA00011E0150003D0062103F079FCA671294663
:10FFB0003846FDF733F9F8BD1500FCD0062103F0F3
:10FFC0006EFC38462946A671FDF738F9F8BDF8B53C
:10FFD0000D46064600211E2003F0CEFA0446707C32
:10FFE000FDF7DDF86070002020703620405D294666
:10FFF000A070062230311B4BE01C98476878C00780
:020000041801E1
:10000000C00F60726878C0070FD0A8886081E88848
:10001000A081A889E081E8892082A88AE082E88A14
:100020002083288A6082688AA0820A4F204635375A
:10003000778201F025F9050002D0204603F0F6FA98
:1000400029463846FDF7E7F9F8BD0000F206000042
:10005000849000200E20000055FE00188DFE001830
:100060009FD20018190F000010B501221E21F7F7CA
:10007000CAF9083803F059FB10BD10B50C4601024F
:100080001520F74A8001491D03F0B6FB20460838C9
:1000900003F04BFB10BDFEB501468000F14B029012
:1000A0001A589468002C64D050680190E28900923C
:1000B000921D0C3893B200890A02264601460C367E
:1000C0000027E948521D03F017FB009A054682807D
:1000D0000198818829800198C1886980307A09282F
:1000E00019D137460837727AA81D391DDF4B921E89
:1000F00098477878811E8FB22168002903D06988DB
:10010000081A801C6880304624680C3803F08EFA88
:1001100026460C3622E008360196403EB08F401E3F
:1001200086B2009887420AD2C01B3246864200D36C
:100130000246E8190199CD4B801D491C9847B81912
:1001400087B22068002802D06888801B68802468F5
:10015000019826460C36143803F068FA002CDAD1E0
:10016000C0490298085800218160C160284603F008
:10017000DCFAFEBD10B50446BD484988828B8A4230
:1001800000D211462046F6F7F5FFB648A1004058C8
:100190004068002802D00078012801D0412200E008
:1001A000002201212046F6F774FF002010BDF3B5B0
:1001B00083B00398AB4A8000019010584068002833
:1001C00002D00178072901D040223AE0009004983B
:1001D0004078012809D01027049800254038808FE6
:1001E0002E46801E80B2029024E00227F4E79D494B
:1001F00001983B1D085840680C3801890398020299
:100200009948521D801E03F077FA04460498974BD4
:10021000401946882680A770AD1C0498ADB24119DC
:10022000E01C3A46891C9847E81985B2204603F03D
:100230007CFA02988542DAD30098C088B04205D88B
:10024000002201210398F6F724FF0FE00098761CA6
:100250008680009801214088C9030843009948809E
:10026000804901980858406803F05FFA002005B003
:10027000F0BDF3B583B003987A4980000090085828
:100280004468002C02D02078032801D040223AE0B4
:10029000049878494038808F0026C0034018000C2D
:1002A0003746019029E06F490098637808589B1DF4
:1002B00040680C380189039802026B48521D401FA8
:1002C00003F01AFA054671000498761C0818B1B2BA
:1002D0004A00408828800498491C101847886F807D
:1002E0008EB26078287121460831604B6278681DB3
:1002F0009847284603F019FA01988642D3D3E0883C
:10030000B84205D8002201210398F6F7C2FE0CE09E
:100310007F1CA78060880121C90308436080514980
:1003200000980858406803F000FA00209FE7F3B5F2
:1003300089B000250846019540380595808F0C4608
:10034000801E80B204900999464E8F00F1592846CC
:100350004968002900D00878099A120203920428FB
:100360006ED0052805D0062803D00A2872D0402276
:10037000D6E000916078072801D9102000E0022023
:1003800002900520079048E06019C1788278080241
:100390001043069001900098007805280CD0009832
:1003A000009A43780798083228180019801C02998F
:1003B000F7F796F900282DD02A48039AC059029BD6
:1003C0004068521D0C38018927489B1DC01E03F050
:1003D00093F9064606983080AD1CA8B2211889789A
:1003E000401C317180B22118CA788B7811021943F0
:1003F000801C718085B2029870716119B01D1B4B11
:10040000891C029A98470298281885B2304603F052
:100410008CF902E06078401985B204988542B3D324
:100420000098C1880198814279D90099401C888040
:10043000009801214088C90308430099488077E06B
:1004400000200646029004980691400703D0102031
:10045000009040E073E0012002900220F8E70000E5
:1004600030750000B490002009050000190F00004D
:10047000649000200000FFFFF748039AC059009BDA
:100480004068521D0C380189F448083303F034F9F0
:100490000646601941883180AD1CA9B260184288B7
:1004A000891C89B2601872804288B280891C0298C7
:1004B0008DB2002816D00098B0716119F01DE84B7C
:1004C000891C009A98470098281885B230880190B6
:1004D000304603F02AF904988542CDD302980028CB
:1004E00007D017E0DC483146C0590C39083002F01B
:1004F0001DFF002E0ED004220A210998F6F783FF73
:100500000146708848800998FFF7B7FD00200BB0BE
:10051000F0BD04E00698C1880198814205D8002208
:1005200001210998F6F7B5FD07E00699401C88807F
:10053000C948C059406803F0F8F80598E7E70998FA
:10054000F6F713FE6378801E98421BDDF059039A7C
:100550004068521D0C380189C0481B1D001D03F066
:10056000CBF80546608828806078211D801E82B205
:10057000AA8000206880BA4BA81D9847284603F03F
:10058000D4F8CCE7F05962884068214682806278CE
:100590000839921EC280002202816078801E488045
:1005A000F0590C39083002F0C1FE01200590F059D5
:1005B000C0E7F3B508464038808F85B0801E80B212
:1005C00004904C780F46214601F016F80599A24A8E
:1005D0008900039151584D68002D69D0297802296E
:1005E00066D1002864D000260196142C01D0022088
:1005F00000E0102000900020029032E0964903981D
:10060000009B08589B1D40680C3801890598020220
:100610009248521D401E03F06FF80446B8194088F6
:10062000B61C2080B1B2781842886280019200988E
:10063000891C20718EB2B919601D894B891C009AE2
:10064000984700992A46701886B26B780832601D68
:10065000F7F746F8002801D001200290204603F069
:1006600064F804988642029806D200280AD17D498F
:1006700001988842C2D101E0002803D1E98801989D
:10068000814205D8002201210598F6F702FD0CE011
:10069000401CA88068880121C903084368806E490E
:1006A00003980858406803F040F8002007B02FE78F
:1006B0004122E8E7F3B581B0002000900198664A36
:1006C000860090590F4645680021002D00D02978FA
:1006D000042907D008291FD009291DD00A291BD0B9
:1006E00041223AE0083002F03EFE04460C3410226B
:1006F000791C5B4B133098471020A071204603F003
:1007000014F82088E988814201D8002225E0401CA5
:10071000A880514880593CE03946403FBA8F4E4846
:10072000521E94B2083900224A8080590C39083090
:1007300002F0FCFD2889002802D0844200D3044640
:10074000454FB8598068C189091989B2C181012012
:1007500000904002814205D9112201210198F6F74B
:1007600098FC19E00198F6F700FD401EA04204DC59
:100770002889A04205D8002803D00198FFF78BFCF8
:10078000C3E7E9880919E980002801D0001B288106
:10079000B859406802F0C9FF0098FEBDF3B585B0B6
:1007A00005982D4A8000039010584068002802D018
:1007B00001780B2901D0412247E006994039898F01
:1007C0000190491E002589B22E460095029132E023
:1007D00021490398B200085840680C3801890198F3
:1007E0001718F888801D83B2059802021B48521D15
:1007F000001D02F081FFB988044601800298F98843
:10080000401B814200D2084682B2A2800020608054
:100810000698134B4119A01D491C9847A0884119FF
:100820008DB2F988884201D050200090204602F015
:100830007CFF761CF6B201984078B042C8D8029886
:10084000854201D050200090009A01210598F6F7CA
:1008500020FC00202AE70000B490002005050000DD
:10086000190F0000FFFF000010B56649820089588B
:100870004968002902D009780C2901D0412200E002
:1008800000220121F6F705FC002010BDF8B55D4FF0
:100890000B468600B9594C68002C02D021780C29EF
:1008A00005D041220121F6F7F4FB0020F8BD1846DF
:1008B0004038808FE188801F85B298882A46401A88
:1008C00080B221460C3160814118981D4E4B9847EB
:1008D000002804D1608921894019884201D900206B
:1008E000C0436081B859406802F01FFFDDE710B5D2
:1008F00044498300C95800224968002900D00A7879
:100900000C2A03D00F2A0BD0412204E04A8909891E
:100910008A4205D052220121F6F7BBFB002010BD10
:100920000022F8E770B50D464039898F374A091F14
:100930008EB281005158B21D93B202022878C98943
:10094000521D1B2816D0324802F0D6FE04462878E5
:100950001B2812D01320207066806888A0802A4B44
:10096000291DA01D32468A3B9847204602F0DDFE35
:10097000002070BD2648401EE6E71220EBE770B568
:10098000044608790D46122809D12049A0000858CC
:100990002202C1891E48521D163002F0D7FE2A7964
:1009A00001212046F6F775FB002070BDF8B507461B
:1009B000087A0C46FF260025C10707D0002805D07D
:1009C0001D2803D84008134980000D58608800286E
:1009D00003D002F007FC00206080002D0FD0207AA9
:1009E0001D2807D01B2805D0390215208001491D7C
:1009F00002F055FF214608313846A84706463046E2
:100A0000F8BD0000B4900020A30F00008C900020DF
:100A10000D050000145B0118032283079B0F02D011
:100A200083079B0F00E01346244843708B079B0FFE
:100A300001D08A07920F0270704702461B3AE02AE3
:100A40000AD8FF224932904206D31D4A904203D869
:100A50001A4A403A9087D187704770B50146174DC2
:100A60000C240020803D1C2242435219937B072B0B
:100A700003D116693678F6070FD1052B03D1126919
:100A80005278D20709D1401CC0B20428EBD30B48DE
:100A900006220C4B0A3898470024204670BD70B5DA
:100AA0000546014605480622064C0A38A047034879
:100AB000062229461038A04770BD00004C91002046
:100AC00090420000190F000010B50346E94C0020C9
:100AD0001C21414309198A7B521E022A03D8096945
:100AE0000978994204D0401CC0B20428F0D3FF20FA
:100AF00010BDF3B581B04227FFF7E6FF0446042896
:100B000020D21C20DB4960434618356900270622A5
:100B1000D94B2846143002999847B07B022811D14E
:100B2000EFF3108672B6287BC00709D070204443CB
:100B3000D248FF3406225934CF4B201802999847E7
:100B400086F310883846FEBDF8B504460C260078BA
:100B5000FFF7BAFF6946C74D0870FF2806D01C2171
:100B600048434019807B01282DD104E00846F7F75F
:100B70005AFF060027D1684600781C2148434019D7
:100B80000069002801D002F051FD684600781C2160
:100B900048434119FF200C610876217B002903D0CE
:100BA000012908D0022906D1B24906227031204617
:100BB000B14B14309847684600781C2250430121FD
:100BC0004019817300263046F8BDFEB50546422027
:100BD00000902878FFF778FF0746FF2850D00720BD
:100BE00000901C20A349784340180190A978002662
:100BF00049004418607D143400280DD002F074FBC5
:100C000006464088E9784018402805D9607802F007
:100C100070FB0020607033E06878032801D0012861
:100C20000CD16078002801D002F063FB02F044FB95
:100C30006070002824D002F057FB06463088728886
:100C40008E4B801880B2C0188B4BEA786968984741
:100C50007088E978401870806878032801D00228ED
:100C60000CD10198807B02280CD02078002801D07C
:100C700002F03FFB60782070002060700020009040
:100C80000098FEBD6278A9783846FDF715FDF1E7BA
:100C9000F8B5054612260078FFF716FF0746FF282D
:100CA00008D01C203946414372480C18617D002948
:100CB00055D101E0422652E0E17D00294FD169780B
:100CC000002944D0064620694188CA0717D0090781
:100CD000890F07D0417B0E30F7F778FE002801D04E
:100CE0000B263CE000201C2141438919897B002907
:100CF00003D0401CC0B20428F5D304280BD0A07B3D
:100D000002280AD02A79698838462669FDF726FB29
:100D1000002808D022E0072621E02A796988384691
:100D2000FDF7FBFA1AE00220A073B078514DC0071E
:100D300014D06846F7F777FE00280FD16846007890
:100D400020761C22042150434019817306E0384666
:100D5000FDF785FC002801D10320A0730026304652
:100D6000F8BD10B5FFF7B0FEFF2808D01C21414A9E
:100D700041438918897B012903D00C2010BD4220F2
:100D800010BD00F05BF8002010BDF8B50C460978E6
:100D90001C225143374AE0788E18211D3769009193
:100DA000B17B357E032918D000281BD02846009936
:100DB000FCF7C0FE28461C2148432E49401800215C
:100DC000C180009909894900818005210181418103
:100DD0000121C1738581B17317E000212848FCF718
:100DE0001AFB04E060783C2801D0432801D101209F
:100DF000B073B878C00705D01C211E4A0020694393
:100E00008918887360783C2809D1E078002801D0DF
:100E1000002100E03C212846009AFCF735FBE078F1
:100E2000002802D16078002804D0617838782A46FA
:100E3000FEF7E9FDFF2030760020F8BDF8B500246C
:100E40000C491C225043274645182E19307D002896
:100E500002D002F04EFA3775641CE4B2042CF4D3CD
:100E60002869002802D002F0E1FB2F610020A8735E
:100E7000F8BD0000CC900020190F00000080002079
:100E80003920000038B505460C2300206946F94C8E
:100E9000087009781C2048430019827B062A01D378
:100EA000082A05D9491CC8B2694608700428F0D33D
:100EB00068460078042806D21C2148430019807B2C
:100EC000062818D104E06846F7F7ADFD030012D1FB
:100ED000684600781C21484300190069002801D0A9
:100EE00002F0A4FB684600781C2148430019062143
:100EF000056181730023184638BD70B503460C2583
:100F0000DC4A00201C2141438918897B062901D332
:100F1000082903D9401CC0B20428F3D3197800294A
:100F200004D0012917D01225284670BD0428FBD211
:100F30001C2148438418A07B0728F5D1FDF787FEC4
:100F4000050006D00620A0730021032002F0A7FCB4
:100F5000EAE7082023E00428E6D21C2141438C184C
:100F6000A27B082AE0D0217E5E784908002549004E
:100F7000002E00D0012631432176FD2631405E78D7
:100F8000022E0ED000267600314321765988A182A8
:100F90009988E182072A06D0FDF7E4FC0720A073B8
:100FA000C2E70126EFE720690078800702D5B14A41
:100FB000763200E0002299885888FDF757FEB3E7A3
:100FC00010B5AC4A00201C2141438918897B0729B0
:100FD00004D0401CC0B20428F5D303E0042801D299
:100FE000FDF7C0FC002010BDF0B5487E8FB0401C5E
:100FF000C0B209900C46087D1C2148439D49062239
:10100000401807699C4D002105A8A8470622002129
:101010006846A8470025E07D2E460290FF282BD089
:10102000954B0622211D05A85C3B9847607D400733
:101030002FD56078002810D03878C507E07BED0FF9
:101040008009012801D1022005438A498A4B0622E2
:10105000703168465C3B98470EE02146864B06227D
:101060000A3168465C3B9847257E002D04D0E07B22
:101070008009032800D0FE25607D400709D5684619
:1010800040798009012804D1FE2D02D17878022808
:101090007ED3207D1C21484376494018007EC1073D
:1010A00077D00999012905D08006800F06D0022843
:1010B00003D101E00007F8E701267DE0A27CFF21D3
:1010C0000020002A03D0208A010B0005000D05AA8C
:1010D0000B920A37029A03970C92627D079108924D
:1010E0000290608C049000200D90054620370A90F5
:1010F00036E00E2003996843461831460B9802F0FB
:101100001CFA00282BD0F17A0C98814227D1B17AB1
:101110000898814223D1317B079881421FD10799DA
:101120000020FF2909D00E21039A69438918CA8833
:1011300002998A4201D0F18001200499062909D33D
:101140000E214D43039969180A8904998A4201D0F6
:10115000318130E000282ED101200A902BE06D1C57
:10116000787EA842C5DC0D98002824D1387E0E2157
:1011700048430399404B4518062228465C3B0B998F
:1011800098470898A8720C98E8720798287301E0AD
:1011900039E035E00298E88004982881387E401CC8
:1011A000C0B23876042801D100203876787E042831
:1011B00001D2401C78760A9EA07D012801D0002033
:1011C00004E0002E01D0022000E001200999227DD8
:1011D00001290CD01C214A432649CF2351180A7EED
:1011E0001A40000102430A76002E09D00BE01C21B0
:1011F0004A432049F32351180A7E1A408000F1E740
:101200002046FEF73FFD607F002802D0208C01F0D1
:10121000E9FF00200FB0F0BD10B548781C2148430D
:1012200014494418A07B08280ED0E08A002810D06A
:10123000052109024843A18A0A225143421A00218A
:10124000032002F0D9FA08E000210C48FCF7E3F88B
:1012500001E0FEF7A0FD0620A073A07B062802D0C7
:10126000207E800704D5206900214030C170817044
:10127000002010BDCC900020750F0000422000001F
:10128000F0B5002689B0054668460C240670704B00
:101290002022314601A898476846067068460078C3
:1012A0001C216C4A41438918897B052905D0401CC3
:1012B000C0B2694608700428F0D368460078042854
:1012C0005DD3687A02F0F0F806466846F7F7ABFBA4
:1012D000040054D12EE0142060434119CA89C88A01
:1012E0005200904200D3104682B20220022A00D857
:1012F00002460B8A088B5F00B84200D3384683B29F
:10130000934200D813469C46630101A81818476011
:10131000C98901AF4900F9506346C360002182606A
:101320008174C174694609780182FBF746FB002885
:1013300002D1641CB442CEDBB44201DA3B241EE08D
:10134000684601781C204143424801AB081805213A
:101350000561817300200BE04101C9184A69D2037D
:10136000140C1422424352195483098B9183401C5C
:10137000B042F1DB68460078FDF799FD044620464F
:1013800009B0F0BD70B50024324D0C261C2060431E
:101390004019807B052804D0641CE4B2042CF5D3EA
:1013A0000BE0042C09D2FDF73FFF1C2044436419D5
:1013B000206902F03BF900202061304670BDF8B58D
:1013C0000E781C22234B487872430090D418A27BDD
:1013D000C878052A3AD1091D27690D46002F27D064
:1013E000002822D03046FCF7A5FB698CE1802989D2
:1013F00014224900A180009902235143CA19D18ABD
:101400002046022900D819460181128B8A4200D950
:101410001146418186810421C173FBF796FA2A4661
:1014200000213046FCF730F808E00020A07308E007
:1014300000210948FBF7EFFF0020A0732069002876
:1014400004D0206902F0F2F8002020610020F8BDED
:10145000750F0000CC9000200E20000070B51546DE
:10146000100A0C46214A81005158002911D02279D6
:10147000032A10D0403109788907890F032905D044
:1014800000290CD001223D21F7F7ECFA208801F069
:10149000A9FE002070BD2146FCF721FEF9E7F5F713
:1014A000B8FC01022A462046091D02F056F9012027
:1014B00070BD70B5150AD8B2032804D02846FDF7D0
:1014C00078FF002070BD0949A8000C58002C09D0F5
:1014D0002046203001F047FF02F0A8F8E08F0221FB
:1014E0008843E0872846FCF743FDEAE79092002016
:1014F000F7B50098042682003C4810278458656898
:101500006878884209D103280FD004280CD12046DE
:1015100005221830364B291D9847E08F0121B8432A
:10152000E0870098FCF7E4FBFEBDE08F291D3843FF
:10153000E0876A890098FAF7B3FC0028EDD16E7055
:10154000FEBD00290BD129498300C958127849688A
:10155000002904D00978082901D10521C8E770477E
:10156000F8B50E4607462149800008580025C18F6E
:10157000C90702D14068002801D0242525E0F08861
:101580001C49101A80B2884201D228251DE0390278
:10159000491CFF200C230A46073002F0ADF8044630
:1015A00008202070032060700522711C104B201D44
:1015B0009847F0886081224601213846FCF758FBA5
:1015C000002203213846FFF793FF2846F8BD81002B
:1015D00006484058002806D04021095CC9438907C5
:1015E00001D0183070470020704700009092002012
:1015F000190F0000FF7F000030B50B4601460020A8
:101600002022012409E00D46D5409D4205D31D4608
:101610009540491B2546954040191546521E002D00
:10162000F1DC30BD70B500242546002801DA012424
:101630004042002901DA01254942FFF7DDFFAC42B3
:1016400000D04042002C00D0494270BDF0B51FB41C
:101650000646002082B005464024019100901BE020
:10166000019922460F46304600F042F8049A059B45
:10167000801A994110D310461946224600F028F8E6
:10168000361A8F410197224601200021009F00F069
:101690001FF838184D4100902046641E0028DFDCFA
:1016A000019B00982946324607B0F0BD064C012543
:1016B000064E05E0E36807CC2B430C3C98471034FA
:1016C000B442F7D3F2F7ECFCB05B0118D05B011821
:1016D00010B5202A04DB0146203A9140002010BDBD
:1016E000914020239C1A0346E3401943904010BDCB
:1016F00010B5202A04DB0846203AD040002110BD56
:101700000B46D340D0402024A21A914008431946EA
:1017100010BD0000F0B51A4D6C6BE00716D0A86A3A
:1017200001273843A862002116482B6802888618D2
:10173000521C3371D2B20280491CC9B20829F3D3BA
:10174000A86B3843A863686A38436862E00615D519
:10175000A86A10231843A86207E00A482A6801888B
:101760004418491C2271C9B20180286A0005F4D4CA
:10177000A86B1843A863686A18436862F0BD00004C
:1017800000300240563100200FB410B503A9044BBD
:10179000044A029800F024F810BC08BC04B01847B2
:1017A000E92901189830002030B47446641E257869
:1017B000641CAB4200D21D46635D5B00E31830BC85
:1017C000184702E008C8121F08C1002AFAD1704762
:1017D0007047002001E001C1121F002AFBD17047B1
:1017E000FFB591B00F460546002606E025280AD031
:1017F000149A139990476D1C761C28780028F5D10F
:10180000304615B0F0BD002400940121F34A029443
:1018100000E004436D1C2B780846203B98401042A2
:10182000F7D128782A280ED0022128780246303AAB
:10183000092A15D8009A0A235A43303A80180C43D3
:101840006D1C0090F1E701CF0090002805DA01201F
:1018500040030443009840420090022004436D1C62
:1018600028782E2815D10420044368786D1C2A2876
:101870000AD101CF6D1C02900BE002990A2251435C
:10188000303940186D1C02902878014630390929FA
:10189000F3D928786C2810D006DC4C281AD0682898
:1018A0000ED06A2817D104E0742813D07A2812D1F8
:1018B00010E00120400504430CE00121090501E08E
:1018C000032109050C436978814203D101200005F9
:1018D00024186D1C6D1C287803906E281ED00CDC1B
:1018E000632831D004DC00288AD0582811D1B2E016
:1018F00064287BD069280CD178E073282DD004DCD3
:101900006F2870D0702804D1A7E075286CD0782893
:101910006BD0149A13999047761C62E06002400FD6
:10192000022807D003280AD0042838680AD00660A5
:101930003F1D56E03868F11706604160F8E73868E7
:101940000680F5E70670F3E73878694608740020EA
:10195000487404A80390012003E038680390002035
:10196000C0433F1D61070FD5002101E00199491CCB
:10197000029A0191914213DA8142F7DB019A0399AD
:10198000895C0029F2D10BE0002101E00199491C9A
:1019900001918142FADB019A0399895C0029F5D112
:1019A00001990098139A401A00902146149B00F068
:1019B0003BF901998019461807E0039803990078CC
:1019C000491C0391149A139990470198401E019065
:1019D000401CF2D12146149B139A009800F014F990
:1019E00086196D1C09E741E033E034E00A2000214C
:1019F000049005916002410F022905D001CFC21762
:101A00009446032905D007E0FF1DFF08FF0003CF20
:101A100006E000B2C2179446042902D140B2C117B1
:101A20008C4600226146944506DA0A46002140426F
:101A300091418C462D2102E0210504D52B216A46D7
:101A40001176012103E0E10701D02021F7E70191A0
:101A500054E00A200BE0102009E01020049000213F
:101A60000420044308200591029003E0082000218F
:101A7000059104906002410F022905D001CF002298
:101A80009446032906D006E0FF1DFF08FF0003CFA0
:101A90008C4603E080B2042900D1C0B2002101913C
:101AA00021072BD50399702906D0049A1021059B94
:101AB0004A401A4305D00EE040216A4611760121C2
:101AC00008E06146014306D030216A461176039949
:101AD000517602210191049A0821059B4A401A433C
:101AE0000CD16146014301D1610707D530216A4617
:101AF0001176012101910299491E029103995829F9
:101B000004D037A103910FA90F910DE039A1F9E796
:101B10006146059B049AFFF799FD039B8C469B5CED
:101B20000F9A521E0F92137061460143F0D10F9825
:101B300007A9081A20300390600704D5012000048B
:101B40008443029801E0012002900399884201DD5C
:101B5000401A00E0002041180290019809180098EE
:101B6000401A0090E00306D42146149B139A009873
:101B700000F05AF886190020049008E006A9085CD5
:101B8000149A139990470498401C761C049001996C
:101B90008842F3DBE0030CD52146149B139A00988E
:101BA00000F042F8861904E0149A30201399904707
:101BB000761C0299481E02900029F5DC08E00F9877
:101BC0000F990078491C0F91149A13999047761C2D
:101BD0000399481E03900029F1DCFBE60928010067
:101BE0003031323334353637383961626364656693
:101BF0000000000030313233343536373839414255
:101C00004344454600000000F8B5044600251E4642
:101C10001746880404D405E039462020B0476D1CDF
:101C2000641EF9D52846F8BDFFB50446002581B0ED
:101C30001E46C80301D5302700E02027880404D5BC
:101C400005E038460399B0476D1C641EF9D5284657
:101C500005B0F0BD10B5A02803D0A92801D0AA284E
:101C600001D100F07DF810BD10B50222044B002117
:101C700002489847002000F021F810BD5A32002099
:101C8000750F0000002801D1014801707047000065
:101C90005A32002010B5144600280CD11146A52058
:101CA00000F05EF8452C06D103480078022802D1E6
:101CB000012000F0ADFD10BD62320020F8B51C4FD0
:101CC0000246002404250126797838781300FFF7AE
:101CD0006BFD0504070F151D0600002920D0F8BD77
:101CE0000229FCD1002100F05FFF03207870F8BDCD
:101CF0000329FCD100F061FF7D70F8BD0029FCD004
:101D00000329FAD000F0BCFE7C70F8BD03290BD08B
:101D1000002905D0032903D0387800F0B1FE7C708B
:101D200000F008F87E70F8BD00F047FF7D70F3E723
:101D30005A32002000B589B000206B46187001218E
:101D4000597003225A80587159760720187620203E
:101D5000049005906946002000F078FE09B000BDAF
:101D600030B50221204C89B0A0280ED0A52834D04F
:101D7000A92820D0AA2806D161700120FFF79EFF74
:101D8000022000F045FD09B030BD6B4619700120FE
:101D90005870062098700320D8701871002159716E
:101DA000FF259D71D87119201872597299720B22F2
:101DB0002078A9210EE000A91420023100F0F0FCE7
:101DC000411C6A461170092151702478821C6B46AF
:101DD000AA21204600F076FED5E76078032801D0DE
:101DE0000428D0D16170CEE75A32002010B5002807
:101DF00007D0012000F00CFD00F0FCFCFFF734FFE1
:101E000010BD0222054B00210348984704490022D7
:101E1000881D00F075FE10BD62320020750F0000B5
:101E2000AC58011810B50C46022808D0032810D071
:101E3000042803D10021204600F0B1FC10BD084861
:101E40004470032000F0E4FC0021204600F0E4FD93
:101E500010BD022000F0DCFC0120FFF72FFF10BDB9
:101E6000623200200020704738B51D0A0C460B78FE
:101E7000D62234A136A0FFF787FC2078801E03000D
:101E8000FFF792FC070513122312481A1200E0789C
:101E90000090A378DC222BA134A0FFF775FC22462A
:101EA00029460420FFF7BEFF38BDA378E32225A111
:101EB00039A0FFF769FC38BDE92222A140A0FFF755
:101EC00063FC284600F0BCFD38BDEF221DA143A0F5
:101ED000FFF75AFCF0221BA147A0FFF755FC002595
:101EE0006019817846A0FFF74FFC6D1C102DF7DBC1
:101EF0001DA0FFF749FCF12212A13FA0FFF744FC0F
:101F000000256019817C3EA0FFF73EFC6D1C062D6C
:101F1000F7DB13E0237FF8220AA13BA0FFF734FC94
:101F2000F92208A134A0FFF72FFC00256019817861
:101F300033A0FFF729FC6D1C1C2DF7D30AA0FFF777
:101F400023FC38BD6170705F676170632E630000B1
:101F50003C25732C25643E626F6E645F696E642855
:101F6000696E666F3A2564290D0A00003C25732CC2
:101F700025643E50414952494E475F5355434345BE
:101F8000454428617574683A25582C6C746B3A2561
:101F900064290D0A000000003C25732C25643E5086
:101FA000414952494E475F4641494C454428726574
:101FB00061736F6E3A30782558290D0A00000000D1
:101FC0003C25732C25643E52455045415445445FA1
:101FD000415454454D50540D0A0000003C25732CCB
:101FE00025643E49524B5F455843482869726B2C23
:101FF00061646472290D0A003C25732C25643E003F
:1020000025303258200000003C25732C25643E42C8
:102010006F6E64204C544B5F455843482873697A6F
:10202000653A2564290D0A0070B51E0A0C460B7826
:1020300088B06F2248A14BA0FFF7A6FB2078514D36
:102040000300FFF7B1FB080540404046427A2140BB
:10205000684600F0C3FB69463046F3F712FC63782C
:102060007B223DA148A0FFF78FFB7C223AA14EA026
:10207000FFF78AFB00246D46295D4DA0FFF784FB26
:10208000641C072CF8D31BE06946304600F086FB41
:1020900069463046F3F782FB637887222EA146A07B
:1020A000FFF772FB88222CA13FA0FFF76DFB0024F5
:1020B0006D46295D3EA0FFF767FB641C1C2CF8D31E
:1020C00043A0FFF761FB08B070BD8D2222A141A0A3
:1020D0000DE06378992220A143A0FFF755FB6078BB
:1020E000002807D0012809D0AE221BA145A0FFF788
:1020F0004BFBE8E79D2218A149A0F8E701F02AFA76
:102100004C49FFF779FA4C4810220C180021684618
:10211000A84769460C70200A4870200C8870200E71
:10212000C8702346A9220CA144A0FFF72DFB6A46E4
:1021300001213046F3F7F0FAC5E7B62206A146A022
:10214000FFF722FB102200216846A8476946304667
:10215000F3F769FBB7E700006170705F6761706358
:102160002E6300003C25732C25643E626F6E645F15
:102170007265715F696E64287265713A2564290D14
:102180000A000000750F00003C25732C25643E50AA
:10219000414952494E475F52455128617574683A2A
:1021A00030782558290D0A003C25732C25643E0003
:1021B00025303258200000003C25732C25643E4C0D
:1021C000544B5F455843482873697A653A2564291A
:1021D0000D0A00003C25732C25643E49524B5F4597
:1021E0005843480D0A0000003C25732C25643E54DA
:1021F0004B5F4558434828747970653A2564290D2A
:102200000A0000003C25732C25643E544B5F4B456F
:10221000595F454E5452593E3E3E0D0A00000000A3
:102220003C25732C25643E544B5F4F4F423E3E3E4F
:102230000D0A0000A0BB0D00A08601003C25732CF8
:1022400025643E544B5F444953504C41593A253024
:1022500036640D0A000000003C25732C25643E43C3
:1022600053524B5F455843480D0A000030B50D46A8
:102270004C7A0A7A87B0C988A888059402AC07C44A
:1022800069882888019100901B0A34220B490C4868
:10229000FFF77AFA362209490AA0FFF775FA0024F7
:1022A0002819817A09A0FFF76FFA641C062CF7DB66
:1022B0000848FFF769FA07B030BD00006C25011827
:1022C000505B01183C25732C25643E0025303258A4
:1022D000200000008426011870B51E0A0D460B88E8
:1022E000FF220C321BA11EA0FFF74EFAFF220D3277
:1022F00018A126A0FFF748FA00242819817825A004
:10230000FFF742FA641C082CF7DB24A0FFF73CFA25
:102310002888A91C00F040FA04000BD0FF221332D9
:102320000CA11FA0FFF730FA224610213046F3F728
:1023300062FB70BDFF22193206A120A0FFF724FA2C
:10234000002211463046F3F756FB304600F078FB8A
:1023500070BD00006170705F676170632E63000084
:102360003C25732C25643E656E63727970745F72D0
:1023700065715F696E6428656469763A30782558BE
:102380002C72616E64290D0A000000003C25732C3C
:1023900025643E0025303258200000000D0A000060
:1023A0003C25732C25643E2D3E46696E64205361A6
:1023B0006D65204C544B0D0A000000003C25732C29
:1023C00025643E2D3E46696E642044696666204C55
:1023D000544B0D0A000000007FB5574E1C46851B6C
:1023E0001B0AB04274D011DC544E851BB0423BD066
:1023F00007DC534D451B1BD0012D22D0022D11D1DE
:1024000023E00C2D41D00E2D0CD154E0062D6BD0C5
:1024100004DC022D60D0042D04D161E0082D72D0BF
:10242000192D78D00346FF227A3246A148A06FE0EA
:10243000487800900B782B224CA14FA0FFF7A4F90D
:1024400076E02346FFF712FF72E00C468978208879
:10245000019100901D46412244A150A0FFF794F93C
:102460002246294602200DE00C46897820880191F9
:1024700000901D464B223DA156A0FFF785F922464C
:1024800029460320FFF7CEFC52E01C46CA88888804
:102490000B884988019303920091029023465422AD
:1024A00032A15AA0FFF770F904230222012120462D
:1024B000F2F716F93CE088884A8809880192009171
:1024C00002905D2229A161A0FFF75EF930E0FFE7ED
:1024D0002346FFF7A9FD2BE02346FFF7C5FC27E0C5
:1024E0002346FFF7F9FE23E01D460C460B78FF223A
:1024F00023321EA164A0FFF747F922462946052092
:10250000C0E700E007E00B78FF222C3217A166A09D
:10251000FFF73AF90CE0CA888C884888098803924A
:10252000009101900294662210A167A0FFF72CF998
:10253000002004B070BD0000130700000307000076
:10254000000700006170705F676170632E630000B8
:102550003C25732C25643E556E6B6E6F77204D7352
:102560006749643A307825580D0A00006170705F41
:10257000676170632E6300003C25732C25643E4325
:102580004D505F455654286F703A25642C73746122
:102590003A30782578290D0A000000003C25732C7C
:1025A00025643E676170635F636F6E6E6563746917
:1025B0006F6E5F696E64286369643A25642C636892
:1025C000646C3A25642C726F6C653A2564290D0A97
:1025D000000000003C25732C25643E676170635F3A
:1025E000646973636F6E6E6563745F696E6428639C
:1025F00069643A25642C68646C3A25642C726561C0
:10260000736F6E3A30782558290D0A003C25732CDB
:1026100025643E706172616D5F75706461746528D8
:102620006369643A25642C696E764D3A25642C6999
:102630006E76493A25642C6C6174653A25642C7475
:10264000696D6F3A2564290D0A0000003C25732C42
:1026500025643E706172616D5F757064617465645C
:102660005F696E64286369643A25642C696E7476C8
:102670003A25642C6C6174653A25642C74696D6F1D
:102680003A2564290D0A00003C25732C25643E651B
:102690006E637279705F696E6428617574683A253B
:1026A00064290D0A000000003C25732C25643E734C
:1026B000656375726974795F696E642861757468A1
:1026C0003A2564290D0A00003C25732C25643E6CD4
:1026D000655F706B745F73697A655F696E642863A8
:1026E00069643A25642C7478423A25642C747854D1
:1026F0003A25642C7278423A25642C7278543A2533
:1027000064290D0A00000000032210B55202801A4D
:1027100004D0A42813D0A5281DD116E008780128DC
:1027200007D0032807D0A02815D34978FFF792FADD
:1027300011E0002000E00120FFF758FB0BE00A78D1
:1027400048781146FFF79EFA05E00B788A784878BA
:102750001946FFF79FFA002010BD00000EB50B4888
:102760000090032080026946088109480190001406
:102770004881684602F042FD02F044FD02F057FD38
:1027800002F003FD0349042008600EBD004E002046
:10279000005A002000E100E00020704770477047B9
:1027A00070B50A22094B0D460C2805D20446024694
:1027B00007A12846984707E005A1284698473220F8
:1027C000A8723620E8720C24204670BD190F000054
:1027D0006D79426C652D55617274000003210170A2
:1027E0000021417081701022C2700171012242717A
:1027F0008171704710B500210846F3F772FE002082
:10280000F3F756FF00F092F800F044FB10BD000013
:1028100001490870704700006232002010B5084B73
:1028200000218A008458D2181460491C2629F8D344
:10283000BFF35F8F03488360BFF34F8F10BD00006D
:102840000030002000ED00E070B51E4CB62160881D
:10285000261D091A89B2301800F0ECFB002500286B
:1028600006D06188081880B26080B6281DD308E0C1
:102870006088002819D06078411C6170142814D930
:102880006570114908780328307802D0AA2815D03D
:1028900016E0AA280AD053280DD00A4A4878121DFB
:1028A000618800F009FB00280AD070BD25704878C7
:1028B00000F0C6F804E00120207001E000F0F4F818
:1028C000658070BD9C300020623200207CB51446CB
:1028D000154A054610885688801C83B2002032466F
:1028E000C240D20703D0A34206D09B1C9BB2401C1F
:1028F000C0B20928F3D3092000290ED109280DD22E
:1029000001A900F039F8002808D0009068468388B3
:1029100022460021284600F097F97CBD002003469E
:10292000224680210090F5E76432002038B500216E
:102930000E4800910180FF211E31418000200324B8
:102940000A46C240D20706D0430022465B1C9A408A
:10295000009B1A430092401CC0B20928F0D3044BDC
:10296000044A69460148F3F7E5FA38BD64320020AD
:10297000CD2801184859011810B504460022104608
:102980002300FEF711FF090615090C0F1515151286
:102990001500052209A00EE009220AA00BE005227D
:1029A0000BA008E006220CA005E007220CA002E024
:1029B000142A00D914220A8010BD0000424C45356B
:1029C0007800000031312E302E322D4C45000000B1
:1029D000312E302E3000000031312E302E320000EA
:1029E000025E04400000030010B50446C1B200209E
:1029F00000F0AAFB204610BD10B5002903D0012924
:102A000006D0002010BD19461420FFF7C9FE10BDE6
:102A100000201880022010BD30B58BB00C46054652
:102A20002C22064B00216846984708A80472694684
:102A30002846F1F775FD0BB030BD0000750F0000A2
:102A400010B503221321F1F738FD10BD70B505460E
:102A50000E463520202303220621400100F04CFEC3
:102A60000446A02020701C22044B65703146201DB6
:102A70009847204600F059FE70BD0000190F000075
:102A800010B504463520022303220621400100F040
:102A900033FE042C01D3A82100E0A721017044706B
:102AA00000F043FE10BD000010B5012303220621F3
:102AB000034800F021FE0121017000F036FE10BD38
:102AC00001060000FFB515460E46074681B02323D8
:102AD00003220621084800F00FFE0670477045806B
:102AE0000446064B2A46001D04999847204600F0EC
:102AF0001CFE05B0F0BD0000A6060000190F000086
:102B000070B50E4605462A2303220621154800F01B
:102B1000F3FD03210170297841706978C176A98895
:102B2000C1840446A97820300172A97841727C21C1
:102B3000618445210901A184002E0CD0707980099F
:102B4000032803D1A07E01210843A0760622064B6C
:102B50003146201D9847204600F0E7FD0449034810
:102B6000086070BD01060000190F0000FD4100184B
:102B700050910020F8B5064617460D4635203A23F9
:102B800003220621400100F0B7FD0446A420207076
:102B9000044B66702A463946A01C9847204600F030
:102BA000C4FDF8BD190F000008B56A461180002168
:102BB00091700421FFF7DEFF08BD10B504463520F3
:102BC000022303220621400100F096FDA521017099
:102BD000447000F0AAFD10BD70B50E4601021C46FF
:102BE0001546062303220648491D00F085FD467060
:102BF000458084804221017000F097FD70BD000087
:102C000011050000F8B50F4611461E4608318BB27B
:102C100001021546512003220001491D00F06CFD00
:102C2000044612202070A780E580002E05D02046A3
:102C3000044B2A46314608309847204600F075FD7F
:102C4000F8BD0000190F0000F8B50F461D46991D8C
:102C50008BB20102164603220A48491D00F04CFDC2
:102C600047704680044685804020207006980028E2
:102C700004D00146044B2A46A01D9847204600F088
:102C800054FDF8BD11050000190F000070B50D4688
:102C900001021446042303220548491D00F02CFDBF
:102CA000457044804121017000F03FFD70BD00007F
:102CB0001105000000201349884700F041F800F09A
:102CC0002FF810490A205A3988470F484169890965
:102CD0008901223141610B488C388047044600F05D
:102CE0008BF9214609A0FEF74FFD2046FFF736FD80
:102CF0000C20F1F7D8FA62B600F046FF00F046FA71
:102D0000FAE70000D10800004010034053746172DC
:102D1000742872736E3A2558292E2E2E0D0A000043
:102D200001208007826A80218A438262026A0A4304
:102D30000262026A8A430262826A0A4382627047BE
:102D400001208007C16A0322D2021143C1620A48EE
:102D50000168082211430160026801210A430260F0
:102D600002688A4302600548026902239A430261AD
:102D700002690A43026170474000004000000340BE
:102D80000121890708690007000F022805D00428DF
:102D900005D008280DD0042070470020704708692E
:102DA000C00501D50220704748680128FBD00320E8
:102DB00070470520704710B5002000F0CFF910BD16
:102DC000FEB50C46324906460878101AC5B20846C8
:102DD00047887000002C09D0012C1BD0022C46D053
:102DE000032C02D10879401C0871FEBD032D07D0C9
:102DF00000200346802100903046FFF725FFFEBDEE
:102E0000C740B807800F6946888001A802230021C7
:102E10000090F1E71C46052D02D0032D0DD024E0D3
:102E20006078002803D100213046FFF72FFF61882A
:102E300030466268FFF7BFFFFEBD6378002B14D1F8
:102E40006388022B11D163685C781D7823022B43C1
:102E5000022B0AD803248440A74383401F434F809A
:102E600000213046FFF712FFFEBD8021F9E7002167
:102E70000B46052D06D0032D07D003213046FFF762
:102E8000ABFEFEBD01235B02F8E70223F6E700007C
:102E90005C32002010B50548002101800522027136
:102EA0004180034B034AF3F745F810BD5C32002024
:102EB000C12D0118AC59011870B58924002917D00B
:102EC0000C4D2B79002B13D06B884400E3409B07FB
:102ED0009B0F0CD02B8800249B1C9EB213460A46E5
:102EE0003146FFF78FFE2879401E287100E08A24C2
:102EF000204670BD5C320020F0B5364C87B0A0682B
:102F000081B235480818A060354D3448E86335492A
:102F100010208860344FB8693449884257D16E46D2
:102F2000002001A98200D3191B68401CB350062859
:102F3000F8D308690A22431C002B25D0134683438B
:102F400022D1A3681F263605C005C00EB343000575
:102F50000343A360E86B0B8A400940019B04DB0E2E
:102F60001843E863A0680E690F231B04B603360FED
:102F7000984336043043A060E86B98430B699B028A
:102F80001B0F1B041843E863C868194B441C05D089
:102F90001446844302D18005800E18610868441CE1
:102FA00008D0824306D15A69800592099201800EA9
:102FB00002435A618868411C09D0002807D00D4B94
:102FC000D9697C22800A914310400143D96107B03E
:102FD000F0BD0000000003400000B10114037400C4
:102FE0000010034000100040000F0018B6D5F5C8CF
:102FF0004010034040C0024010B5042203210020CD
:1030000000F06AF803228B21002000F037F811232A
:1030100014222121002000F049F8044800214180B9
:103020000180012002490003086010BD56310020D4
:1030300000E100E030B5104C054620886288801A17
:10304000FF300130C3171B0E1B181B0A1B02C01ACE
:1030500080B2884200D9084600280BD0002306E041
:10306000A1180979521CE9545B1CD2B29BB283426D
:10307000F6D3628030BD0000563100200A4B0003B9
:1030800010B5C0180023C360C36880242343C36005
:103090008160C168A143C160C16907231943C1614F
:1030A00020210A43C26010BD0030024010B5084C18
:1030B00000030019C1618261A415C168002A01D012
:1030C000214300E0A143C16002498162436210BD17
:1030D00000300240FF0F000030B5FF24174B823450
:1030E0009500ED182C60A1248900CB181C604300CA
:1030F0008024134D234349190B60114621430F4C83
:10310000C300803C1B195960E105CC6A0123C01C37
:1031100083401C43CC62486A18434862486A98431B
:1031200048620920074B03E05969D140C90704D11F
:103130000146401EC0B20029F6D130BD002100403A
:103140000020004000000140034A00038018026A8A
:103150009206FCD541607047003002400A4B0003E4
:10316000C01805E0036A9B06FCD513784360521C27
:103170000B46491E89B2002BF4D1016A8906FCD5A1
:10318000016AC905FCD470470030024010B5FFF752
:103190005BFB07480178032909D106490978002912
:1031A00005D0044A4078121DB621FFF785FE10BDF8
:1031B000623200209C30002010B5554C0021208840
:1031C00000280DD000F097F91F21081A2188C0B2FD
:1031D0000122824091432180DF21C001C9004118B2
:1031E000084610BDDF21C90010B5401AC109EFF330
:1031F000108072B6464A138801248C402343138002
:1032000080F3108810BD70B5414C00206188002902
:1032100012D0084600F06FF91F21081AC1B2C80089
:103220000019EFF3108272B6638801258D40AB431D
:10323000638082F31088183070BD364910B540188D
:10324000C109EFF3108072B6314A538801248C40D3
:103250002343538080F3108810BD70B52C4C0020A0
:10326000A188002914D0084600F045F91F21081A4A
:10327000C1B2182097224843D2008018EFF3108281
:1032800072B6A38801258D40AB43A38082F31088DA
:1032900070BD972210B5D2001821801AFEF7ACF944
:1032A000EFF3108172B61A4CA288012383401A43AF
:1032B000A28081F3108810BD10B5154C0021E08864
:1032C00000280FD000F017F91F21081AE188C0B2BA
:1032D000012282409143E180820000211219518134
:1032E000401CC1B2084610BD094980004018001DAD
:1032F000704759210901884202D3401A800900E031
:10330000401E034AD188012383401943D18070476E
:103310007091002008F4FFFF01460020096802E0D8
:103320000968401C80B20029FAD170470268002A5F
:1033300005D042681160416000200860704701605C
:10334000F9E70368002B05D043681960426000204C
:10335000106070470160F9E70268002A00D14160FF
:103360000A600160704702460068002804D00168C6
:103370001160002900D15160704710B50024234628
:10338000026805E08A4201D1012405E01346126873
:10339000002AF7D1002C07D00A68002B06D01A604B
:1033A00042688A4200D14360204610BD0260F7E7C0
:1033B000002906D013680B604368934200D1416036
:1033C000704703681B680360F6E71368002905D09F
:1033D0000B604368934200D1416070470360F8E797
:1033E000F7B50F4606460025046814E0204602990A
:1033F000B84700280DD02068002D01D0286000E0DB
:1034000030602068002802D00020206005E0756050
:1034100003E025462468002CE8D12046FEBD10B408
:103420000C000ED00023016801E00B460968A142A0
:1034300001D00029F9D1002B03D01A60116010BC13
:10344000704710BC114687E70B000DD0016800E003
:103450000968994202D00029FAD105E0002903D079
:103460000B68002B02D002E011465FE7426008685B
:1034700010600A607047F7B504680E4607460025DD
:10348000002C08D0029A214630469047002803D1EC
:1034900025462468F4E77E603460002D01D02E605C
:1034A000FEBD3E60FEBD0000410855221140401A9D
:1034B0000246332180080A40084010180109081804
:1034C0000007000F70472021020401D01021104690
:1034D000020201D010460839020101D01046091F2E
:1034E000820001D01046891E420001D01046491EBC
:1034F000C00F081A70472021020C01D0102110467D
:10350000020A01D010460839020901D01046091FED
:10351000820801D01046891E420801D0881E7047DB
:10352000081A70470021425C002A01D00020704731
:10353000491C0629F7DB0120704710B50022835C87
:103540008C5CA34201D0002010BD521C062AF6DB81
:10355000012010BD0549064A08685043054A8018F5
:10356000086040087047014908607047C892002011
:103570006D4EC64187D61200F3B5C01C00248508E5
:10358000AD002D1D81B0264627460C2D00D20C25FE
:10359000EFF31080009072B6029802213018FEF707
:1035A0002BF80806810D4F482A46081880690C320E
:1035B0000EE04188A9420AD3914202D28368002BCF
:1035C00005D0002C02D063888B4200D904464068A5
:1035D0000028EED1002C03D06088904200D205462E
:1035E000761CF6B2022E02D2002CD5D001E0002CBF
:1035F0000BD06088A8420CD1A16860684860606800
:1036000000280AD0A168816007E03748F8F796FDE6
:1036100007E0401B80B26080041965803348208039
:10362000271D009880F310883846FEBDF0B50023B2
:10363000021F2F49118054881946EFF31085AC46BC
:1036400072B69D00274E5F00AD19AD69BE19368C6C
:10365000A84204D3AE19864201D3294601E05B1C7F
:10366000DBB2022B01D20029EBD00020214B2DE050
:103670004D886D18954211D14888001982B24A8050
:1036800048685318984228D14388D2184A80426823
:103690004A604068002820D081601EE08A4213D230
:1036A0004260906010191380884209D148685060C8
:1036B0004868002800D082604888001950800CE0DB
:1036C00051608A60548008E0084649680029CFD1DB
:1036D00042605160906054801380604680F310888F
:1036E000F0BD0000F88F0020F2F2F2F23883000003
:1036F0000FF000005AA50000F8B504460F46184622
:103700001D46164601210C30FFF736FF0021C94344
:1037100001608480C780068145810C30114B0446CE
:103720002A46002198472046F8BD10B501460C39BD
:10373000EFF3108472B60C48FFF7F8FD0B480168F0
:1037400008221143016084F3108810BD10B50023D6
:10375000FFF7D2FFFFF7E9FF10BD03460C3BD9800E
:103760001A81E2E7750F0000F88F00203C900020DE
:10377000F8B50C460746010AC0B2082822D21A4AF8
:10378000800012580020904700281BD00178A142E9
:1037900018D004701548164D082600903A46154971
:1037A0000098FFF71DFE01000CD0EFF3108472B6F5
:1037B0000E480838FFF7BAFD28683043286084F3C4
:1037C0001088EBE7F8BD10B5010AC0B2FF24082845
:1037D00007D2054A8000125800209047002800D0E8
:1037E0000478204610BD00001C90002000900020AE
:1037F0003C90002069670018F0B50746414885B045
:1038000015460E46824201D9054602E0002D00D140
:103810000A253A043D4832433B490490FFF7E0FD56
:10382000040006D101211020FFF7A6FE8780044680
:10383000C680EFF3108672B602A800F092F986F304
:103840001088029800907D200399000145436D186F
:1038500001912F492846FDF7CFFE2D492D4A4143BE
:10386000691AE1600099081800010009A06021466A
:103870000498FFF700FE254810380069A04203D1E4
:10388000C168806800F0A3F8E168A068F2F780FFE3
:10389000002802D0042000F03FF805B0F0BD70B55C
:1038A0001A4C0246103C2569002D29D0AB881748D8
:1038B00093421AD1EB888B4217D1FFF754FD24694C
:1038C000002C0DD0E168A06800F081F8E168A068E4
:1038D000F2F75EFF00280ED0042000F01DF80AE089
:1038E0000021481E00F073F805E012040A4306495F
:1038F000FFF776FD0546002D02D02846FFF796FE1D
:1039000070BD0000FFFF7F02FB67001808900020D9
:1039100071020000D367001810B5EFF3108172B682
:103920000A4B1A680124844022431A6081F31088EC
:1039300010BD10B5EFF3108172B6044B1A68012464
:103940008440A2431A6081F3108810BD3C9000208F
:103950000A49002804D048694004400E18307047D6
:1039600008694004400E28307047002902D08000CA
:103970002C307047C000503070470000800000506D
:103980000521431C10220907002B06D0694B586201
:103990000A6288699043104301E088699043886116
:1039A000704710B50522441C20231207002C0AD0B2
:1039B00027242401611A5F4CA062E16213629069BE
:1039C0009843184301E090699843906110BD30B569
:1039D000EFF3108472B6451C052240231207002D18
:1039E0000AD027252D01691A524D28636963136295
:1039F00090699843184301E090699843906184F37B
:103A0000108830BDF0B5002084460120494EC00723
:103A1000B063B06BC00FFCD1B06B050146482D09F7
:103A20000088002845D145480068002841D101217F
:103A3000C90600220520000783697020034038D0A2
:103A40003F4FD80609D5706A401B04012409A01E07
:103A5000B8422ED28C4200D2214698060DD5B06ACB
:103A6000401B04012409A01EB84222D28C4204D279
:103A7000F06A214627221201121A580612D5306B1D
:103A8000401B00010009831EBB4212D2884209D8A4
:103A9000736B27242401E31A884201D3934201D295
:103AA00001461A46F06B80180A22800951434018DB
:103AB00084466046F0BD7FB504461020EFF31082C7
:103AC00072B61D4B1D8805431D8082F310881E4E63
:103AD0001C481D4D5C36002902D01022A84702E088
:103AE00010220021B047002C04D010222146684645
:103AF000A84703E0102200216846B0470D4800990E
:103B000040384163019981630299C163094A03996D
:103B100011604C2151600421052212071162936942
:103B20008B430B439361026B01218A430A43026377
:103B30007FBD0000C0000050F08F00203C900020AE
:103B4000FFFFFF0730810020190F000001200D4901
:103B5000C0078863886BC00FFCD1886B0001000927
:103B600070470121074AC9079163916BC90FFCD1C6
:103B7000916BD26B0901090927231B019A1A06C010
:103B800070470000C000005070B50B480088400727
:103B900010D40A4C20681F250AE0FFF7ACFC281A55
:103BA0000006800D00194068002800D0804720687A
:103BB0000028F2D170BD0000F08F00203C90002062
:103BC0001FB50220FFF7B5FE054B684610220349DA
:103BD000984769460020F2F7A3FE1FBD40810020F0
:103BE000190F000070B5EFF3108572B62048FFF78B
:103BF000BAFB040002D00020C043206085F3108887
:103C0000002C26D020464038808F1A49884220D187
:103C1000E088194B010A0006A288800D1B58104647
:103C20009847051E05D021460C312389E288A088DB
:103C3000A847002804D001280BD0022809D103E0AE
:103C40002046FFF7F3FC04E0094821460830FFF75F
:103C50006DFBEFF3108072B605490968002904D1A5
:103C600006490A6808239A430A6080F3108870BDE9
:103C7000F88F0020388300001C9000203C9000202A
:103C80007FB51C4D0420FFF754FE2C69002C30D06A
:103C9000EFF3108672B66846FFF763FF86F310886D
:103CA00001990098039102900146A0680122411AEF
:103CB000C91E09010909D20691420CD2E168FFF739
:103CC00086FEE168A068F2F763FD002811D00021AC
:103CD000481EFFF77CFE07481030FFF744FB044600
:103CE000C1888088FF22FFF731FD2046FFF79EFC48
:103CF000C8E77FBDF88F0020F8B50620FFF719FE52
:103D0000104E3588002D1BD0002401270CE03846CA
:103D1000A040284204D07088C1B22046F3F7E9FAE7
:103D2000641CE4B2032C02D270880028EFD13088E2
:103D3000002805D07088002802D00620FFF7ECFD8F
:103D4000F8BD00008C920020F1B582B00298F549D0
:103D5000800001900D582C468034207AA17A800092
:103D600040180299C0B20902009155E0708FB18FDE
:103D70008007800F012816D0022814D003283AD1DA
:103D80000846FFF786FAE8490198029B0858002880
:103D900006D0006A4268002A02D0417A184690474D
:103DA0000322009922E0708F000A042805D97E22A0
:103DB000525B520601D5001F80B200281BD06F6AEB
:103DC0000818FA88B9889205920D8918884212D38A
:103DD00028462430FFF7C7FAE86AB84201D100202C
:103DE000E862B888FFF729FA009902228320800050
:103DF000491CFFF7ABFC708F102188437087207B34
:103E00000421401E2073A07A401CFDF7F5FBA1722F
:103E1000207A80004018C0B2217B002905D0010122
:103E2000C2480E18308FC00BA0D14035E98F082052
:103E30008143207B002800D00120C0000143E98796
:103E4000FEBDF1B588B00898B64980000C58042131
:103E500025464035E88F8843E8870898000202909D
:103E6000E5E0B34B1C21987A4843B04980394018AB
:103E70000090478A818A01918907890F0391C18A3D
:103E80000026C9B20691216D0591E98F4904490CBC
:103E9000002F11D00022D2031143E987FA070DD079
:103EA000A4490878401C0006000E087003D018686A
:103EB0000028FBD08047B5E00122ECE79D4A0023B3
:103EC0001370CA0704D0428B008B16040643E664C5
:103ED000C80570D4FF2001300143E987C8070CD022
:103EE000A878012809D120462030817F002904D0FC
:103EF0000121C1770898F7F7EEF9A88E2887E88F97
:103F0000C00711D00098808B27218005800D090102
:103F1000081A04908D20005DFFF71AFD41000498F7
:103F2000401A00B2844908E0606CE064206509E052
:103F30004018761E360100B236090028F8DB688585
:103F400066642665E88F810707D402210843C2070B
:103F5000E887D20F0223029911E0C0071FD0206D1D
:103F6000410805984008081A216E00010009490817
:103F7000FDF742FB002912D002230299FF226E486E
:103F8000491C6238FFF7B8FB0646206D216E4008D9
:103F90004908FDF731FB31803046FFF7C6FBE88F5B
:103FA000410508D4810706D50199490703D50121A8
:103FB00089020843E887380734D4E06C60656620DE
:103FC00007422FD1F80607D5E88F80210843E887FC
:103FD00002208921085525E00198060A22D003987D
:103FE00000281FD0042E04D9E88F800601D5361F83
:103FF000B6B20098878C504802990823FF22663891
:10400000491CFFF779FB0780468003990171A98E4F
:10401000C180FFF78AFBE88F04210843E8870099F5
:10402000002088848F2106980855F6F7F9FF089834
:10403000F7F70EF8002800D013E709B0F0BDF8B587
:104040000F46384889004458002C3AD01300FDF739
:10405000ABFB0504043B3F463800154601212046D2
:10406000F8F78EFA8920005D022822D0FFF76EFD56
:10407000014620464030C28F930723D5530721D4F1
:1040800012071FD48278012A1CD00E22266E636C80
:104090009B191B011B096364C38E26465B1CC386E8
:1040A000002D01D0A27D521CB275C08FC20B3846C4
:1040B00033E04034E08F000632D53D213846F7F733
:1040C000B6F8F8BD1022E1E73846FFF7BAFEF8BDB2
:1040D0003846FFF739FE3846F7F7BEFAF8BDFFF766
:1040E00035FD054601212046F8F74AFA2046803082
:1040F0000146407A022813D0626C206E101802012B
:104100001209204640306264C28E521CC286A07DD5
:104110000022401CA075087A2946F7F716F9F8BD69
:104120001621CBE760910020909200208083002030
:1041300050910020D092002071020000F1B590B0A3
:104140001098002780000B90E8E0EB481C21807A53
:104150004843EA494518688A3D21084206D1A88AA1
:104160000007000F052802D0032877D0D4E0A98CDF
:104170006846E34B2222E34CC918A0476846428BAD
:10418000E14910460A388842F0D86846C08A0628B5
:10419000ECD31921C9018842E8D86946098BFF236D
:1041A000F4339942E2D8491C414390008142DDD268
:1041B000A88A69464006C00F0D90062209A823462A
:1041C000984709A80D99F4F701FC0028CED12C23BB
:1041D000FF220021CD48FFF78FFA0746041D688BA8
:1041E000298B00040843A98B272289050C90890D8F
:1041F0001201E88A561A800BFFF7AAFB4000301A1A
:10420000C24906B26B3106E0701806B20C98401E27
:10421000000100090C90002EF6DB10983870002089
:1042200078700120F8702070B9490B980858808E7A
:10423000C00607D5A88A8006C00F05D0AE48C07A50
:10424000400701D5012000E00020E0730B980858DA
:10425000018F002903D02030807E01E042E0002061
:10426000B87004222046A74B103003A998470322B8
:104270002046A44B193004A998476846C17C2046C3
:1042800020300E9001716846808A60846846C08A3A
:1042900020816846008B60816846408BA0810522A2
:1042A0002046984B143007A9984708A84078062262
:1042B000C1060E98C90E417108A84078914B40097B
:1042C000A07309A9A01C98470D9860700C98E06134
:1042D0002684E88A810B0E9881713846FFF725FA0B
:1042E000012719E08A490B9808582030407F0028A0
:1042F00012D0A98C6846824B0C22824EC918B04756
:10430000A88A69464006C40F062203A8B04703AA3C
:1043100021461098FBF757FBF6F782FE1098F6F748
:1043200097FE002800D010E7384611B0F0BDFEB56A
:10433000064677488B00C458002C41D00027002A3D
:1043400016D0012A14D0022A3AD0042A38D12546A0
:1043500008462035297F02297CD001212046F8F724
:104360000FF9A08E000776D5A07D401CA075B3E0A4
:104370000091019201212046F8F702F925462035E7
:10438000A87E401CC0B2A876297F022904D0218FC4
:1043900000290BD0884209D3218F002903D08842FD
:1043A00001D3432200E00022012106E0E87EFFF76E
:1043B000C5FE002805D0002211460098F9F7E8FE56
:1043C000FEBDA08E400711D42A78002A05D0012313
:1043D00000210098F9F70EFF2F706A78002A05D0A7
:1043E000012319460098F9F705FF6F70A08E49491F
:1043F0000007019813D5002802D0A07D401C00E0E2
:104400000A20A075A182606A6660E0602046F7F726
:10441000BEFF002801D12F77FEBD3C22C4E7002853
:104420001AD0A06A301A0201E06A120940008242E2
:1044300002D3A07D401CA075A662E87F002802D0B0
:104440006068B04202D0606A401C08D0A182616AF4
:10445000E16006E031E032E00522A275ECE72E498A
:10446000A182FFF777F81121FDF7C6F84804E97F2C
:10447000000C002907D0002802D0202802D002E03A
:10448000012000E01F20E16A490089190818010194
:10449000090920466160F7F77AFF0028BBD0E87F62
:1044A000002803D00021C94361602F77606A411C56
:1044B000B2D0E1688142B0D0FEBD002219E0A06A0E
:1044C000301A0101E06A09094000814204D3A07D4D
:1044D000401CA0756168A1622046F7F758FF0028CC
:1044E00099D0E87F0028E7D1606A401CE4D0E87EDC
:1044F0003C22012162E7000050910020008300204F
:1045000000800020190F0000760C00000602000059
:10451000A092002001A0000001600000F0B5810021
:10452000B54889B0006841580591407A8006000E70
:10453000203103910890D8E0B0481C21807A48438C
:10454000AF494518A88C00900598AE4A408E90421D
:104550007ED8688A3D220290104001D0102877D181
:104560000020059C01903E3406900490FF2703989C
:10457000012207944277A88A0607360F072E44D2F5
:104580000027042E0CD1A04900984018211DFEF7E9
:10459000D4FF002812D00398407E062811D01B2794
:1045A00024229A4B002120469847012E0BD0002E42
:1045B00011D0022E11D0062E11D011E0FF20A075CF
:1045C0008FE01A27ECE7A88A15270006C00F20768F
:1045D000062001900BE0132702E0102700E01227CD
:1045E00006200690A88A000A801FC0B2049000200E
:1045F000A075677560760421A176A0747F20E076AF
:10460000A88A4006C70FE77502E0A07DFF2868D0A2
:104610000298C00607D5607D4007CFD57648006870
:10462000407C0128CAD9607D15281ED1019A0099C5
:10463000754B891889B2C9182046744B0A30062276
:104640005C3B9847688A4006C00F00D0012000E01C
:1046500049E06070688A4006C00F06D1207E0028BD
:10466000ACD0E07B80090328A8D0FF2F12D0664988
:104670000098231D41181846644B06225C3B98475E
:1046800002980006C00F2070288C60800298C00637
:10469000C00FE0742423FF2200215D48FFF72CF8AF
:1046A0000746E88A2077594B242238465C3B079915
:1046B000984704987877049800280BD0009838849D
:1046C0000698B8774D481C22807A002150434C4A06
:1046D0008018818448480068407A38753846FFF76A
:1046E00024F803984676F6F79BFC0398007DF6F7CE
:1046F000AFFC002800D01FE7089801014048803037
:104700000818018FC90B03D0018F4904490C018798
:1047100009B0F0BDF8B5044637480068002832D02B
:104720008B00C05800282ED00027002A13D0012A61
:1047300011D0022A46D0042A25D10446FFF706FAF2
:10474000214605462031087E02283FD000200F7602
:10475000002816D13CE01646024620300091017E2A
:10476000057D022904D000210776002904D10BE041
:104770000121F9E7F6F754FC2846F6F769FC002812
:10478000F8D1F9F7B7FFF8BD01211046F7F7F8FEA9
:10479000702045431F482818418D4905C90F04D092
:1047A000418D01229202914341850098FFF7B6FEA8
:1047B000002E01D0012200E0002221460098F9F7E6
:1047C000DEFFF8BD0846FFF7A9FEF8BD0120BEE7F1
:1047D00001212046F7F7D4FE606A281A0101A08D56
:1047E00009094000814203D3A07D401CA075656289
:1047F0002046F7F7CCFDF8BDB09200205091002084
:10480000008300207206000000800020750F000069
:104810000102000040810020F0B58100CB4887B044
:104820000568685802902030019060E0C8481C215B
:10483000807A4843C7494418608A3D21084253D1D1
:104840002E462036307E00284ED1A08AA18C00074B
:10485000000F05910121019A0028917501D00128CE
:1048600042D1A08AE18A000A890B0091618B0A0477
:10487000218B0A430492A18B27228905890D1201FD
:10488000511A22300391C0B20099FFF76EF8074623
:104890000098FFF75DF8381A039940004018AE49B8
:1048A000FF304A1E2D308018FCF7A6FE049A8018AF
:1048B00000010009E863208CA886A08A8006C00F4A
:1048C00000D00120402148550098B075A34B0599B0
:1048D0000298C9180622A24B2E309847A08A40069B
:1048E000C00FE87601203076F6F79AFB0198007E3B
:1048F000F6F7AEFB002899D107B0F0BDF0B5810006
:10490000924889B0056868580690287D2F46800631
:10491000000E20370590387E00287DD005980101D3
:104920008C4880300818008FC00B75D041202C2394
:10493000FF220021C000FEF7DFFE0490041D069850
:10494000B97D0A2220305143007E4E197021484320
:1049500084494018808C80000790E86B0190708932
:1049600041000198401A3189000189000009029133
:1049700008360391FCF740FE08460399091A01988E
:1049800008180101090901980091081A0101079806
:104990000909814205D200990298401800010009D6
:1049A000009000202070E87E0622C007C00F6070D3
:1049B0000699A01C6A4B2E319847294604221C31C7
:1049C0002046674B1030984730882081708860847B
:1049D0002946052215312046614B1430984704982A
:1049E000317A41702046B97D203001908171B088C4
:1049F0006081F088A08103222046594B3946193046
:104A000098470198F978017101983979417178795D
:104A1000A0730098E06100E00DE04020405DE0738D
:104A200004980121C1700498297D01700498686080
:104A3000FAF756F901E0002038760598010145485B
:104A400080300818018F4904490C018709B0F0BD76
:104A5000FEB53E4B05461868002833D08C0000593F
:104A600000282FD00027002A13D0012A11D0022AB3
:104A700052D0042A26D10446FFF768F8214605469D
:104A80002031487B02284BD000204F73002817D1DB
:104A900048E016460246203000950191417B057E94
:104AA000022904D000214773002904D10BE0012121
:104AB000F9E7F6F7B5FA2846F6F7CAFA0028F8D16A
:104AC000FAF70EF9FEBD01211046F7F759FD7020E7
:104AD0004543244840382818418D4905C90F04D062
:104AE000418D01229202914341850198FFF794FE86
:104AF0000198FFF703FF154800680028E2D000592D
:104B00000028DFD0002E01D0012200E00022009911
:104B10000198FAF72CF9FEBD0846FFF77DFEFEBDB1
:104B20000120B2E701212046F7F72AFD606A281A22
:104B30000101208D09094000814203D3A07D401C62
:104B4000A07565622046F7F722FCFEBDB4920020F6
:104B5000509100200083002071020000008000209E
:104B6000190F000080810020F8B505252D07EC699C
:104B7000534EA00726D502202862A96B514C3E2037
:104B80006268521853085F00D21B4143CF184E4948
:104B900038466260FCF730FD4C4906434E604A4A95
:104BA0005043381A521E101A08600B202863012047
:104BB000A861801E286221880820014304208143C7
:104BC0002180F8BDE00737D0012028620020A861CD
:104BD0003F49E9603D4B80339E63996BC90FFCD11F
:104BE000996B3C4E0A01374912094988CF0607D50F
:104BF0005F6AD71B3F013F09B74201D210273843F4
:104C00008F0607D59F6AD71B3F013F09B74201D2E4
:104C1000202738434F0607D51B6BD21A1201120901
:104C2000B24201D240221043264A8143A96113882F
:104C300008218B4313800443E00606D51020286228
:104C4000A9698143A96100F01FF9A00606D52020BB
:104C50002862A9698143A96100F040F8200404D5C5
:104C600000F08EF80120C00328621B49600608D5B9
:104C700040202862AA698243AA6108681022104372
:104C8000086060070CD504202862AA698243AA61E3
:104C90000C4A13881026B34313800A6802430A6043
:104CA000200706D508212962A8698843A86100F079
:104CB00057F82869C00384D5012000046861F8BD55
:104CC00000000080F08F00207102000040000050C2
:104CD0001E000100000000083C900020FEB5274D9A
:104CE00068462C68FEF73DFF0126F6062F460C3776
:104CF00016E0E17D6068401A0099401A401C0001EE
:104D00000009B04224D200281ED002280AD81B482D
:104D1000FEF729FBA8608169002900D088472C682C
:104D2000002CE6D1386800280BD0082105200007A8
:104D3000016282698A430A4382610168B143314357
:104D40000160F7F7F4FAFEBD0198A1688842DED948
:104D50000A48FEF708FB01463846FEF7E7FADEE7A9
:104D600010B5064C0C342046FEF7FDFA002804D09E
:104D7000C1690029F7D08847F5E710BDB891002038
:104D8000F8B505200007416A0801040F0E0F3B48E3
:104D90000A0701D5032202E0CA060BD50222A500AC
:104DA0004359002B05D00119803128180978006C6F
:104DB0009847F8BD314D4A07314B01278035002A0D
:104DC00031DA298AB74039421BD03201D11809881B
:104DD0008906490F062914D1B40003590422002B77
:104DE00005D08119803120180978006C9847A87C7B
:104DF000B04203D1401C0007000FA874288AB843B2
:104E00002882288A002808D0411E0842D1D1A87CD7
:104E1000401C0007000FE874F8BD1A4801882022E2
:104E200091430180F8BD8907FCD52201D11809887A
:104E30008906490F042911D00022A6008359002BAE
:104E400005D00119803130180978006C9847288AFC
:104E50003946A14088432882E97C04E00122ECE73E
:104E6000641C2407240F3A46A240104201D1A142FB
:104E7000F6D1AC740028D0D0F8BD0000CC91002051
:104E800000800020F08F0020F8B5012700250E4E8D
:104E9000FF06FEF75BFE3468002C12D06168401AF2
:104EA00000010009B8420CD20748FEF75CFAA1687D
:104EB000002901D020468847002DEAD0FAF7D4F91E
:104EC000F8BD002CFAD1F8BDB8920020000A0628DF
:104ED00003D0072803D003487047034870470348AE
:104EE00070470000651E011809270118D923011811
:104EF0000246002003290FD2002A0ED0104BD11AEF
:104F00009A4219D00CDC0F49511813D00E4A891857
:104F10000ED0092900D10D4870470D484018704740
:104F2000E0290BD0E12901D0E229F8D109487047E6
:104F30000948704709487047094870470948704751
:104F400012070000F9FBFFFF02FDFFFF6347001897
:104F5000CC920020815C0018994500187746001813
:104F6000A75A0018A74600180246002000290FD1B2
:104F7000002A0ED035235B01D11A9A4213D00ADCE5
:104F80000C49511813D012290BD09E2900D10A4880
:104F900070470A487047062907D05229FAD10848B5
:104FA00070470848704708487047084870470848E5
:104FB00070470000FFF9FFFF31D40018D1920020A4
:104FC0004DFF001829F70018DDD20018F9F8001875
:104FD000F9F4001802460020032910D2002A0FD04D
:104FE00051231B01D11A9A421BD00CDC0E495118D7
:104FF00011D0FA2911D0FF39082900D10B48704788
:105000000B4840187047012909D0302901D03129B7
:10501000F8D1084870470848704708487047084862
:105020007047084870470000F9FBFFFFA1CE001849
:10503000D2920020FDCF001859D00018FBCB0018E9
:1050400001CF0018B9CE001801460D4B0020CA1A36
:10505000994210D007DC03290FD0FF39FF3903290B
:1050600000D108487047012A03D0032AFAD1064824
:10507000704706487047064870470648704700006A
:1050800005020000E90F0118BF1301188B0D01186C
:1050900019120118C10F011802460020042912D26A
:1050A000002A11D083239B00D11A9A4217D00EDC1C
:1050B000FF3A521E1BD0012A19D0062A15D0FF3AFA
:1050C0000C2A00D10B4870470B4840187047012943
:1050D00009D0022905D00329F8D1084870470848AB
:1050E00070470848704708487047084870470848A4
:1050F000704700005D140118D59200206FA80018B9
:10510000B31401184B8B001851DE0018CFDD0018C6
:10511000E1DE00180246002003290AD2002A09D045
:105120000849511809D0FF39FC3908D0012900D1AC
:1051300005487047054840187047054870470548BE
:1051400070470000F5FDFFFF9DF40018D992002084
:10515000DFF3001875F300181C490020C8601C49D3
:1051600025220A70491C0870401CC0B2491C0B283B
:10517000F9D326220A7002E00870401CC0B2491C14
:105180002528F9D327200870704710B51248114917
:1051900041631249020481631149C163816B032396
:1051A0009B059943114381630B480E4940300160D0
:1051B0000D4941600D4901610D494161EFF71EF84C
:1051C0000C48812101600C49416010BDD88F00203E
:1051D00000810020205000004000005040004000AE
:1051E00000E400E4550A5A0050065000051A030076
:1051F000070A030000900040B034E80310B500F047
:105200007BF810BD10B50F480024C169042211437A
:10521000C16111074A6A881302434A624A6A82439B
:105220004A62FFF799FF204600F012F810BD10B552
:1052300005490320F1F79FFAFDF736FC03490420E6
:10524000086010BD00000340CD4E011800E100E0F1
:1052500070B5064600F0B4F8304600F0FBF8304672
:1052600000F0A2FA304600F01DFA304600F0CEF908
:10527000304600F01DF905241A4D2407002E14D0E5
:10528000304600F085F800F037FA2068400040080A
:10529000E100084320602068C00FFCD11349124888
:1052A000086200202880686070BD11490220F1F773
:1052B000C5FA1048A0610120288070BD70B509486A
:1052C0000088C00701D0012400E00224EFF310851C
:1052D00072B600F033F82046FFF7BAFF85F3108866
:1052E00070BD0000F08F0020C8002C01C0000050ED
:1052F000C13B01180C80000070B5054624221F4CEC
:1053000000211D48A047202200211D48A04720223F
:1053100000211C48A0471B481B4901611B49002470
:105320004161A0002A586000401901892046F1F728
:10533000FDF9641CE4B2022CF3D370BD10B50E4825
:10534000FEF711F8002802D0FEF770F9F7E70A4CD3
:1053500008342046FEF707F8002802D0FEF766F969
:10536000F7E7054C10342046FDF7FDFF002802D07A
:10537000FEF75CF9F7E710BDF88F0020750F00000D
:105380001C9000203C900020E53B0118813C011856
:1053900010B5094C022808D12068002805D006481D
:1053A000FDF7E1FFFEF742F9F6E700202060034930
:1053B0006060087010BD00005C900020CF9200205B
:1053C00070B505001BD0012D11D0022D16D100247F
:1053D0002046F1F74AFB641CE4B2022CF8D3002407
:1053E0002046F1F75AFC641CE4B2032CF8D328469B
:1053F00000F0BEF900210620FEF7BAF970BD0E4993
:105400000620F1F7B8F900240C480E4B047028224E
:1054100021460B4898470C490720F1F7ACF90020CA
:105420000A4A0B4B3F2111548500401CC0B25C510D
:105430000328F8D370BD0000694F0118D1920020F5
:1054400064900020750F0000F14E0118CC920020EE
:105450008C90002070B5002400280ED001281CD0AC
:10546000022809D1F0F745FE00212046F1F730FE71
:10547000641CE4B2032CF7D370BD09490520F1F791
:105480007AF90020074A084B102111548500401C6E
:10549000C0B25C510328F8D370BD0448046070BDED
:1054A000D54F0118D2920020B4900020989000208F
:1054B00070B51D4D002829D0012817D0022824D10D
:1054C0001A4E002401212046F8F703FB1C206043FC
:1054D00080190069002801D0FEF7A8F8641CE4B226
:1054E000042CEFD300210420FEF7D9F903248422F1
:1054F00000210E48A8470D481B2140308187FF211D
:105500004931C18740300470447070BD08490020A3
:10551000F1F731F907490120F1F72DF910220021A7
:105520000548A84770BD0000750F0000CC90002012
:10553000495001189950011890920020F8B5FF25A4
:10554000052401352407022814D12068A8432060CF
:10555000206840004008E100084320602068C00F38
:10556000FCD1E060401E60613349086901221203EA
:1055700090430861314820603148E0602E4931484D
:10558000403108620026701C0621FCF735F81C200B
:1055900041433120000108188003010C1C203246D1
:1055A0004243294817183982FDF706FEB884761C55
:1055B000062EE8DBC420A0620020E062234E1F23F9
:1055C0001B027021414389194A8A07029A433A43D0
:1055D0004A82401C0428F4DB2068A843284320604A
:1055E000F8BD10B510221B4B002119489847FF2029
:1055F000174CF53020811848A0801848E080FDF74E
:10560000A9FF207316490020087010BD10B50400D2
:1056100010D0FFF7E6FF2046FFF790FF204600F08E
:10562000FBF8204600F012F9204600F023F920464E
:1056300000F018F810BD0000C00000500F06100068
:105640001E000100D902FFFF0083002040810020DE
:1056500050910020750F0000D6BE0000898E00001A
:10566000D092002070B50E4E02280FD10024A50064
:105670007059002806D021460420F7F771FA7059B6
:10568000FDF7D4FF641CE4B2042CF0D300200146E3
:105690008200401CC0B2B1500428F9D370BD000094
:1056A0006091002010B51149002808D010480880EA
:1056B0003F204880FF2088800F20C88010BD0D4B00
:1056C0000020C201C400D2186418401CA28306281E
:1056D000F7D3002059231B0182018400D2186418DB
:1056E000401C22810428F7D310BD000070910020D7
:1056F000FF030000F80B000070B51422144C0021C9
:105700001248A047942200211248A0470020124AC4
:1057100005461A2103019B181980401CC0B21028AD
:10572000F8D30E482022056045600D480021056031
:1057300045600C48A04700210A48C94301600A4857
:1057400001600A498180857170BD0000B891002018
:10575000750F0000CC910020008000206092002096
:10576000B89200206C920020C0920020E457000004
:1057700010B502280BD010220A4B00210848984788
:105780000748042118304171C171817110BD002496
:105790002046F7F789FE641CE4B2042CF8D3EFE747
:1057A0006C900020750F000070B50025002814D003
:1057B00001280DD002280FD10620FEF7BAF80024E8
:1057C00001212046F1F75FFD641CE4B2032CF7D3FE
:1057D0000C4805800621418070BD0B490620F1F779
:1057E0002DF80A490420F0F7C6FF0020084A094BAB
:1057F0003F2111548400401CC0B21D510328F8D32E
:1058000070BD00008C920020F93C01181551011860
:10581000D9920020C090002070B50B4D02280AD10B
:105820000324A0002858002801D0FDF7FFFE641EC5
:1058300064B2002CF5DA002001468200401CC0B2A0
:10584000A9500428F9D370BDA092002010B5084CCF
:1058500002280AD12068002807D00068002801D05B
:10586000FDF7E4FE2068FDF7E1FE0020206010BD9A
:10587000B092002010B50C4C022811D120680028ED
:105880000ED04068002802D00C38FDF7CFFE20680B
:105890000068002801D0FDF7C9FE2068FDF7C6FEAC
:1058A0000020206010BD0000B4920020260833A123
:1058B00001D20A010100B900032800000002000023
:1058C000292A000000021400032800000002000042
:1058D000242A000000021400032800000002000037
:1058E000252A000000021400032800000002000026
:1058F000272A000000021400032800000002000014
:10590000262A000000021400032800000002000004
:10591000282A0000000214000328000000020000F2
:10592000232A0000000208000328000000020000F3
:105930002A2A0000000208000328000000020000DC
:10594000502A0000000207000A180000B858011889
:1059500012000000160A1040D19F4C6CB455E3F7BA
:1059600000FF0000160A1040D19F4C6CB455E3F7BD
:1059700001FF0000160A1040D19F4C6CB455E3F7AC
:1059800002FF000003280000000200006459011813
:105990000030004002290000000A02000328000035
:1059A0000002000074590118000C004254590118FB
:1059B000845901180500400019520018D3520018EC
:1059C000C153001819540018595400189554001860
:1059D000D95400183355001863550018AF550018F6
:1059E000DB5500180328000000020000002A000018
:1059F000000220000328000000020000012A00002D
:105A0000000202000328000000020000042A000037
:105A1000000208000328000000020000A62A00007F
:105A2000000201000328000000020000C92A000053
:105A3000000201800328000000020000052A000087
:105A40000020040002290000000A0000397C001830
:105A50006D7C0018937D0018197F00186182001872
:105A6000EB8200188F830018AB800018B3840018F5
:105A70000000000027850018178600181BA40018D6
:105A800061150118178B00187794001821950018DC
:105A900087950018CB95001889E0001865980018C4
:105AA000F9980018E7930018359400182B8D00180A
:105AB00049E00018AF980018FBA400180FA60018C2
:105AC00069E000180000000000000000339C00188E
:105AD0009F9C00188BAD001817AE001879AE001807
:105AE0000C010801020F17070D050105010D020148
:105AF000090109010101010306010205090118015B
:105B00001801030500000000090109010301030158
:105B1000050100007F09011875010118AF01011886
:105B2000730201182F030118B5060118B5060118F4
:105B30009D070118B305011869080118000000004D
:105B40008D080118EF080118250901182509011809
:105B50003C25732C25643E676170635F636F6E6ED6
:105B6000656374696F6E5F7265715F696E642863E7
:105B700069643A25642C6368646C3A25642C636F0D
:105B80006E6E5B696E74763A25642C6C6174653A4E
:105B900025642C746F3A25645D2C6163633A256437
:105BA0002C63616464723A2564290D0A00000000C8
:105BB000D05B01189830002004000000C2170118C3
:105BC000D45B01189C300020CC010000D2170118D2
:045BD00000000000D1
:040000051800409906
:00000001FF
